:020000040800F2
:1000000000200010014C0308313603085B70010822
:100010002F3603082D3603082B3603080000000096
:100020000000000000000000000000002936030866
:100030002736030800000000253603081571010863
:10004000694C0308694C0308694C0308694C0308B0
:10005000694C0308694C03089D1B0008C91C000873
:100060008D1C0008511C0008151C0008A97C000804
:10007000997C0008897C0008797C0008697C00086C
:10008000557C0008417C0008694C0308694C030852
:10009000CD390308694C0308694C0308D91B0008D3
:1000A00021400108F5430108694C03087145010826
:1000B000394301087D420108694C0308694C030873
:1000C000694C0308694C0308694C0308694C030830
:1000D000694C03084D720108D1710108557101087E
:1000E0005F1B0008694C030815360308694C0308B8
:1000F000ED400108694C0308B5410108694C03084B
:10010000000000000000000000000000694C03082F
:10011000694C0308694C03081DB5020809B50208BB
:100120002D7C0008197C0008057C0008F17B000884
:10013000DD7B0008694C030800000000000000009F
:10014000694C0308694C0308694C0308000000006F
:10015000000000000000000000000000000000009F
:100160000000000000000000694C0308694C03080F
:10017000694C0308000000000000000000000000BF
:0801800000000000694C0308B7
:100188000A4B30B503F10C0493F900205D78072A77
:10019800C8BF143A811804338D7213F8025C855471
:1001A80013F8012C0A759C42EED130BD5451030856
:1001B80003682DE9F0415D6A1DB12B46BDE8F041A9
:1001C8001847002A174611DD04460E460F4400E082
:1001D80023689B68204698470028F9D0236816F8BA
:1001E800011B1B6820469847BE42F1D1BDE8F0814B
:1001F80003681B6918470023282202704370837024
:10020800C3707047437A5A1C0344D2B2427299723F
:10021800037A93420AD84AB110B5044604F10A0198
:10022800D0E9003098470023637210BD7047CB07B0
:1002380002D4024B024ADA60704700BF00ED00E0CA
:100248000400FA0520B10078B0FA80F04009704740
:1002580001207047037903F01803082B0AD002D84D
:100268002BB100207047102B16D0182BF9D1B0F8FD
:100278000B007047114BB0F80B0093F90030591C74
:1002880006BF0F4B1B78DBB2C3EB0312C3EB820331
:1002980000EB430080B27047084BB0F80B0093F9AD
:1002A80001305A1C06BF064B5B78DBB203EB4302F6
:1002B80003EB820300EB430080B27047000000208C
:1002C8005C290020F0B5067906F06003402B09D1BF
:1002D80044794FF0FF350023012006F00706A342BA
:1002E8000BD1F0BD602B08BF45794FF001040CBF5E
:1002F80004FA05F54FF0FF35EDE7042E0CD8DFE8DA
:1003080006F0030D18242E0030B1C85CD75C784085
:1003180028420CBF012000200133E0E70028FBD071
:10032800C856D756A0EB070CDCF1000040EB0C00D8
:10033800F2E70028F0D031F8130032F81370784053
:1003480028420CBF01200020E6E70028E4D031F95C
:10035800130032F91370C71B78427841DCE7002894
:10036800DAD051F8230052F82370784028420CBFA5
:1003780001200020D0E745E790ED057A90ED004A8E
:10038800D0ED066AD0ED014AD0ED047A90ED035A1B
:10039800D0ED025AA4EE007AB0EE406AB0EE470AF9
:1003A800B0EE667AA4EE867A67EEC07AA5EE407A59
:1003B800E5EE867A80ED057AC0ED067A7047D0EDD5
:1003C800057A90ED013AD0ED003AD0ED064A90ED6D
:1003D800024A90ED077A90ED035A90ED086AD0ED45
:1003E800045AC0ED067AF0EE406A27EE830AC0EDA3
:1003F800056AA3EEA60A80ED087AA4EE240AA5EE03
:10040800470AA5EEC60A80ED070A7047D0ED007AC4
:1004180090ED017A30EE670AE7EE007AB0EE670AEF
:10042800C0ED007A704770470378202B024600F130
:100438000100F9D0092BF7D02D2B00F0A4802B2B2D
:1004480003BF5378B7EE000A0246B7EE000AA3F1DD
:100458003001C8B209289FED577A10D8F2EE046A25
:1004680007EE901AF8EEE77A12F8013FE7EE267ADF
:10047800A3F13001C8B20928B0EE677AF0D92E2B63
:1004880063D003F0DF03452B02D020EE070A704744
:1004980010B451782D294FD02B2979D0A1F13003F0
:1004A800092B02F101027AD80024002303EB83030D
:1004B80001EB430312F8011FA1F130000928A3F151
:1004C8003003F3D9B3F59A7F1A4628BF4FF49A72CE
:1004D800072B6CD9DFED386A1346F7EE007A083B34
:1004E800072B67EEA67AFAD802F00702DAB1F2EE25
:1004F800046A012A67EEA67A15D0022A67EEA67A60
:1005080011D0032A67EEA67A0DD0042A67EEA67AE0
:1005180009D0052A67EEA67A05D067EEA67A062ADC
:1005280018BF67EEA67A002C3BD087EE277A5DF8D5
:10053800044B20EE070A70479178A1F13003092B8C
:1005480002F1020230D80124AFE75378A3F1300159
:10055800C8B2092802F1010293D8F2EE046AF0EE5B
:10056800665A07EE901AF8EEE77A12F8013F87EE1E
:10057800A66AA3F13001C8B2092866EEA56A37EE6B
:10058800067AEED97DE75378BFEE000A02465EE7A9
:100598009178A1F13003092B02F1020284D9F7EE18
:1005A800007A27EE277AC2E7F7EE007ABDE7F7EE82
:1005B800007A9BE70000000020BCBE4C0028F0B485
:1005C80003DA2D230B7040420131092804464FF00D
:1005D800010307DD03EB83035B00B0FBF3F2092A99
:1005E800F8D883B10F48A0FB0326B4FBF3F2092A1D
:1005F80002F1570C02F1300709DD03FB1244F3083E
:1006080001F801CBEFD100230B70F0BC704703FB5E
:100618001244F30801F8017BE5D100230B70F0BC0C
:10062800704700BFCDCCCCCC884270B44FF00104E9
:1006380042D301FB04F4B0FBF4F58D42F9D2ECB1DE
:1006480042BB092D04FB150005F1570605F13002E0
:100658000EDDB4FBF1F403F8016B7CB1B0FBF4F5EB
:10066800092D04FB150005F1570605F13002F0DCF1
:10067800B4FBF1F403F8012B002CEFD100221A701F
:1006880070BC704703F8016BB4FBF1F4002CF5D093
:10069800B0FBF4F5092D04FB150005F1370605F14B
:1006A8003002EFDCB4FBF1F403F8012B002CEFD19E
:1006B80000221A7070BC70470546002AEAD1C0E7CC
:1006C80003685A1C0260197070472DE9F047089CAE
:1006D8002578002B804689460CBF4FF0200A4FF042
:1006E800300A661C25B3002A26DD334601E002469F
:1006F80098B113F8011B501E0029F8D1971E60B15C
:100708003D46013D51464046C8476B1C002BF8DC6E
:10071800257827EAE770013045B1041B2946404691
:10072800C847301916F8015B002DF7D1BDE8F087EE
:10073800002A03DC2846F9E70020EEE7571EDFE72A
:10074800034600F11001FF221A705A7002339942D1
:10075800FAD1027042708270C270027142717047A1
:1007680030B42322242325252D242E210270437002
:100778002F22FF23857044718171C2714373837383
:10078800C37003710372437230BC704730B40023E6
:100798000225012429213D2203700323457084701A
:1007A800C1708271C37130BC7047094B09498B42D3
:1007B80003D309E014338B4206D21A88C2F30B0222
:1007C8009042F7D11846704700231846704700BF7B
:1007D800E0D0030890D5030870B50546B0F80900C5
:1007E800FFF7E3FF064B1E7804462846FFF732FD65
:1007F80016B1A368184470BD63681844FBE700BFCE
:10080800300F002038B505460C46FFF7E5FF2A797A
:1008180002F0070302F06002602A28D1022B0ED0F2
:10082800042B18D03BB96A7901239340DBB20278D4
:1008380014B11343037038BD22EA0303FAE76A7957
:10084800012393409BB2028814B113430380F2E75B
:1008580022EA0303FAE76A79012303FA02F203683A
:1008680014B113430360E6E723EA0203FAE7042B13
:10087800E1D8DFE803F00303050507000470DAE7B1
:100888000480D8E70460D6E7002306214FF47A7283
:100898000170C0E90123037370474378007840EA88
:1008A800032010FB01F04FF4807190FBF1F000F38E
:1008B8000F0000B270472DE9F04FDFF8DCC1754C2E
:1008C800DCF804502288B4F90AA0C2EB25135200C0
:1008D800C2EBE502B4F902505B436A43B4F9045031
:1008E8001B135D43AD1305EBE225B5F5FA324FEA6C
:1008F800E57B85B04BF1FF33CDE90023DDE900321C
:100908005343009AA561A2FB0289CDE90201B4F91B
:1009180008200199009809EB43095143D31700FBBC
:100928000311A2FB00230B444FEAEA7B0AFB09F1FF
:100938001F0308FB0B13AAFB080119444FEA102AEE
:100948004AEA016A16034FEA212B47EA12571AEBC3
:100958000602E6884BEB070312F1000A43F5004B49
:10096800AAFB060106FB0B114A10CB1752EA03013A
:1009780000F08E80B4F91060009806FB09F1F717B3
:1009880008FB0711A6FB08673944B4F90E808B46AB
:1009980001994FEAE87908FB01F100FB0911A8FB6E
:1009A80000898944DCF808104FEA4947C1F5801CE2
:1009B80047EAD837B2464FEA4846B4F90C801AEBF2
:1009C800060A66464BEB070BF7174FEAC80601966F
:1009D80000260096F907DDE900674FEACC7016EBB0
:1009E8000A0647EB0B0741EA5C01801B61EB070134
:1009F80040F6354C8946A0FB0C010CFB091133F07D
:100A08002FFFB4F91620B4F914A04E13470B47EA88
:100A1800C14702FB06FCD31707FB03CCA2FB072345
:100A28006344564307FB0366A2FB07233344560E71
:100A380046EAC31632184FEA636747EB010380465C
:100A48000AFB01F14FEAEA7B08FB0B17AAFB080136
:100A58003944C60C46EA413612EB06084FEAE1472C
:100A6800B4F9122043EB07094FEA182141EA09615A
:100A780013010B44029A0AB11B0A1360039B23B1AA
:100A880005EB850580352D121D6005B0BDE8F08F9A
:100A98000023EFE7C01D0020300F0020704770478B
:100AA80010B5064C237B0BB9002010BD14F0B8FD1F
:100AB8002369C01AD0F5FA50F7D5F5E7300F0020B2
:100AC8004FF40063038370474FF400630383704758
:100AD800012380F85030704707B5F7216A462EF099
:100AE800FBFF9DF801309DF800100C4A1B0143EAFA
:100AF80001339DF8021043EA111393609DF8043006
:100B08009DF803101B0143EA01339DF8051043EAE1
:100B18001113536003B05DF804FB00BF300F0020D1
:100B280070B4D0E90041057B02690223AB406360E1
:100B38000B684FF6FE7003400B60EFF311835021F2
:100B480081F31288D66B3168C9071CD4706870B9F4
:100B5800D2E909418C4213D095690D44F56017D844
:100B68001469611A71609062002182F85810326825
:100B780042F00102DBB2326083F3118870BC704727
:100B8800012182F85810DBB283F3118870BC7047DA
:100B9800611A71609462E7E770B40468037B2268A5
:100BA800022101FA03F31A4216D0026911481249C8
:100BB800642505FB02020D785068016875B915694E
:100BC800528928684FF6FE7630402860C868D243BC
:100BD80092B20240CA60636070BC704700690268E4
:100BE8004FF6FE752A400260CA684FF6FF60024061
:100BF800CA60F0E7D45D0020D05D002010B5016820
:100C0800047B0A680223A3401A420AD0054A4068B6
:100C180000241470026822F001021204120C02600F
:100C28004B6010BD0850002030B50446406DA160EF
:100C3800036823F0010303606379257987B013F013
:100C4800040F4FEA03324FEA032303F4806302F4EC
:100C58000052CDE90223009114BF4FF480510021C6
:100C6800EB0748BF042301914FF00001CDE90411BF
:100C780054BF08230493694648BF0C23AD0748BFF7
:100C880004931AF0E9FE2079636D617900F002029D
:100C9800002A15BF4FF440324FF480324FF400342D
:100CA800002410F0010F586808BF2246CC074CBF3B
:100CB800024320EA02025A609A6809074CBF42F0D0
:100CC800080222F008029A601A6842F001021A60CB
:100CD80007B030BD30B40223142101221525222487
:100CE8000372417000234FF6FF714571C4700270A2
:100CF8000271827043818381C3810182817430BC17
:100D0800704710B427212624012200230470417063
:100D18008270C3705DF8044B704710B50368017B9F
:100D28001A6802238B40134204460FD00F4A5369B6
:100D38000133202B53610AD1182200210C4834F0CA
:100D4800B2F9217B226802238B40536010BD222B0D
:100D5800F7D100235361074A13704268136823F0E0
:100D680001031B041B0C1360EBE700BF300F0020CE
:100D7800101000200110002008B5202134F0AAF935
:100D88000346184623B10278202A03F10103F8D05C
:100D980008BD38B52C22002134F085F9034640F20D
:100DA800DC51642040F21A4240F20224187459823D
:100DB800132019219A8240F2753240F26C751C8317
:100DC80098760E2402201977DA830A210122DD821F
:100DD80083F82A0040F6430583F82B1083F8224055
:100DE8009A7383F8252083F829201D841946024820
:100DF800BDE838400FF0F0B9F497030838B5074C50
:100E0800074DAC4203D3074B00221A7038BD6288E5
:100E1800D4E9010134F023F91434F2E7E0D00308EF
:100E280090D50308300F002038B5074C074DAC4269
:100E380003D3074B01221A7038BD6288D4E9011028
:100E480034F00DF91434F2E7E0D0030890D5030824
:100E5800300F002010B500210446012013F08AFD50
:100E6800207010BDF8B5304E304D32782B789A424C
:100E78004FD12F4B93F800C0BCF1000F48D02D4A3A
:100E88002D4B1078002140F20D3E11E05C681F895F
:100E98006760276847F001072760A2F848E0D46830
:100EA800013144F480748C45D46003F59A730FDDE6
:100EB8001A680028EAD15062B3F83041D768013186
:100EC8003C438C45D46003F59A7323F8040CEFDC9B
:100ED80031782B7899421BD003EB83029200174F8D
:100EE800B858BE18A0B9327A92B9727A82B9013369
:100EF80003F00303D8B28142287009D003EB8303BF
:100F08009C003B191A7214F08BFB736803443B5125
:100F1800F8BD29F0E9FF0028FAD0054B93F800C086
:100F2800BCF1000FABD1D3E79C3D00209D3D0020D4
:100F3800F4600020D05D0020F8600020A03D002073
:100F4800002A12DD70B504460D468E182368204627
:100F58009B6898470028F9D0236815F8011B1B687F
:100F680020469847B542F1D170BD70470368DB6AE7
:100F780003B11847704703689B6A03B11847704765
:100F880003682DE9F0415D6A1DB12B46BDE8F041CB
:100F98001847002A174611DD04460E460F4400E0A4
:100FA80023689B68204698470028F9D0236816F8DC
:100FB800011B1B6820469847BE42F1D1BDE8F0816D
:100FC80003685B6918470368DB68184703689B6810
:100FD800184703685B68184703681B681847014B84
:100FE8001868F9E7B4260020054B53F8203033B1D0
:100FF8001A689B88918A0B4218BF1B04936170473B
:101008000453002003682DE9F04F03F13845A94E39
:10101800AD0A0124755D05F01F066D09022D04FA5D
:1010280006F400F08D81032D00F08581012D00F07C
:101038003B818088B0FA80F4C4F11F04A4B2E508AB
:1010480003EB850504F007042E6AA4000F27A740C8
:1010580026EA07062E622E6A01F0030702FA04F454
:101068007A1E3443012AC1F3810EC1F300182C62A1
:10107800C1F3411140F22281C60700F108818507BA
:1010880000F1F680440700F1E480020700F1D28005
:10109800C60600F1C080850600F1AE80440600F166
:1010A8009C80020600F18A80C60578D4850567D43D
:1010B800440556D4020545D4C60434D4850423D443
:1010C800440412D4020401D4BDE8F08F1A6822F057
:1010D80040421A601A6842EA87771F60DA6822F08D
:1010E800404242EA8171D960EEE71A6822F0405224
:1010F8001A601A6842EA07721A60DA6822F04052E7
:1011080042EA0172DA60DDE71A6822F040621A608A
:101118001A6842EA87621A60DA6822F0406242EA94
:101128008162DA60CCE71A6822F040721A601A68A5
:1011380042EA07621A60DA6822F0407242EA016203
:10114800DA60BBE71A6822F440021A601A6842EAB9
:1011580087521A60DA6822F4400242EA8152DA6061
:10116800AAE71A6822F440121A601A6842EA07527B
:101178001A60DA6822F4401242EA0152DA6099E70A
:101188001A6822F440221A601A6842EA87421A60F2
:10119800DA6822F4402242EA8142DA6088E71A6873
:1011A80022F440321A601A6842EA07421A60DA6882
:1011B80022F4403242EA0142DA6077E71A6822F400
:1011C80040421A601A6842EA87321A60DA6822F4E2
:1011D800404242EA8132DA6066E71A6822F44052F5
:1011E8001A601A6842EA07321A60DA6822F4405232
:1011F80042EA0132DA6054E71A6822F440621A605F
:101208001A6842EA87221A60DA6822F4406242EADF
:101218008122DA6042E71A6822F440721A601A687A
:1012280042EA07221A60DA6822F4407242EA01228E
:10123800DA6030E71A6822F0C0021A601A6842EAD7
:1012480087121A60DA6822F0C00242EA8112DA6074
:101258001EE71A6822F030021A601A6842EA07127A
:101268001A60DA6822F0300242EA0112DA600CE70A
:101278001A6822F00C021A601A6842EA87021A6099
:10128800DA6822F00C0242EA8102DA60FAE61A68A9
:1012980022F003021A601A683A431A60DA6822F0E8
:1012A80003020A43DA60EAE6034D6E6934436C616F
:1012B800BFE600BFA88903080010024000224FF0D3
:1012C800010C4FF003090CFA02F636EA00042ED19D
:1012D8005400D3F808A009FA04F5ED4305EA0A0A10
:1012E800C3F808A0D3F808B00EFA04FA4AEA0B0AC1
:1012F800C3F808A0B3F804A02AEA06069E80B3F84B
:1013080004A008FA02F646EA0A06B6B29E801E68EB
:101318002E401E60D3F800A007FA04F646EA0A0633
:101328001E60DE6801FA04F435402C43DC600132AB
:10133800102AC8D1C8E6054DEE693443EC6178E659
:10134800024DAE693443AC6173E600BF0010024041
:1013580010B50409013C052C17D80E4B33F814209E
:1013680000F00F0042FA00F313F001030FD001233D
:1013780003FA00F00138104033F0C2FA064A074B6E
:10138800125D104403EBC00010BD002010BD1846CC
:1013980010BD00BF94890308A0890308A84E002047
:1013A8002DE9F04F4A484B4B4B4C4FF090414FF0D2
:1013B800010A4FF002094FF004084FF0080E4FF0F1
:1013C800100C20274026802530F8022B12F0010F40
:1013D80003D01960A3F804A0083312F0020F03D059
:1013E8001960A3F80490083312F0040F03D01960B1
:1013F800A3F80480083312F0080F03D01960A3F88B
:1014080004E0083312F0100F03D01960A3F804C0E9
:10141800083312F0200F02D019609F80083312F0B1
:10142800400F02D019609E80083312F0800F02D05E
:1014380019609D80083312F4807F05D04FF4807BBB
:101448001960A3F804B0083312F4007F05D04FF4F4
:10145800007B1960A3F804B0083312F4806F05D03C
:101468004FF4806B1960A3F804B0083312F4006FCE
:1014780005D04FF4006B1960A3F804B0083312F4D8
:10148800805F05D04FF4805B1960A3F804B008337F
:1014980012F4005F05D04FF4005B1960A3F804B0A4
:1014A800083312F4804F05D04FF4804B1960A3F82D
:1014B80004B00833D20B04D04FF4004219609A806C
:1014C800083301F58061A1427FF47EAFBDE8F08F5B
:1014D80094890308A84E00200018004800B97047F6
:1014E80003682DE9F04F03F138449C4EA40A012506
:1014F800345D04F01F066409022C05FA06F500F0B5
:101508007481032C00F06C81012C00F0228180880A
:10151800B0FA80F4C4F11F04A4B2E50803EB850512
:1015280004F007042E6AA4000F27A74026EA07063E
:101538002E622E6A01F00307A2407C1E3243012C62
:10154800C1F3810EC1F300182A62C1F3411140F2C0
:101558000981C6070BD51A6822F003021A601A68B7
:101568003A431A60DA6822F003020A43DA60850710
:101578000DD51A6822F00C021A601A6842EA87022E
:101588001A60DA6822F00C0242EA8102DA60440743
:101598000DD51A6822F030021A601A6842EA07125A
:1015A8001A60DA6822F0300242EA0112DA600207B1
:1015B8000DD51A6822F0C0021A601A6842EA87122A
:1015C8001A60DA6822F0C00242EA8112DA60C606BE
:1015D8000DD51A6822F440721A601A6842EA072286
:1015E8001A60DA6822F4407242EA0122DA6085065B
:1015F8000DD51A6822F440621A601A6842EA8722F6
:101608001A60DA6822F4406242EA8122DA6044060B
:101618000DD51A6822F440521A601A6842EA073255
:101628001A60DA6822F4405242EA0132DA600206AD
:101638000DD51A6822F440421A601A6842EA8732C5
:101648001A60DA6822F4404242EA8132DA60C6055A
:101658000DD51A6822F440321A601A6842EA074225
:101668001A60DA6822F4403242EA0142DA608505FB
:101678000DD51A6822F440221A601A6842EA874295
:101688001A60DA6822F4402242EA8142DA604405AC
:101698000DD51A6822F440121A601A6842EA0752F5
:1016A8001A60DA6822F4401242EA0152DA6002054E
:1016B8000DD51A6822F440021A601A6842EA875265
:1016C8001A60DA6822F4400242EA8152DA60C604FB
:1016D8000DD51A6822F040721A601A6842EA076249
:1016E8001A60DA6822F0407242EA0162DA60850420
:1016F8000DD51A6822F040621A601A6842EA8762B9
:101708001A60DA6822F0406242EA8162DA604404D0
:101718000DD51A6822F040521A601A6842EA077218
:101728001A60DA6822F0405242EA0172DA60020472
:101738000DD51A6822F040421A601A6842EA877783
:101748001F60DA6822F0404242EA8171D960BDE840
:10175800F08F034C666935436561D8E6A8890308AC
:101768000010024000224FF0010C4FF003090CFA60
:1017780002F636EA00042ED15400D3F808A009FA7C
:1017880004F5ED4305EA0A0AC3F808A0D3F808B03F
:101798000EFA04FA4AEA0B0AC3F808A0B3F804A040
:1017A8002AEA06069E80B3F804A008FA02F646EA7A
:1017B8000A06B6B29E801E682E401E60D3F800A0AE
:1017C80007FA04F646EA0A061E60DE6801FA04F41F
:1017D80035402C43DC600132102AC8D1BDE8F08FB7
:1017E800044CE6693543E56191E6024CA669354348
:1017F800A5618CE60010024000B97047036803F148
:1018080038422DE9F04F920AB24DAA5C02F01F054A
:1018180052090124022A04FA05F400F05F81032A20
:1018280000F05381012A00F00D8101F003077A1EB0
:10183800012AC1F3810EC1F300188488C1F3411154
:1018480040F20581E6070BD51A6822F003021A60F8
:101858001A683A431A60DA6822F003020A43DA6027
:10186800A5070DD51A6822F00C021A601A6842EA18
:1018780087021A60DA6822F00C0242EA8102DA6012
:1018880060070DD51A6822F030021A601A6842EA19
:1018980007121A60DA6822F0300242EA0112DA60AE
:1018A80022070DD51A6822F0C0021A601A6842EAA7
:1018B80087121A60DA6822F0C00242EA8112DA60FE
:1018C800E6060DD51A6822F440721A601A6842EAD0
:1018D80007221A60DA6822F4407242EA0122DA60CA
:1018E800A5060DD51A6822F440621A601A6842EA01
:1018F80087221A60DA6822F4406242EA8122DA60BA
:1019080060060DD51A6822F440521A601A6842EA35
:1019180007321A60DA6822F4405242EA0132DA6089
:1019280022060DD51A6822F440421A601A6842EA63
:1019380087321A60DA6822F4404242EA8132DA6079
:10194800E6050DD51A6822F440321A601A6842EA90
:1019580007421A60DA6822F4403242EA0142DA6049
:10196800A5050DD51A6822F440221A601A6842EAC1
:1019780087421A60DA6822F4402242EA8142DA6039
:1019880060050DD51A6822F440121A601A6842EAF6
:1019980007521A60DA6822F4401242EA0152DA6009
:1019A80022050DD51A6822F440021A601A6842EA24
:1019B80087521A60DA6822F4400242EA8152DA60F9
:1019C800E6040DD51A6822F040721A601A6842EAD5
:1019D80007621A60DA6822F0407242EA0162DA604D
:1019E800A5040DD51A6822F040621A601A6842EA06
:1019F80087621A60DA6822F0406242EA8162DA603D
:101A080060040DD51A6822F040521A601A6842EA3A
:101A180007721A60DA6822F0405242EA0172DA600C
:101A280022040DD51A6822F040421A601A6842EA68
:101A380087771F60DA6822F0404242EA8171D960F4
:101A4800BDE8F08F244A55692C435461EDE6002225
:101A58004FF0010C4FF003090CFA02F636EA0400C5
:101A68002ED15000D3F808A009FA00F5ED430AEA90
:101A7800050AC3F808A0D3F808B00EFA00FA4AEA33
:101A88000B0AC3F808A0B3F804A02AEA06069E8049
:101A9800B3F804A008FA02F646EA0A06B6B29E802F
:101AA8001E682E401E60D3F800A007FA00F646EA2A
:101AB8000A061E60DE6801FA00F035402843D86047
:101AC8000132102AC8D1BDE8F08F034AD5692C43EA
:101AD800D461AAE6A889030800100240024A956961
:101AE8002C439461A1E600BF0010024010B10368C6
:101AF80082881A85704710B1036882889A61704796
:101B080018B1838811B10268936170471B04FAE722
:101B180010B40A4B0A4A1C7801238340234052F828
:101B2800200029B9B3FA83F149095DF8044BE7E7C6
:101B3800191C18BF01215DF8044BE1E70053002090
:101B48000453002030B102688388128A1A4214BFF5
:101B58000120002070472DE9F0410C4E356873696B
:101B68001D4010D0DFF828800127B5FA85F4C4F1AC
:101B78001F0408EB840307FA04F49869036898477C
:101B8800A5437461F1D1BDE8F08100BF00040140B4
:101B9800300F00202DE9F0410B4E356873691D4068
:101BA80010D0DFF828800127B5FA85F4C4F11F04A6
:101BB80008EB840307FA04F4986903689847A54377
:101BC8007461F1D1BDE8F08100040140300F0020BC
:101BD8002DE9F0410B4E356873691D4010D0DFF8D0
:101BE80028800127B5FA85F4C4F11F0408EB8403A3
:101BF80007FA04F4986903689847A5437461F1D11A
:101C0800BDE8F08100040140300F00202DE9F041CB
:101C18000B4E356873691D4010D0DFF82880012706
:101C2800B5FA85F4C4F11F0408EB840307FA04F439
:101C3800986903689847A5437461F1D1BDE8F081BC
:101C480000040140300F00202DE9F0410B4E3568AB
:101C580073691D4010D0DFF828800127B5FA85F494
:101C6800C4F11F0408EB840307FA04F498690368B5
:101C78009847A5437461F1D1BDE8F08100040140A3
:101C8800300F00202DE9F0410B4E356873691D4077
:101C980010D0DFF828800127B5FA85F4C4F11F04B5
:101CA80008EB840307FA04F4986903689847A54386
:101CB8007461F1D1BDE8F08100040140300F0020CB
:101CC8002DE9F0410B4E356873691D4010D0DFF8DF
:101CD80028800127B5FA85F4C4F11F0408EB8403B2
:101CE80007FA04F4986903689847A5437461F1D129
:101CF800BDE8F08100040140300F0020094A10B50A
:101D08009369094C43F00103936104F118004022E0
:101D1800002133F0C8F94FF0FF33A365C4F85B30F6
:101D280010BD00BF00100240300F002003681B6A7E
:101D3800184770B44E1C0568C2728672AC69A44616
:101D480070BC60472DE9F041044618460D4616461A
:101D58001F4632F0E9FA2844A0722068E672294644
:101D680045693B4632462046AC46BDE8F0416047EF
:101D7800036810B504461B689847236820469B688B
:101D88009847E37B0133E37310BD10B5036804463D
:101D98009B689847FF230122A373627310BD70B537
:101DA800054600780E46FFF7D3FA044618B13823E3
:101DB80001368371C67120466978FFF71DFDAB783F
:101DC800204613B1BDE8704095E6BDE870408DE649
:101DD8000B4B984211D0A3F57843984202D04FF0AC
:101DE800FF3070470122074B03EB02135A89013277
:101DF80092B25A81588980B270470022F3E700BF37
:101E08000030014010290020F8B584894FF6FF768C
:101E18004FF47A7413F1FF3325D311B30F780131DE
:101E280001E0B44217D00589013CAD07A4B2F8D54A
:101E380007734FF47A7402E0BCB2B4420BD0058940
:101E4800ED0704F1FF37F7D5057BEDB2002AE1D0A5
:101E580015700132DEE7FFF7BBFF003018BF012025
:101E6800F8BDFF27DFE70120F8BD08B5838940F2F8
:101E7800E93300E09BB10289013B12F0020F9BB2EB
:101E8800F8D0017340F2E93300E043B10289013B25
:101E980012F0010F9BB2F8D0007BC0B208BDFFF76B
:101EA80097FFC0B208BDF8B50546806816461F46BC
:101EB80010B1036882881A85686840F2E93483891A
:101EC80001E0002C44D00389013C13F0020FA4B2B6
:101ED800F7D0017340F2E93101E0002938D00389D5
:101EE800013913F0010F89B2F7D0037B6868838941
:101EF8004FF0000C4FF47A714FF6FF724FF0FF0E5F
:101F0800674502D11DE0914219D0038901399C0728
:101F180089B2F8D580F80CE04FF47A7102E0A1B2EA
:101F280091420CD00389DB0701F1FF34F7D5037B1D
:101F3800DBB20EB1337001360CF1010CE0E7FFF7AC
:101F480047FFAB6813B11A689B8893610120F8BDFD
:101F5800FFF73EFFCAE738B504460D46FEF7A0FD79
:101F6800246808B114F0A2F9054B00221A73C9219C
:101F78005B7B2A462046FFF796FF012038BD00BF4D
:101F8800300F002038B583680446154613B11A6827
:101F98009B881385606840F2E933828901E0002B51
:101FA80030D00289013B12F0020F9BB2F7D00173C7
:101FB80040F2E93300E02BB30289013B12F0010F34
:101FC8009BB2F8D0037B606840F2E933828900E075
:101FD800DBB10189013B11F0020F9BB2F8D0057308
:101FE80040F2E93300E083B10289013B12F0010FAE
:101FF8009BB2F8D0037BA36813B11A689B889361DE
:10200800012038BDFFF7E4FEDDE7FFF7E1FEF2E768
:1020180010B504464068A268038823F040031B04F7
:102028001B0C0380038823F038031B041B0C03805C
:10203800038843F04003038012B1136892881A851D
:10204800838940F2E93301E0002B44D00289013B47
:1020580012F0020F9BB2F7D0F523037340F2E93375
:1020680001E0002B37D00289013B12F0010F9BB22F
:10207800F7D0037B6068838940F2E93300E00BB353
:102088000289013B12F0020F9BB2F8D0FF230373C1
:1020980040F2E93300E0ABB10289013B12F0010FD5
:1020A8009BB2F8D0017BC9B2A36813B11A689B88A8
:1020B8009361712918D008D9AC2913D0AF290DD153
:1020C800092010BDFFF784FEEEE712290ED0702913
:1020D80006D1052010BDFFF77BFECBE7732903D09F
:1020E800002010BD072010BD062010BD082010BD1F
:1020F800F0B5836983B0064613B11A689B881385C7
:102108007069DFF8A0C08389C3244FF47A73062767
:102118006D464FF6FF710CF1010C03E0013B9BB2D9
:102128008B421CD002899207F8D504734FF47A7356
:1021380002E0A3B28B4212D00289D20703F1FF3426
:10214800F7D5027BD2B20DB12A7001354FB1013FEC
:10215800FF24BCF1000FE5D09CF80040DBE7FFF757
:1021680037FEB36913B11A689B8893619DF805001F
:102178009DF801509DF802109DF803409DF8042039
:102188009DF8063041EA052143EA002342EA042289
:102198000120A6F85010A6F85220A6F8543003B033
:1021A800F0BD00BF60510308F8B50378012B49D092
:1021B800022B4DD1836801F07F0113B11C689B8805
:1021C800238504464068154640F2E933828902E0D7
:1021D800002B00F0A0800289013B12F0020F9BB295
:1021E800F6D0017340F2E93302E0002B00F093804F
:1021F8000289013B12F0010F9BB2F6D0037B6068A5
:1022080040F2E933828902E0002B00F081800189E5
:10221800013B11F0020F9BB2F6D0057340F2E9338F
:1022280001E0002B74D00289013B12F0010F9BB230
:10223800F7D0037BA368002B68D01A689B8893614A
:102248000120F8BD90F904305C1C01D0022B01DD9F
:102258000020F8BD434C03EB830304EB83035B6866
:10226800002B6DD04579404E6D004FF42040EDB203
:1022780030669C69270400F1FF303DD45C683B4F11
:1022880045F080703C4040F4903020434FF42044A7
:102298005860346601E0671C54D0986910F0020059
:1022A80004F1FF34F7D04FF42040996230660146BC
:1022B80001E04F1C19D0986910F0800001F1FF313E
:1022C800F7D05968294845F00075014045F4803534
:1022D8000D434FF420415D603166986910F00200AB
:1022E80001F1FF311AD14C1CF7D1214A316613880C
:1022F80001339BB21380F8BD441CBAD11C4A306626
:10230800138801339BB213800020F8BD0120F8BD6B
:10231800FFF75EFD8EE7FFF75BFD70E74FF42041A6
:102328009A6231660A4602E012F1FF3211D39969C6
:1023380011F02001F8D020213266D9610120F8BDC2
:102348001846F8BD0A4A3466138801339BB21380D5
:10235800F8BD074C3266238801339BB208462380B8
:10236800F8BD00BF20450020300F0020009800FC79
:10237800602400203122F42116E72DE9F04F8BB0BC
:1023880090F861300390002B40F01F86039B93F870
:102398005830072B00F00F861823CDE90433039B30
:1023A800BD4CBE4EDFF80083BD4F10331846802267
:1023B8006B210293FFF7F8FE6423DFF8F0E2B948D7
:1023C80001934FF01009DEF80430C3F30803002B23
:1023D80040F0C284EFF31183002B40F0BD842568E0
:1023E800826823689D42FAD13B689A42F7D8D6F8AA
:1023F80000C04FF47A7101FB0CF39B1AB3FBFCF39A
:1024080001FB05354FF47A7C4FF0010ADEF8043001
:10241800C3F30803002B40F05E84EFF31183002B15
:1024280040F059842368816822689342FAD13A6857
:102438009142F7D832680CFB02FBABEB0101B1FB10
:10244800F2F10CFB03135B1BB3F57A7FDED3019B20
:10245800013B0193B7D1072268210298DFF848822F
:102468008F4FFFF7A1FE6423DFF840E28D48019308
:102478004FF01009DEF80430C3F30803002B40F0D6
:102488004984EFF31183002B40F044842568826867
:1024980023689D42FAD13B689A42F7D8D6F800C023
:1024A8004FF47A7101FB0CF39B1AB3FBFCF301FBAD
:1024B80005354FF47A7C4FF0010ADEF80430C3F397
:1024C8000803002B40F0E983EFF31183002B40F061
:1024D800E4832368816822689342FAD13A6891427A
:1024E800F7D832680CFB02FBABEB0101B1FBF2F150
:1024F8000CFB03135B1BB3F57A7FDED3019B013B17
:102508000193B7D11A466B210298DFF89C81644F7A
:10251800FFF74AFE6423DFF894E1624801934FF025
:102528001009DEF80430C3F30803002B40F0DC8404
:10253800EFF31183002B40F0D78425688268236865
:102548009D42FAD13B689A42F7D8D6F800C04FF4BA
:102558007A7101FB0CF39B1AB3FBFCF301FB053505
:102568004FF47A7C4FF0010ADEF80430C3F3080315
:10257800002B40F07483EFF31183002B40F06F833E
:102588002368816822689342FAD13A689142F7D861
:1025980032680CFB02FBABEB0101B1FBF2F10CFB67
:1025A80003135B1BB3F57A7FDED3019B013B0193D9
:1025B800B7D101226B210298DFF8EC80384FFFF782
:1025C800F3FD0F23DFF8E4E0364801934FF01009DC
:1025D800DEF80430C3F30803002B40F06384EFF304
:1025E8001183002B40F05E842568826823689D4231
:1025F800FAD13B689A42F7D8D6F800C04FF47A71FE
:1026080001FB0CF39B1AB3FBFCF301FB05354FF4FC
:102618007A7C4FF0010ADEF80430C3F30803002B7C
:1026280040F0FF82EFF31183002B40F0FA82236819
:10263800816822689342FAD13A689142F7D83268A1
:102648000CFB02FBABEB0101B1FBF2F10CFB03133A
:102658005B1BB3F57A7FDED3019B013B0193B7D1B6
:10266800049A0298DFF840800D4F1B21FFF79CFD6C
:102678000F23DFF838E00B4801934FF01009DEF81C
:102688000430C3F30803002B40F07184EFF3118387
:10269800002B40F06C840BE0A44E0020385300203F
:1026A8003C53002010E000E03453002000ED00E02F
:1026B8002568826823689D42FAD13B689A42F7D818
:1026C800D6F800C04FF47A7101FB0CF39B1AB3FBE8
:1026D800FCF301FB05354FF47A7C4FF0010ADEF874
:1026E8000430C3F30803002B40F07D82EFF311831D
:1026F800002B40F078822368816822689342FAD1DF
:102708003A689142F7D832680CFB02FBABEB010147
:10271800B1FBF2F10CFB03135B1BB3F57A7FDED33D
:10272800019B013B0193AAD1059A0298DFF80C831B
:10273800C04F1C21FFF738FD0F23DFF804E3BE4824
:1027480001934FF01009DEF80430C3F30803002B9F
:1027580040F0EC83EFF31183002B40F0E78325680A
:10276800826823689D42FAD13B689A42F7D8D6F826
:1027780000C04FF47A7101FB0CF39B1AB3FBFCF316
:1027880001FB05354FF47A7C4FF0010ADEF804307E
:10279800C3F30803002B40F00882EFF31183002BEA
:1027A80040F003822368816822689342FAD13A682C
:1027B8009142F7D832680CFB02FBABEB0101B1FB8D
:1027C800F2F10CFB03135B1BB3F57A7FDED3019B9D
:1027D800013B0193B7D1039A92F85B30032B00F2C7
:1027E800E88392F85E20A2F10102B2FA82F252095D
:1027F8001A210298DFF844828E4FFFF7D5FC0F2389
:10280800DFF83CE28C4801934FF01009DEF8043001
:10281800C3F30803002B40F0E282EFF31183002B8F
:1028280040F0DD822568826823689D42FAD13B68C2
:102838009A42F7D8D6F800C04FF47A7101FB0CF32E
:102848009B1AB3FBFCF301FB05354FF47A7C4FF080
:10285800010ADEF80430C3F30803002B40F0878137
:10286800EFF31183002B40F082812368816822688E
:102878009342FAD13A689142F7D832680CFB02FBCE
:10288800ABEB0101B1FBF2F10CFB03135B1BB3F5DE
:102898007A7FDED3019B013B0193B7D1039B02985A
:1028A80093F86020DFF89481624F1921FFF77CFCD0
:1028B8006423DFF88CE1604801934FF01009DEF8DB
:1028C8000430C3F30803002B40F06882EFF3118350
:1028D800002B40F063822568826823689D42FAD104
:1028E8003B689A42F7D8D6F800C04FF47A7101FBDA
:1028F8000CF39B1AB3FBFCF301FB05354FF47A7C10
:102908004FF0010ADEF80430C3F30803002B40F04F
:102918001081EFF31183002B40F00B81236881684D
:1029280022689342FAD13A689142F7D832680CFB90
:1029380002FBABEB0101B1FBF2F10CFB03135B1BD8
:10294800B3F57A7FDED3019B013B0193B7D1102207
:1029580037210298DFF8E480364FFFF725FC0F2374
:10296800DFF8DCE0344801934FF01009DEF804305A
:10297800C3F30803002B40F07482EFF31183002B9C
:1029880040F06F822568826823689D42FAD13B68CF
:102998009A42F7D8D6F800C04FF47A7101FB0CF3CD
:1029A8009B1AB3FBFCF301FB05354FF47A7C4FF01F
:1029B800010ADEF80430C3F30803002B40F09B80C3
:1029C800EFF31183002B40F096802368816822681A
:1029D8009342FAD13A689142F7D832680CFB02FB6D
:1029E800ABEB0101B1FBF2F10CFB03135B1BB3F57D
:1029F8007A7FDED3019B013B0193B7D10298DFF8C0
:102A08003C800C4F01223821FFF7CEFB0F23DFF863
:102A180030E0094801934FF01009DEF80430C3F3A1
:102A28000803002B40F0FC81EFF31183002B40F0EA
:102A3800F78107E03C53002010E000E03453002009
:102A480000ED00E02568826823689D42FAD13B6862
:102A58009A42F7D8D6F800C04FF47A7101FB0CF30C
:102A68009B1AB3FBFCF301FB05354FF47A7C4FF05E
:102A7800010ADEF80430C3F30803F3B9EFF3118356
:102A8800DBB92368816822689342FAD13A68914297
:102A9800F7D832680CFB02FBABEB0101B1FBF2F19A
:102AA8000CFB03135B1BB3F57A7FE2D3019B013B5D
:102AB8000193B2D10BB0BDE8F08FEFF3118189F328
:102AC8001288D0F808B00368DB0344BFC8F800A038
:102AD800D0F808B02368D8F80020C9B281F311886B
:102AE800316813440CFB01F2A2EB0B02B2FBF1F2CA
:102AF8000CFB0323D6E7EFF3118189F31288D0F892
:102B080008B00368DB0344BFC8F800A0D0F808B0D9
:102B18002368D8F80020C9B281F3118831681344BA
:102B28000CFB01F2A2EB0B02B2FBF1F20CFB03234C
:102B38005CE7EFF3118189F31288D0F808B00368D5
:102B4800DB0344BFC8F800A0D0F808B02368D8F861
:102B58000020C9B281F31188316813440CFB01F2DB
:102B6800A2EB0B02B2FBF1F20CFB0323E7E6EFF357
:102B7800118189F31288D0F808B00368DB0344BFD9
:102B8800C8F800A0D0F808B02368D8F80020C9B267
:102B980081F31188316813440CFB01F2A2EB0B029C
:102BA800B2FBF1F20CFB032370E6EFF3118189F31A
:102BB8001288D0F808B00368DB0344BFC8F800A047
:102BC800D0F808B02368D8F80020C9B281F311887A
:102BD800316813440CFB01F2A2EB0B02B2FBF1F2D9
:102BE8000CFB0323EFE5EFF3118189F31288D0F88A
:102BF80008B00368DB0344BFC8F800A0D0F808B0E9
:102C08002368D8F80020C9B281F3118831681344C9
:102C18000CFB01F2A2EB0B02B2FBF1F20CFB03235B
:102C28007AE5EFF3118189F31288D0F808B00368C8
:102C3800DB0344BFC8F800A0D0F808B02368D8F870
:102C48000020C9B281F31188316813440CFB01F2EA
:102C5800A2EB0B02B2FBF1F20CFB0323F8E4EFF357
:102C6800118189F31288D0F808B00368DB0344BFE8
:102C7800C8F800A0D0F808B02368D8F80020C9B276
:102C880081F31188316813440CFB01F2A2EB0B02AB
:102C9800B2FBF1F20CFB032383E4EFF3118189F318
:102CA8001288D0F808B00368DB0344BFC8F800A056
:102CB800D0F808B02368D8F80020C9B281F3118889
:102CC800316813440CFB01F2A2EB0B02B2FBF1F2E8
:102CD8000CFB03230EE4EFF3118189F31288D0F87B
:102CE80008B00368DB0344BFC8F800A0D0F808B0F8
:102CF8002368D8F80020C9B281F3118831681344D9
:102D08000CFB01F2A2EB0B02B2FBF1F20CFB03236A
:102D1800FFF799BBEFF3118389F31288D0F808C045
:102D28000268D20304D50122C8F80020D0F808C0F0
:102D38002568D8F800A0DBB283F3118831684FF416
:102D48007A72554402FB01F3A3EB0C03B3FBF1F3D6
:102D580002FB0535FFF7ADBBEFF3118389F312884A
:102D6800D0F808C00268D20304D50122C8F80020B0
:102D7800D0F808C02568D8F800A0DBB283F3118822
:102D880031684FF47A72554402FB01F3A3EB0C034C
:102D9800B3FBF1F302FB0535FFF734BBEFF3118307
:102DA80089F31288D0F808C00268D20304D501223A
:102DB800C8F80020D0F808C02568D8F800A0DBB211
:102DC80083F3118831684FF47A72554402FB01F39A
:102DD800A3EB0C03B3FBF1F302FB05358EE5EFF330
:102DE800118389F31288D0F808C00268D20304D589
:102DF8000122C8F80020D0F808C02568D8F800A03B
:102E0800DBB283F3118831684FF47A72554402FBC0
:102E180001F3A3EB0C03B3FBF1F302FB053514E557
:102E2800EFF3118389F31288D0F808C00268D2033F
:102E380004D50122C8F80020D0F808C02568D8F8C1
:102E480000A0DBB283F3118831684FF47A725544DD
:102E580002FB01F3A3EB0C03B3FBF1F302FB053513
:102E680003E6EFF3118389F31288D0F808C00268EB
:102E7800D20304D50122C8F80020D0F808C025687C
:102E8800D8F800A0DBB283F3118831684FF47A7266
:102E9800554402FB01F3A3EB0C03B3FBF1F302FB74
:102EA800053582E5EFF3118389F31288D0F808C05D
:102EB8000268D20304D50122C8F80020D0F808C05F
:102EC8002568D8F800A0DBB283F3118831684FF485
:102ED8007A72554402FB01F3A3EB0C03B3FBF1F345
:102EE80002FB0535FFF793BBEFF3118389F31288D3
:102EF800D0F808C00268D20304D50122C8F800201F
:102F0800D0F808C02568D8F800A0DBB283F3118890
:102F180031684FF47A72554402FB01F3A3EB0C03BA
:102F2800B3FBF1F302FB0535FFF71ABBEFF311838F
:102F380089F31288D0F808C00268D20304D50122A8
:102F4800C8F80020D0F808C02568D8F800A0DBB27F
:102F580083F3118831684FF47A72554402FB01F308
:102F6800A3EB0C03B3FBF1F302FB05350AE4EFF323
:102F7800118389F31288D0F808C00268D20304D5F7
:102F88000122C8F80020D0F808C02568D8F800A0A9
:102F9800DBB283F3118831684FF47A72554402FB2F
:102FA80001F3A3EB0C03B3FBF1F302FB0535FFF7C9
:102FB80092BB019A1CE4039B93F85D30002B44D12B
:102FC8001023CDE90433FFF7EAB91C09013C052CAD
:102FD80003F00F033FD8684A32F8140040FA03F2AE
:102FE800D60738D5012707FA03F3013B184031F01B
:102FF80087FC624BDFF898A113F8049081441AEB20
:10300800C90428D05AF83900A388028A1A407FF4E4
:10301800BDA9B3FA83F12025C1F11F01039EE27116
:10302800A571574AF2604D1C1AD1B3FA83F3C3F164
:103038001F03581C3FF4AAA9012202FA03F35149BD
:103048000A6813430B60FFF7A1B918231021CDE9D3
:103058000431FFF7A4B9039A494BD3600123EEE783
:1030680000F13842920ADFF82CC1DFF82CB11CF8C5
:1030780002C0454D0BEB01080CF01F0205EB810166
:103088004FEA5C1C06F10C0EBCF1020F07FA02F2C3
:1030980098F81480C1F818E04BD0BCF1030F66D043
:1030A800BC455FD008A90027CDE9083718F0A4FA75
:1030B800A3885AF83910DFF8E4C0B3FA83F3C3F1F0
:1030C8001F03D8B200F0FC0202F1804202F5803200
:1030D80000F0030080004FF00F0E0EFA00F9D2F84E
:1030E80008E02EEA090EC2F808E0D2F80890C1F309
:1030F8008721814041EA0901916003F01F0E23F006
:103108001F014FF0010909FA0EFE454441F80CE091
:10311800082208A808938DF824708DF826908DF859
:1031280025202CF067FC95F85830F02B06D8A3889A
:103138007BE7164FB9690A43BA61B3E70BEB080698
:10314800F02296F824308DF81C3007A803238DF858
:103158001E708DF81F9085F858208DF81D3018F0D6
:1031680077F8E4E7094F79690A437A619AE70749EA
:10317800CF693A43CA6195E794890308A08903088F
:10318800D90A000800040140300F00200010024056
:10319800A84E0020A88903085451030814040140CC
:1031A8004269138823F040031B041B0C2DE9F04FE0
:1031B800138013889BB223F0380343F03003138045
:1031C800138883B043F040031380019012F028FA6B
:1031D800044612F025FA8442FBD0019C2046FFF7F2
:1031E800CCF8A36913B11A689B881385019B5869A9
:1031F80040F2E933828902E0002B00F0AB800289BB
:10320800013B12F0020F9BB2F6D06A23037340F21F
:10321800E93302E0002B00F09D800289013B12F0A7
:10322800010F9BB2F6D0037B019B586940F2E9334A
:10323800828902E0002B00F090800289013B12F0A5
:10324800020F9BB2F6D01023037340F2E93302E079
:10325800002B00F082800289013B12F0010F9BB223
:10326800F6D0037B019B9B6913B11A689B88936115
:1032780064233B4CDFF8F490DFF8F480394DDFF835
:10328800F4A0394E009312F0CBF94FF47A774FF04F
:10329800100C4FF0010ED8F80430C3F30803002BCC
:1032A80039D1EFF31183002B35D12368A96822683F
:1032B8009342FAD132689142F7D8D9F8002007FB37
:1032C80002FBABEB0101B1FBF2F107FB03131B1A85
:1032D800B3F57A7FDFD3009B013B0093D3D1019BE9
:1032E8005A69138823F040031B041B0C13801388AE
:1032F80023F038031B041B0C1380138843F040038E
:10330800138012F08DF9044612F08AF98442FBD03A
:1033180003B0BDE8F08FEFF311818CF31288D5F874
:1033280008B02B68DB0344BFCAF800E0D5F808B042
:103338002368DAF80020C9B281F31188D9F800109F
:10334800134407FB01F2A2EB0B02B2FBF1F207FBFD
:103358000323BCE7FEF73CFD66E7FEF739FD81E78E
:10336800A44E002010E000E03C5300203853002019
:1033780000ED00E034530020427A4AB110B504460B
:1033880004F10A01D0E9003098470023637210BDA8
:103398007047A8B10D4B012210B402FA01F103F1F4
:1033A800750402E00333A3420BD013F8012C8242C8
:1033B800F8D11A780A42F5D001205DF8044B70471D
:1033C800704700205DF8044B704700BF8151030827
:1033D80030B40A4D002305F12C0401E0272B0AD054
:1033E80003EB43020133A15C8142F7D12A4430BC8C
:1033F80092F82E007047002030BC704754510308E3
:10340800024B01461868FCF7FDBE00BFA825002046
:1034180038B5064D441E14F8011F286811B9BDE8D7
:103428003840A9E7FCF7EEFEF5E700BFA825002025
:1034380010B504460B48FFF7EBFF0B4B1868FFF776
:103448009BFF0A4B186813F0F9FD1DF073FA084B3F
:10345800084A24B1084909480860DA6010BDDA60F2
:10346800FCE700BF048E0308A8250020AC25002037
:1034780000ED00E00400FA05FC9F0020EFBEADDE81
:1034880038B5094D2868FFF777FF084B00241C70F2
:10349800074B1C60074B1C701DF0DAFB2046FFF73A
:1034A800C7FF2C6038BD00BFA8250020B425002028
:1034B800B0250020B02900200120B9E70048A7E77F
:1034C800E793030838B5064D002455F83400013455
:1034D800FFF79EFFFFF7F2FF282CF6D138BD00BF9B
:1034E800AC7D030808B5FFF793FFBDE80840E5E7A2
:1034F800024A136823EA000010607047B85B002096
:103508002DE9F341056906460F467DBBD0F80080DA
:10351800C8F30A0323B30023D6F8008001932DF0E3
:103528000DFC042819D1224C236943F001032361BF
:10353800BBB2A8F800302DF001FC04282ED108F108
:1035480002030193019B3F0C1F802DF0F7FB2369B9
:10355800042823F00103236125D06FF0010505E05D
:103568002DF0ECFB042805D04FF0FF35284602B0BB
:10357800BDE8F0810E4C236943F002032361C4F8CF
:103588001480236943F0400323612DF0D7FB23699E
:10359800042823F002032361BDD0E5E7236923F063
:1035A80001032361D9E7336804333360DEE700BFE2
:1035B80000200240F8B504460D468E180027B54293
:1035C80001D12069F8BDE368591CE160234415F86E
:1035D800012B1A720429F2D1A1682046FFF790FF47
:1035E800C4E90370EBE730B402681146531C03606A
:1035F80011F8024B0160D31C517803609378151DB4
:1036080005601B0443EA0123D078234343EA0060A2
:1036180030BC70470368591C1A46016012F8021B37
:103628000260587841EA0020704703685A1C02601B
:103638001878704738B504460068154631F00FFD14
:1036480022682A44226038BD036810B40A0A5C1C48
:1036580004601A7003685A1C026019705DF8044B04
:10366800704703685A1C026010B4197003680A0A8C
:103678005C1C04601A7003680A0C5C1C04601A70F5
:103688000368090E5A1C026019705DF8044B7047F4
:1036980003685A1C026019700368090A5A1C026000
:1036A8001970704710EE103AC3F3160242F07E52BA
:1036B80007EE102ADFED167ADFED164A9FED165A4F
:1036C800DFED165A9FED166ADFED163ADFED166A42
:1036D8009FED164AE7EE274ADB1507EE903AA4EE6F
:1036E800875AF8EEE77AE5EE075A67EEA37AA5EE71
:1036F800876AB5EEC00AE6EE077AF1EE10FAD4BF93
:10370800B0EE440AB0EE660A37EE800A704700BF92
:10371800DACDFE3CB9D593BE5CB8903FAA841DC0F3
:1037280022E061401872313F07F1B3C2000080FF08
:10373800DFED1D3ADFED1D7A9FED1D7A9FED1D4AE5
:10374800DFED1D4A9FED1D5ADFED1D5A9FED1D6AE5
:10375800DFED1D6AE0EE237AF4EEC77AF1EE10FA97
:1037680088BFF0EE477AF4EEC47AF1EE10FAB8BFEB
:10377800F0EE447AFDEEE77A17EE903AC3F31602BC
:1037880042F07E5207EE102AA7EE245A03F0FF43B8
:1037980000EE103AE5EE075AA5EE876AE6EE076AEC
:1037A80026EE800A704700BF3BAA384B00007E4EC9
:1037B8000000FF4E00000000ED185E3C81900FBB3A
:1037C800AF9D2A3EB2D19F3EE886023F07EE901A8F
:1037D800F8EE677A9FED837A27EE800A20EE070AD3
:1037E800FDEEC07A17EE903A2033402B00F281802C
:1037F800DFED7D7AB4EEE70AF1EE10FA40F3E680E9
:10380800B0EE407A9FED796ADFED796A01E0B0EEBB
:10381800677AB4EEE67AF1EE10FA77EE467AF6DCDD
:103828009FED747AF4EEC77AF1EE10FA40F1D18088
:103838009FED6E6ADFED706A01E0F0EE477AF4EE14
:10384800E67AF1EE10FA37EE867AF6D4DFED6B7A87
:10385800B4EEE77AF1EE10FA40F3A780DFED627A72
:1038680037EEC77A27EE076ADFED655ADFED657A2E
:10387800DFED656A9FED655AE6EE257A67EE065A32
:10388800E6EE276AF7EE007AA5EEA67AF0EE675A1A
:10389800E7EE055AE7EE457A87EEA55ADFED577A47
:1038A80030EE277AFDEEC76A16EE903A2033402BA9
:1038B80024D99FED577AF6EE006AB7EE006AF7EE64
:1038C800004AC4EEA57A0023836143610362C361A1
:1038D80080ED045A67EEA66A27EE866A27EE877A95
:1038E800C0ED006AC0ED026A80ED016A80ED037ADE
:1038F8007047B7EE005AF0EE455ACFE7B4EEE70A44
:10390800F1EE10FA6BDD9FED396ADFED396A01E0FF
:10391800B0EE677AB4EEE67AF1EE10FA77EE467A10
:10392800F6DC9FED347AF4EEC77AF1EE10FA53D54F
:103938009FED2E6ADFED306A01E0F0EE477AF4EE93
:10394800E67AF1EE10FA37EE867AF6D4DFED2B7AC6
:10395800B4EEE77AF1EE10FA33DCDFED2E7AB4EE4E
:10396800E77AF1EE10FA44BFDFED227A37EEC77A34
:1039780027EE076ADFED224ADFED226ADFED227AC1
:10398800E6EE246A67EE064AE6EE267AB7EE006AA5
:10399800A4EEA77AF6EE006A36EE476AF8EE007AE9
:1039A80027EE277A66EE266A89E7DFED1A7AB4EE03
:1039B800E77AF1EE10FA44BFDFED0E7A37EEC77AF8
:1039C80050E7DFED097A37EEC77AD1E7F0EE407AB3
:1039D80026E7B0EE677A39E7B0EE677AB6E7F0EE39
:1039E800477A9EE727D4D236DB0F4940DB0FC94020
:1039F800E4CB1641DB0F49C0E4CB16C1DB0FC93F4E
:103A080092E741B99730083C15A82ABEF304353F20
:103A180000000000DB0FC9BFDFED2E7AB4EEE70A25
:103A2800F1EE10FA4ADDDFED2C6A9FED2C7A01E009
:103A3800B0EE670AB4EEC70AF1EE10FA70EE667AD5
:103A4800F6DC9FED277AF4EEC77AF1EE10FA3ED550
:103A5800DFED216A9FED237A01E0F0EE407AF4EE83
:103A6800C77AF1EE10FA37EEA60AF6D4DFED1E7A21
:103A7800B4EEE70AF1EE10FA14DDDFED167A37EE50
:103A8800C00A60EE006A9FED196A9FED197ADFEDB2
:103A9800197AA6EE867A20EE266AE6EE877AA6EEF0
:103AA800270A7047DFED147AB4EEE70AF1EE10FA50
:103AB80044BFDFED0B7A37EEC00AE2E79FED087AE4
:103AC800F0EE407AF4EEC77AF1EE10FAC0D4B0EE18
:103AD800670ACBE7DB0F4940DB0FC940E4CB16414F
:103AE800DB0F49C0E4CB16C1DB0FC93F92E741B9F0
:103AF8009730083C15A82ABEDB0FC9BF01212FF05B
:103B080009BF70B50D461446FDF736F90646A0B153
:103B1800FFF7F4FF40F634039842A8BF1846B0F503
:103B2800617FB8BF4FF461701923A0F5617090FBF5
:103B3800F3F028702378013323703046FDF71CF921
:103B48000646A0B1FFF7DAFF40F634039842A8BF53
:103B58001846B0F5617FB8BF4FF461701923A0F51E
:103B6800617090FBF3F0687023780133237030465E
:103B780070BD02B370B48E1803E0121B14D1B142A9
:103B880015D010F8012BA2F14103192B11F8013BB4
:103B9800A3F1410598BF2032192D03F12004ECD977
:103BA800D21A01D1002BEAD1104670BC704700220E
:103BB800104670BC70471046704770B504460846FA
:103BC8000D4630F0B1FB064602E014F8013F43B160
:103BD800324629462046FFF7CCFF0028F5D120467B
:103BE80070BD1C46204670BD4FF0FF32FFF7C1BFC5
:103BF800A0F16103192B98BF20387047A0F1410349
:103C0800192B98BF20307047202805D00938042880
:103C18008CBF0020012070470120704770B5044612
:103C280008460E4630F080FB3146054602462046DF
:103C3800FFF79FFF68B9635D1846FFF7E5FF00B916
:103C480033B901352C44204601340378202BFAD0AF
:103C580070BD0020FCE7613819288CBF00200120C6
:103C68007047413819288CBF002001207047303830
:103C780009288CBF002001207047A0F13003092BD0
:103C880007D920F02000413819288CBF00200120D6
:103C9800704701207047F8B5064615460846B6FB3A
:103CA800F2F434B905FB14640B4B1B5D00F8013BBF
:103CB800F8BDB4FBF2F75FB905FB1747064B05FBE8
:103CC8001464DA5D00F8012B1B5D00F8013BF8BDB8
:103CD8003846FFF7E0FFEFE700980308B5EEC00AA3
:103CE800DFED677A674AF1EE10FACCBF30EE270AAB
:103CF80030EE670ADFED647A20EE270A2DE9F047F7
:103D0800FDEEC07A88B017EE904A84EAE476002384
:103D1800A6EBE476CDE902330493A2FB06325FEA10
:103D2800D208054641D105AF58483946554BA3FB43
:103D38000623DB0803EB8303A6EB4303002CC35CD9
:103D48000B704FF00002ACBF20232D234A70384679
:103D58008DF8083030F0E8FA0128394639D00228C1
:103D680042D0032805BF302302A802A88DF80930E5
:103D780031F0A1F902A830F0D7FA0338C4B22246CC
:103D880002A9284631F0CDF900232B55284630F0FA
:103D9800CBFA2E22431C02A92A542144E81831F0F8
:103DA800A6F9284608B0BDE8F087394BA3FB0623DF
:103DB8005B0922D105AF35483946324AA2FB0832A1
:103DC800D20802EB8202A8EB4202835C01F8013BB5
:103DD800ACE7302302A88DF809308DF80A308DF849
:103DE8000B3031F068F9C5E7302302A88DF80930A7
:103DF8008DF80A3031F05FF9BCE7264AA2FB0612BB
:103E08005FEA92190ED105AF204839461D4AA2FB38
:103E180003C2D20802EB8202A3EB4203C35C01F89F
:103E2800013BCAE71C4AA2FB06125FEA523A0ED1CE
:103E380005AF16483946134AA2FB09C2D20802EB5D
:103E48008202A9EB4202825C01F8012BDEE71348EB
:103E5800B6FBF0F058B905AF39460A20BAFBF0F2C4
:103E680000FB12A20948825C01F8012BE3E705AFC9
:103E780039460A220193FFF70EFF019B0146ECE742
:103E88006F12033ACDCCCCCC00007A4400980308DA
:103E98001F85EB51D34D62105917B7D1A086010089
:103EA80070B406688E4217D90139751E002311F8BF
:103EB800014F0822634013F0800F4FEA430318BFF5
:103EC80083F0D503013ADBB2F5D18D42EFD1721CF4
:103ED8000260337070BC7047721C0023026033703C
:103EE80070BC70470A44914215D010B40139541E71
:103EF80011F8012F0823504010F0800F4FEA4000BE
:103F080018BF80F0D500013BC0B2F5D1A142EFD176
:103F18005DF8044B704770474840082310F0800F45
:103F28004FEA400018BF80F0D500013BC0B2F5D180
:103F380070470A44914215D030B40139551E41F2F8
:103F4800210211F8014F082380EA042004044CBF21
:103F580082EA40004000013B80B2F7D18D42F0D1A7
:103F680030BC7047704770B502221449144C154E86
:103F78004FF6FF70FFF7DDFF22884AB1A518B5425A
:103F880019D2052A17D92146FFF7D3FF2C46F3E7A4
:103F980021460222FFF7CDFF0222A118FFF7C9FF31
:103FA800094BE41A094BA3F8644041F60F53C31AAE
:103FB8005842584170BD0020FCE700BF00F00308DC
:103FC80002F0030800000408FAEF0308300F00208D
:103FD8002DE9F043002489B006460D461F46A04649
:103FE80005E025290CD030460134A847039A531C14
:103FF800039311780029F4D1204609B0BDE8F08375
:10400800931CCDE903385078302842D0A0F1300312
:10401800DBB2092B4FF0000945D96C282AD0642857
:1040280073D019D9732858D063D9752840F0828085
:1040380007F1040C386805AB00220A216746FCF733
:10404800F3FA05AB049A009329464B463046FCF731
:104058003CFB039A0444CAE725283CD051D9582888
:104068006BD06328C2D139783046A8470437013469
:10407800039ABCE7039B5A1C03921B78642B52D00B
:1040880016D8252B27D064D9582B18D0632BEAD003
:10409800ADE7D31C03939078A0F13003DBB2092B72
:1040A8004FF00109B9D804AA03A92CF05CFEB4E7C3
:1040B800732B12D051D9752B2DD0782B97D1A3F112
:1040C8005802B2FA82F23868520905AB1021043757
:1040D800FCF7AAFAB5E7252185E73B68049A00931F
:1040E800294600233046FCF7F0FA04370444039AC3
:1040F8007DE76E287FF47AAF039A3B6804371C602B
:1041080075E700283FF478AF70E7386805A9FCF731
:1041180055FA043795E7386805AB00220A21FCF701
:1041280083FA04378DE73B1D386805A91F46FCF75D
:1041380045FA86E778287FF459AFA0F15802B2FA19
:1041480082F23868520905AB1021FCF76DFA043782
:1041580077E7002B3FF450AF49E76E2BCDD046E709
:1041680010B5064C0B46024605492068FFF730FF9C
:104178002068BDE81040FFF7FFB800BFA825002061
:104188007F03000838B504460D460848FFF740F994
:1041980029462046FFF7E4FF0548FFF739F9054BA4
:1041A8001B7813B1044B01221A7038BD108E030816
:1041B8001B8E030804270020052700200FB407B52D
:1041C80004A951F8040B0191FFF7DCFFFFF776F91A
:1041D80003B05DF804EB04B0704738B50F4D2B7889
:1041E80063B10F4C23784BB10E48FFF7E7FF0E4839
:1041F800FFF7E4FF00232B70237038BD0B4B93F8B7
:1042080066203AB1986E10F0BDFE0020BDE8384037
:10421800FFF70EB910F0D4FDF7E700BF0427002020
:10422800052700201F8E0308568E0308300F002034
:1042380038B5052215490446FFF79BFC58B9144ABE
:1042480013781BB901211170124A13701248BDE886
:104258003840FFF747B9032210492046FFF789FC89
:1042680080B90B4C0B4D227842B12B7833B10C48F6
:10427800FFF7A4FF002323702B7038BD0948FFF710
:1042880031F9F7E70848BDE8384097E7129703087F
:104298000427002005270020748E03087897030858
:1042A8001F8E03088A8E03089E8E0308004885E740
:1042B800AD8E03080FB407B504A951F8040B01919A
:1042C800FFF760FF03B05DF804EB04B070470FB46C
:1042D80007B504A951F8040B0191FFF741FFFFF757
:1042E800EDF803B05DF804EB04B0704710B5104C5E
:1042F80003461846FBF7A6FF58B10E4B0E4893F934
:1043080001104B1C0ABF0D4BC9B25978BDE81040CB
:10431800DDE71846FFF7F2FB052804D8C0B227F0FE
:1043280003F92346E5E705210548BDE8104045E7C0
:10433800E993030800000020B98E03085C290020D7
:10434800C88E030810B5104C03461846FBF77AFFD1
:1043580058B10E4B0E4893F900104B1C0ABF0D4B79
:10436800C9B21978BDE81040B1E71846FFF7C6FB97
:10437800022804D8C0B212F04EF92346E5E702211C
:104388000548BDE8104019E7E9930308000000203C
:10439800BD8E03085C290020CD8E030838B50D4674
:1043A800FFF7ACFB0C4B19788842044605D201464E
:1043B8000A48FFF78CFF204638BD2DB1FF2803D1EE
:1043C8000748FFF784FFF6E701390648FFF7F6FECE
:1043D8004FF0FF34EFE700BF51270020E88E0308B5
:1043E800F98E03080C8F03082DE9F3410346FBF708
:1043F80029FF044620B1FFF759FF02B0BDE8F0815C
:1044080001AA2B49DFF8A880184630F083FD27461B
:10441800054626467DB9022CEDD1A7F57A73B3F58A
:104428007A7F20D94FF4FA634FF47A7221492248EF
:10443800FFF7C4FEE1E74CB1012C0FD001AA4146B9
:10444800002030F067FD01340546E3E701212846E6
:10445800FFF7A4FF431C0646F0D1CEE72846FFF736
:104468004DFB0746EAE7B8B21CF0F0F9FF2EBCEEA8
:10447800C00A124B0BD1124AF8EE407A1278AA42BF
:1044880012DC10EE101A0F48FFF721FFB5E7F8EE1F
:10449800407A03EB860310EE102A31460A48C3ED32
:1044A800007AFFF714FFA8E7E3EC017A0135E6E7A5
:1044B80032960308B2970308328F0308E8340020C5
:1044C80051270020588F03084B8F03082DE9F34725
:1044D8000346FBF7B7FE044610B1FFF7E7FE25E0F9
:1044E80001AA2A49DFF8B480DFF8B490DFF8B4A055
:1044F800184630F00FFD26460546274655B9244B89
:104508003246A1B218682EF06DFD78B92148FFF740
:1045180055FE0BE06FB1012FDFD1B31E594259414F
:104528002846FFF73BFF421C044622D102B0BDE8F3
:10453800F08728462FF0F8FE4146064602462846F0
:10454800FFF717FBA0B1324649462846FFF711FB93
:10455800B8B1324651462846FFF70BFB98B13246B0
:104568000D492846FFF705FB0028B6D1032600E0D1
:104578003E4601AA0549002030F0CCFC013705462B
:10458800BCE70126F5E70226F3E700BF32960308E9
:10459800AC250020738F0308708F0308678F03080A
:1045A8006A8F03086D8F03082DE9F3470346FBF76D
:1045B80049FE044618B92B4A9278042A04D8FFF712
:1045C80075FE02B0BDE8F08701AA2749DFF8AC8084
:1045D800DFF8AC90DFF8ACA0184630F09BFC012760
:1045E800264640B9214B224A1B689B1A214A18BF0C
:1045F80001231370E5E766B90121FFF7CFFE431CDD
:104608000446DED001AA18490020013630F082FCA9
:10461800E7E7FFF773FA2F2805461ED8D7B126F02B
:10462800C1FC062D06D1052012F064FC5046FEF7A9
:1046380059FF09E0012012F05DFC0F490123EAB29D
:104648000978E0B226F064F829464846FFF73FFEAD
:104658000027D7E70628F0D1E8E72F214046FFF7E3
:10466800ADFDCFE7A85D002032960308C45D0020A9
:10467800199E0208986A002051270020B18F03086C
:10468800A08F0308918F03082DE9FF4107462FF0FB
:104698004BFE08283CD1002201AEB85CFFF7A8FA0F
:1046A800B0540132082AF8D10024DFF870808DF860
:1046B8000C40385DFFF79CFAC5B230552946404694
:1046C80030F008FD28B101342946301930F002FDD8
:1046D80020B1FFF7EBFD04B0BDE8F081082CE8D16C
:1046E8000D4930460BF078FD0B4C0C4800231A5D41
:1046F80004A90A44195C02F80C1C0133082BF6D1F2
:10470800002301A906488DF80C30FFF7E0FDE2E729
:104718000028E9D0DDE700BFE82D002090700308ED
:10472800D18F0308034B044A04491B6812680968BF
:104738000348CCE5B4F7FF1FB0F7FF1FACF7FF1F26
:10474800D88F0308F7B50646FBF77CFD054658B138
:10475800002401A920462EF091FA0134FFF7F2FF58
:10476800122CF6D103B0F0BD3046FFF7C7F9C4B23A
:10477800112C61D8701CFCF7FFFA334D0746D0B9ED
:10478800324B13F814108A1E514251412F4B13F823
:104798001420154495F8A120002948D003EB4403C0
:1047A80019205B7840F2EE2100FB031321462848CC
:1047B800FFF78DFDD6E705F1A1060178304630F008
:1047C80089FC58B1032C8CBF03230023801B2B4486
:1047D80053FA80F090F8A560032E02D1FFF766FD2A
:1047E800C0E73846FCF7C8FAF0B1022EF6D1FFF759
:1047F80085F940F6CA0280B29042144BA8BF104611
:1048080040F2EE22904203EB4403B8BF1046A0F2F8
:10481800EE20192290FBF2F05870B31E594259410C
:104828000A4B03F81460B1E7022EF6D1D6E7214609
:104838000848FFF74CFD95E711232A460649074823
:10484800FFF7BCFC8EE700BF54510308402000204E
:10485800EC8F0308FC8F030809900308328F0308C4
:104868000FB407B504A951F8040B0191FFF778FCC0
:1048780003B05DF804EB04B070472DE9F843044633
:104888002FF052FD024680B320461949FFF771F90F
:10489800044650BBFEF712FE1648174D174E184F28
:1048A800DFF86480FEF71EFE2B7D072194FBF1F1F3
:1048B800C1EBC10206EB8303A21A0132013138466B
:1048C800D3F8AC90FFF7CCFF6A7D49464AB10D4852
:1048D800FFF7FDFC01340C2C05F11C05E4D1BDE803
:1048E800F8834046FFF7F3FCF4E7BDE8F843DDE45E
:1048F8001190030816900308B00B002054510308C8
:104908001B9003082D9003089791030838B50B4BAB
:1049180003EBC0040D4694F8A021094803EB820379
:10492800D3F8AC10FFF79CFF94F8A63123B1691CAB
:104938000448BDE8384093E738BD00BF5451030828
:1049480098910308B59403087FB50B4B04930B4B60
:1049580003930B4B02930B4B01930B4B00930B4AA6
:104968000B4B0C490C48FFF77BFF0C48082107B09C
:104978005DF804EBABE400BF789003087D90030872
:1049880087900308909003089C90030834900308CC
:1049980063290020429003084D900308A290030861
:1049A8002DE9F04F93B00025DFF8A4B1DFF8C0A1DE
:1049B800DFF8C0910795A84608A9E8B226F040FF9D
:1049C8009DF82830002B6DD0022D40F09A809DED87
:1049D800117AB5EE407AF1EE10FA00F08980DFED39
:1049E800586AC6EE877AFDEEE77AF8EEE77AFDEECA
:1049F800E77A17EE906A99F80040089B012C79D95C
:104A080096FBF4F41A4602214E48FFF729FF0D9A47
:104A1800002A00F08B8041F2883002FB04004FF43A
:104A28007A73B0FBF3F00F9B002B00F0818041F20A
:104A3800883103FB04114FF47A7CB1FBFCF1062D9D
:104A480003D0079F0F44804407979BF803C0BCF12D
:104A5800000F6FD04FF47A7C0E9FB7FBFCFCCDF8AB
:104A680010C04FF00A0C91FBFCFE0CFB1E11CDE9A7
:104A780002E190FBFCF10CFB1100CDE9001021468E
:104A88003148FFF724FC022D08D199F80030012B9A
:104A980004D9324609992D48FFF719FC0AEB85130A
:104AA80000229A630135182D86D1294BDB78E3B1B2
:104AB800284B29481968294B1A684FF47A73B1FBB7
:104AC800F3F3274952090968FFF701FC0798079B88
:104AD8000A2293FBF2F302FB130798FBF2F100970B
:104AE80002FB11821F48FFF7F2FB13B0BDE8F08FFD
:104AF800002680E7099A1C480221FFF7B1FE3446D8
:104B080085E7109C5CB107EE904ADFED0D6AF8EE80
:104B1800677A86EEA77AFDEEC77A17EE904A089A6A
:104B280008482946FFF79CFE002670E710467AE7FA
:104B3800194684E721460D48FFF7C9FBA3E700BFE4
:104B480000247449BA900308DC9003080091030814
:104B58005C290020E83E002010910308E03E002078
:104B6800EC3E002030910308C99003080C9103081B
:104B780098000020881E00202DE9F047214FDFF81B
:104B8800A480DFF88490DFF8A0A0054628462FF01F
:104B9800CBFB064658B91C4B1C481A781C4B03EB38
:104BA8008203BDE8F047D3F87412FFF790BB0246C2
:104BB80039462846FEF7DDFF78B91648164C174DDA
:104BC800FEF726FC54F8041F19B12846FFF748FEE3
:104BD800F8E7BDE8F047FEF771BC002458F8241048
:104BE80021B90F48BDE8F047FFF7E8BA3246284632
:104BF800FEF7BFFF01340028F0D189F80040554680
:104C0800C4E700BF68910308D41B00205E91030825
:104C1800545103086D910308C8530308979103087A
:104C280078910308CC530308E99303082DE9F84F5A
:104C380080460E4617462FF077FB0446F0B94048E9
:104C4800404FDFF82081FFF70BFE0C2520460EF0C1
:104C58007FF83368184205D005FB0473404699680D
:104C6800FFF7FEFD0134182CF0D1336813B936482C
:104C7800FEF7CEFBBDE8F84FFEF720BC02463349ED
:104C88004046FEF776FF0546B0B931482D4EDFF8AD
:104C9800C880FEF7BDFB2C460C2520460EF058F8C0
:104CA800384205D005FB046340469968FFF7D8FDF4
:104CB8000134192CF1D1DDE798F800302D2B03BF12
:104CC80008F1010804F1FF34012500254FF0000A1E
:104CD80047F0807B1B4B0C2202FB0A324046D2F87D
:104CE800089022464946FEF744FFF8B950460EF0B0
:104CF8002FF81BEA000F19D075B1BAF1180F1CBFB5
:104D08003768074337601348FEF782FB4946124865
:104D1800BDE8F84FFFF7DBBABAF1180F1CBF3568CA
:104D2800854335600D48FEF773FBEFE70AF1010A8A
:104D3800BAF1190FCED10A48BDE8F84FFFF73EBACD
:104D480085910308508203088F910308689103082E
:104D58006D9103089B91030897910308A491030898
:104D680078910308969103086FF07F4200495DE748
:104D78003037002040F20222004957E73837002038
:104D88002DE9F047424D07462FF0CEFA414B95F8F2
:104D980066801E680446B8F1000F15D0D5F86890F3
:104DA800C4B93D483D4D3E4FFEF732FB012655F84C
:104DB800241059B106FA04F313EA090F02D0384651
:104DC800FFF74EFD0134F2E7B146E9E7BDE8F047E9
:104DD800FEF774BB224633493846FEF7CAFE78B957
:104DE8003148324C324DFEF713FB54F8041F0029AA
:104DF800ECD00B78002BF8D02846FFF731FDF4E70C
:104E0800B8F1000F03D10123AE6685F866303B7810
:104E1800DFF888A02D2B03BF013704F1FF344FF0D2
:104E280001094FF000094FF000085AF8286026B928
:104E38002048BDE8F047FFF7C1B922463146384659
:104E4800FEF797FE08BB012303FA08F2110604D502
:104E58001948BDE8F047FEF745BB9305F8D4AB6E9B
:104E6800B9F1000F0BD023EA02031448AB66FEF732
:104E7800CFFA31460E48BDE8F047FFF728BA13438A
:104E88000F48AB66FEF7C4FAF3E708F10108CCE770
:104E9800300F0020B85B0020AC9103083854030899
:104EA800B6910308689103086D9103083454030808
:104EB8009791030878910308BA9103089B91030816
:104EC800A491030830B52C4885B0FEF7A1FA15F077
:104ED800B3FC28B9294805B0BDE83040FEF702BB4D
:104EE80015F0A0FC08B92648F5E7264B1B68DB69D6
:104EF80098470028F7D015F08DFC0268037D81796A
:104F08000446407C0290207C0190608A0090520800
:104F18001D48FFF7A5FCE51D0C3415F8010BFEF73D
:104F28006FFAAC42F9D1194C1948FEF771FA627858
:104F3800032A06D8DFE802F00E0E0A021548FEF72B
:104F480067FA05B0BDE83040FEF7B8BA1248FEF778
:104F58005FFAF6E71148FEF75BFA41F2D453E35CD7
:104F6800022B05D0032BECD10D48FEF751FAE8E7E8
:104F78000C48FEF74DFAE4E7C6910308D091030800
:104F8800DE910308602A0020ED910308BC6D002023
:104F98001B9203082B920308319203083E920308E0
:104FA8005D92030844920308F0B5482285B047494A
:104FB8004748FFF755FCFEF781FA464A46494748F5
:104FC800FFF74EFCFEF77AFA454B464A4648D21A96
:104FD800464BB3F86410FFF77AF9454B4548196812
:104FE8004FF47A73B1FBF3F1FFF73AFCFEF766FA78
:104FF8004149D1F89C20002A58D007EE902ADFEDCD
:105008003F6AB8EEE77AC6EE877AFDEEE77ACDED2D
:10501800037A3B4B1B885BB107EE903ADFED376AAA
:10502800F8EE677A86EEA77AFDEEC77A17EE903A21
:10503800C96959B107EE901ADFED306AF8EEE77AE0
:1050480086EEA77AFDEEC77A17EE901A2D482E4EF7
:1050580000882E4F6428CDE900310146039B2C4877
:10506800A8BF6421FFF733F92A4B2B491A782B4B39
:1050780009882B4803EB82032A4AD3F86033127855
:10508800FFF725F9284B29481988FFF720F9002050
:10509800FFF718FF2648FEF7BBF9264B1C680125C9
:1050A80034B905B0BDE8F040FEF708BA0392B0E79E
:1050B80094FAA4F3B3FA83F305FA03F256F823102B
:1050C800384624EA0204FFF7CBFBE9E76F920308AE
:1050D800749203080020001000080000879203085B
:1050E80000F0030800000408AB920308300F00200A
:1050F800A44E0020D592030898000020002474498B
:10510800BA390020EE360020347F0308979103084F
:10511800EF9203086C2900205029002054510308FD
:10512800359303086D290020602400205C93030850
:105138006B9303080C2B00202DE9F04F87B0034632
:10514800FBF780F8074620B1FFF7B0F807B0BDE8D5
:10515800F08F05AA7F49DFF840A2DFF840B2184671
:105168002FF0D8FEB84681463D463E464FF0FF3404
:10517800B9F1000F28D178482146FFF771FB774A2B
:1051880060B24B4602EBC30191F90610814200F070
:10519800BD800133042BF5D1002E14BFB0464FF467
:1051A8006148002D08BF03250023EDB20293CDE925
:1051B80000851A4619460DF03DFC0446002838D1F2
:1051C8006748FEF78FF9C1E7B8F1030F07D8DFE8A2
:1051D80008F0020F14244846FEF790FC044605AA7E
:1051E8005C4900202FF096FE08F101088146BFE7D0
:1051F8004846FEF783FC0646F1E751464846FEF767
:10520800DCFC08B145F0010559464846FEF7D5FCD7
:105218000028E4D045F00205E1E748462FF084F87D
:10522800504902464846FEF7A4FC002808BF01275B
:10523800D5E7414676B94C48FFF712FB4B48FEF7D5
:1052480051F94B4B186803681B6A33B12246494928
:10525800984702E04848FFF703FB484B484949484C
:10526800434D002F18BF1946FFF731F837B12868AA
:105278000368DB6913B10022434998472D68284623
:1052880011F0DCFE204611F0D9FE00210846FCF79B
:105298003FFC00210120FCF73BFC2846FBF799FE68
:1052A800A0B101210020FCF733FC2846FBF78BFE58
:1052B80006462046FBF78AFE0028FAD031462046EB
:1052C800FBF78AFE00210846FCF722FC2046FBF784
:1052D80080FE0028E1D001210020FCF719FC2046BF
:1052E800FBF771FE06462846FBF770FE0028FAD049
:1052F80031462846FBF770FE00210846FCF708FCFB
:10530800CBE7A1682148FFF7ABFA0EE052F833402B
:10531800002C3FF441AF002EF3D031461C48FFF774
:105328009FFA31462046FAF763FF5DB12179A94219
:1053380008D018482A46FFF793FA2368E9B29B6910
:1053480020469847E36A0BB10023E362002E84D11C
:1053580074E700BF329603089A930308186C00207C
:10536800A393030894930308B89303084694030887
:10537800AC250020F9010008D593030881930308A0
:10538800E993030869940308370200080D94030899
:10539800EA930308289403088E930308919303085B
:1053A8002DE9F041037903F06002202A2CD002D8BD
:1053B80052B1BDE8F081402A4AD0602AF9D1274885
:1053C800BDE8F041FEF783BF03F00703022B02D0CC
:1053D800042B09D07BB9B0F80720B0F80510204895
:1053E800BDE8F041FEF773BFD0F805101D48BDE8D1
:1053F800F041FEF76CBFB0F90720B0F90510184866
:10540800BDE8F041FEF763BF4679174D174805EB35
:10541800C605FDF7FDFF95F8787300240123A74220
:1054280003D8BDE8F041FEF749B8D5F8746356F8DB
:1054380024204FEA84084AB113B90D48FDF7E8FF64
:1054480056F808100B48FFF70BFA00230134E6E77B
:1054580041790948BDE8F041FEF739BFDE940308F9
:10546800A29403088C94030854510308B9940308C0
:10547800CA94030898910308CD9403082DE9F041D4
:105488001746027902F06003402B05460C462BD1E3
:105498000026554FDFF8708115E02B7903F00703DC
:1054A800022B15D0032B19D0012B14BFA15DA157D6
:1054B8003846FFF7D5F96B79013BB34202DD404628
:1054C800FDF7A6FF01366B79B342E6DCBDE8F08153
:1054D80034F816103846FFF7C3F9ECE734F916101C
:1054E8003846FFF7BDF9E6E702F00702042A6DD84F
:1054F800DFE802F0031F282A2D002478202B3ED055
:10550800602B4CD0002BE1D1B5F80560B5F80780C9
:1055180035482146FFF7A4F9A6424EDCA0454CDBEE
:10552800002FD3D0424631463048BDE8F041FFF75E
:1055380097B994F90040202B21D0602B2FD0002B55
:10554800C4D14BE02488D9E7B4F90040F3E72668D2
:10555800202B344613D0602B21D0002BB6D13146F6
:105568002348FFF77DF9D5F805108E4225D8002F7E
:10557800ACD02048BDE8F041FFF772B900246A7941
:105588001D4B03EBC20393F87823A24215DDD3F831
:10559800743353F82400BDE8F041FDF739BF6A7948
:1055A8001441E30704D51548BDE8F041FFF758B9A1
:1055B8001348BDE8F041FFF753B9FDF77FFF2246D6
:1055C80029681048BDE8F041FEF774BE202BD5D0FD
:1055D800602BEDD0002B7FF479AF1C46B5F9056040
:1055E800B5F9078094E700BFB69403080B96030843
:1055F8009F940308F894030854510308F39403088C
:10560800FE94030802950308F694030838B50D467E
:105618000446FBF7E1F82A4601462046BDE8384033
:105628002CE72DE9F74FDFF8C4B081468A460025FC
:10563800D8462B4B0D2418686C43FDF79DFE04EBF0
:105648000B031B7903F018034B4504D0B9F1000F85
:105658003ED1182B3CD10D2303FB05820093B2F8F1
:105668000900FBF7A2F8444407462046FAF7F2FD82
:10567800D7E901210646024401442046FAF722FEF2
:105688001AF0100F0246009B00D008BB03FB0583ED
:105698001AF0200F1B680FD072B9194611480093F1
:1056A8000192FFF7DDF87968019A31442046FFF747
:1056B800E5FEFDF703FF009B0B481946FFF7D0F8FE
:1056C800B968002231442046FFF7D8FEFDF7F6FE00
:1056D8000135B5F5B37FACD103B0BDE8F08F00BF9D
:1056E800A82500201C9503081D9503088058030869
:1056F800052838B50D460CD8064C60700648FEF7EC
:10570800F5FDFDF7DBFE29461020FFF78AFFFF2392
:10571800637038BD00000020E9930308022838B5FB
:105728000D460CD8064C20700648FEF70BFEFDF718
:10573800C5FE29460820FFF774FFFF23237038BDF4
:1057480000000020E99303080CB407B510F020000E
:105758000BD079B92320FDF753FE05A904980191D0
:10576800FEF7FEFCFDF7AAFE012003B05DF804EB8E
:1057780002B070470020F8E70CB4C30607B500D59F
:1057880061B905A904980191FEF7EAFCFDF796FEB8
:10579800012003B05DF804EB02B070470020F8E781
:1057A8002DE9F04F354C87B08046354A237860881C
:1057B80002EB8303D3F8AC90FAF7F7FFD0E901A323
:1057C8000493304B1B7813B9CDF810A09A4608F013
:1057D8004003DFF8BCB005930026A379002B08BF6F
:1057E80001239E4206DB284B08349C42DDD107B0DA
:1057F800BDE8F08F6279237906FB0323049A01360A
:10580800D55CBAF1000F11D1B5FA85F77F090DB350
:1058180005F00F032D0940350293CDE900654B468D
:105828005A4639464046FFF7A7FFD6E71AF803302D
:10583800EA1A57425741C3B103F00F021B0940331C
:105848000292CDE900635A464B4639464046FFF777
:105858007BFFDCE7059B002BBFD100964B460B4A2C
:1058680039464046FFF788FFB7E700964B46074A98
:1058780039464046FFF768FFC9E700BFF4520308FE
:1058880054510308300F0020CC5303083D950308FA
:10589800279503082DE9F04F87B005AA8C492FF00A
:1058A80039FB064628B94120FFF77AFF07B0BDE863
:1058B800F08F8849DFF86082FEF796F988BB864842
:1058C800864C874E874FFDF70DFE04F59875A37932
:1058D8002168A28808EB830301F13841B2FA82F209
:1058E800890A4131D3F8AC30C2F11F023046FEF7C5
:1058F800B7FFE17911B13846FEF7B2FF0834FDF77A
:10590800DDFDA542E3D1724905AA00202FF002FB74
:105918007549FEF769F90028C8D16E48FEF7ADFF52
:10592800C4E708F5D0770024B94617F8343008EBF7
:105938008303E500D3F8ACA050462EF0F5FC5146A1
:1059480002463046FEF715F938B101341B2CECD16C
:1059580031466648FEF732FCA8E705AA5C492FF0F5
:10596800D9FAA8440746FEF7C9F898F8A6310646BA
:10597800002B40F09880002800F39F80A944B9F8D4
:105988000200FAF712FF3D78002D00F08980F3B28B
:10599800019399F8046099F80530019AD0F80480C9
:1059A8005349384602FB0636FEF71EF960B908F877
:1059B800060018F80680B8F1000F16D14D48FDF71B
:1059C80091FD73E7012372E0602D8CBF613D413D7D
:1059D800072D65D8781CFEF791F80F2860D8013597
:1059E80040EA051508F80650E3E74046FBF7B0FC27
:1059F8008146002854D04FEA1813403302933E4F93
:105A080008F00F030026039300252EE07888FAF7A4
:105A1800CCFE7A793B7905FB03234268D15C41458A
:105A280022D1B44204D101998D421DD00021D15414
:105A3800DDE9021231485FFA85FB5FFA86FAFEF764
:105A48000FFF59465046FEF761FFB44209D12C4872
:105A5800FEF706FF50465946FEF758FF2948FEF75D
:105A6800FFFE2948FDF73EFD0135BB79002B08BF35
:105A780001239D42CADB01361B2E07F10807C3D15B
:105A8800D9F80010B9F80420204801F13841B2FAD9
:105A980082F2890AC2F11F024131FEF718FC05E7BC
:105AA800FEF704FC02E7002801DD9E4207DD012223
:105AB80017491848FEF782FBF8E6012882D105AAA3
:105AC800034900202FF026FA013E074656E700BF9B
:105AD800329603081190030851950308A84E002038
:105AE80054950308B59403085F9503086395030864
:105AF8004C95030885950308F45203088B95030811
:105B0800AF950308B295030883BA0308BC95030848
:105B18007F950308328F0308545103082DE9F04F8D
:105B28004A4085B098461D4FD34306460D4600248B
:105B3800039320460DF00CF90E9B184228D0039BC6
:105B4800174ADFF860A0034214BF4FF001094FF075
:105B5800000910EA050302934FF00C0303FB04232A
:105B68004946D3F808B0CDF800B014BF3A465246BB
:105B780043463046FFF7E8FD029ACDF800B04346A9
:105B8800002A14BF52463A4649463046FFF7F4FD0C
:105B98000134182CCDD105B0BDE8F08F80960308EC
:105BA80050820308C895030870B506462EF0BCFB62
:105BB800114C054690B11122002120462FF073FAAE
:105BC8002A460E4930462FF09AFA38B1102D2A4647
:105BD800314628BF102220462FF0A3FA2378064A20
:105BE800002B08BF0121054B1CBF002113460120D3
:105BF800034ABDE87040BFE5A42E002087CB030808
:105C0800D795030870B505462EF08EFB044690B173
:105C1800112200210F482FF046FA22460E49284645
:105C28002FF06DFA38B1102C2246294628BF1022D1
:105C380008482FF076FA094B13F8112F002A064A64
:105C480006BF012113460021054A0120BDE8704026
:105C580092E500BFB52E002087CB0308A42E0020B4
:105C6800CF9503082DE9F04F002489B0834692466A
:105C78000D4626464FF019094FF46178BAF1000F26
:105C880022D004EB84030AEB030705223946284691
:105C980007932FF0D5F93A79079B19FB02820492F2
:105CA800FA781AF8033019FB02820392BA78029242
:105CB800B0FA80F67A78019276090093104A234662
:105CC80031465846FFF740FD2B790D4A19FB0383EF
:105CD8000493EB7819FB03830393AB7802936B78F7
:105CE800019315F8053B0093314623465846013485
:105CF800FFF742FD0A2CC1D109B0BDE8F08F00BF03
:105D0800DF9503082DE9F0478AB08246FAF79AFA38
:105D1800064638B1002247490120FFF7A3FF0AB021
:105D2800BDE8F0875046FDF7E9FE092804467ADC0D
:105D3800850005EB00080AF101008DF81F60FBF7EC
:105D48001BF83C4F824608EB07093E4650B1FDF769
:105D5800D5FE0D2806D89DF81F3008F80700013336
:105D68008DF81F305046FBF707F8824658B1FDF70B
:105D7800C5FE052807D82B19334458709DF81F30E5
:105D880001338DF81F305046FAF7F6FF824658B1B6
:105D9800FDF7B4FE082807D82B19334498709DF8EE
:105DA8001F3001338DF81F3008F103010DF11F0278
:105DB80031445046FDF7A5FE9DF81F20052A2AD13B
:105DC800002308A9484608938DF824302FF038F9A5
:105DD8002B19334493F801C020B1BCF1000F1AD03D
:105DE8009B78C3B1254472194FF461701179192356
:105DF80013FB01010491D17813FB010303939378FA
:105E08000D4ACDE901C30021735D0093084623467E
:105E1800FFF7B2FC83E7002348F8073089F804301D
:105E2800FEF744FA7BE70923324604490448FEF7A3
:105E3800C5F974E768390020DF9503087F950308E2
:105E4800328F03082DE9F047344F8CB00646894657
:105E580015460024C4EBC40309EB030210689188BB
:105E68009279089040F30748ADF824108DF8262061
:105E7800B8F1000F4AD0002D4DD02B440AA918685C
:105E88009A880A909B79ADF82C2008A807228DF8EB
:105E98002E302FF0D5F89DF82E3006939DF92D3031
:105EA80005939DF92C3004939DF82B3003939DF9AD
:105EB8002A300293B0FA80FA9DF8293001934FEA0C
:105EC8005A1A9DF8283000933A46234651463046E0
:105ED800FFF73AFC9DF8263006939DF92530059387
:105EE8009DF9243004939DF82330CDE902839DF871
:105EF800213001939DF8203000933A4623465146BD
:105F080030460134FFF738FC102CA3D10CB0BDE8A3
:105F1800F047FDF7D3BAAA46DCE700BFF5950308BA
:105F28002DE9F0478AB005462EF0FEF9024630B951
:105F380085490120FFF786FF0AB0BDE8F0870522F2
:105F480082492846FDF715FE044670B901467022BD
:105F58007D482FF0A8F87E4B1C60DC609C615C6279
:105F68001C63DC639C645C65E6E704227949284687
:105F7800FDF7FFFD044620BB2846FAF7FDFE07465D
:105F88000028D9D02EF0D0F9DFF8EC81064658F871
:105F980024501DB97048FEF711F9CDE7324629465D
:105FA8003846FDF7E6FD50B9204619F0EDFC2946C4
:105FB8006A48FEF78CF96A48FFF7B2FFBCE701347C
:105FC800E5E7072267492846FDF7D3FD0446002880
:105FD8006ED1284620212FF07DF8054680BB624807
:105FE800FEF73EFC2C46614D214628460134FEF75B
:105FF80037FC0E2CF8D1FDF761FA554EDFF87C918D
:106008005B4FDFF87C81002421464846FEF728FCD8
:10601800DFF870A1002532680123AB40134214BF9A
:106028003946414650460135FEF71AFC0E2DF2D18D
:106038000134FDF743FA082C06F10C06E4D17BE79E
:1060480001AA4C494B4E2EF065FF02AD00283AD00C
:10605800022C15D1029A072A35D803990D2932D86E
:106068000378722B17D06E2B2DD10C23534338484D
:10607800012202FA01F1C25822EA0102C25013E0D9
:10608800FDF73CFD01AA45F82400314600202EF01A
:1060980041FF0134DAE70C232D4C5343012000FA69
:1060A80001F1E0580843E0502E48FFF739FF43E775
:1060B800284601AA2F492F4E2EF02CFF002402ADAE
:1060C80078B1082C02D1FEF7F1F835E7FDF716FD97
:1060D80001AA45F82400314600202EF01BFF0134A8
:1060E800EEE7082CEFD1029B0F2BECD8DDF80CE083
:1060F800BEF1070FE7D8049F0D2FE4D8059E06F1DF
:106108006402C82ADFD8069DFF2DDCD807986428CA
:10611800D9D808996429D6D88842D4DA099C032C9E
:10612800D1D8DFF824C0C3EBC3020CEB02030CF890
:1061380002E018715F709E70DD7059719C7108489B
:10614800FFF7EEFEF8E600BFF03300209493030853
:1061580070360020129603087891030817960308F2
:10616800E9930308219603089991030829960308DF
:106178005F96030832960308CC530308B6940308C5
:10618800709703082E9603082DE9F04FDFF818B131
:1061980089B08046894616460D4614460027002ECB
:1061A8006DD00C22214628462EF04AFF94F90B3078
:1061B800049394F90A300393B4F908300293B4F9BC
:1061C80006300193B0FA80FAB4F9043000934FEA2C
:1061D8005A1A3B465A4651464046FFF7B5FA95F9D2
:1061E8000B30049395F90A300393B5F908300293FC
:1061F800B5F906300193B5F9043000935A463B4689
:10620800514640460137FFF7B7FA082F05F10C054C
:1062180004F10C04C3D10024DFF890A0254686B30E
:106228000027012303FA07FB325959F80430534079
:106238003BEA030314BF0123002312EA0B0F079361
:1062480006D000972B46524607994046FFF77CFA3E
:1062580059F804301BEA030F06D000972B46524624
:1062680007994046FFF788FA01370E2FD9D1013533
:10627800082D04F10C04D2D109B0BDE8F08FB24664
:10628800ADE73746012359F80420BB40134206D036
:1062980000972B46524601214046FFF76DFA013719
:1062A8000E2FEFD1E3E700BF349603084C9603089E
:1062B800F0B58BB00546F9F7C5FF002868D0354919
:1062C800002201200BB0BDE8F0405DE72D2903D086
:1062D800A1F13003092B56D8052C04DD0BB0BDE81D
:1062E800F040FDF7E3BF2846FDF708FC0AAB621C47
:1062F80003EB440424F80C0C15F8013F303B092B40
:10630800FAD9144629780029E0D1062CE6D1BDF93E
:106318001C309AB2072AE1D8BDF91E40A4F2EE2239
:1063280092B240F2DC508242D8D8BDF92050A5F292
:10633800EE2292B28242D1D8BDF92260B442CDDCBD
:10634800B542CBDBBDF9247007F1640292B2C82ACA
:10635800C4D8BDF926001128C0DCDFF838C00C22EB
:1063680002FB03C240B29480D58016819772D07226
:10637800CDE90370CDE901560094074A0846FFF7B6
:10638800FBF90BB0F0BD2029A8D101352246B8E7AA
:106398000446B7E770360020349603082DE9F74F16
:1063A800DFF864A081468B4617460E46002447B3A3
:1063B80007EB84080422414630462EF041FEB8F827
:1063C80002300193B0FA80F537F8243000936D0954
:1063D8002346524629464846FFF7B6F97388019383
:1063E8003BF8243000935246234629464846013458
:1063F800FFF7C2F9042C06F10406D8D103B0BDE8B2
:10640800F08F3D46EAE700BF61960308F7B50546F9
:10641800F9F718FF064630B12A490022012003B0D7
:10642800BDE8F040BAE728492846FDF7DDFB38B952
:10643800244B264AC3E90022C3E9022203B0F0BD77
:106448002846FDF75BFB0328044632D82846FAF7AE
:1064580093FC074660B1FDF751FB01260546384617
:10646800FAF78AFC40B903B0BDE8F040FDF71EBF5B
:1064780040F2EE250646F2E7FDF740FB002EF2D08B
:10648800A5F2EE2240F2DC539A42ECD8A0F2EE22BA
:106498009A42E8D80B4B0E4A23F8245003EB8403A6
:1064A80000215880CDE9005023460846FFF764F9DB
:1064B800C4E7084908480323324603B0BDE8F04062
:1064C800FDF77CBE0C20002094930308E803D00756
:1064D8006196030809900308328F03082DE9F04FED
:1064E8002DED088BDFF80C9193B0804692460D464F
:1064F8001446002695ED008AB5EE408AF1EE10FAB2
:1065080070D0D5ED019A95ED029AD5ED038ABAF1CE
:10651800000F3ED094ED000A94ED01BAD4ED02AA22
:1065280094ED03AAB4EE408AF1EE10FA5FD1F4EECE
:106538004B9AF1EE10FA5AD1B4EE6A9AF1EE10FACB
:1065480055D1F4EE4A8AF1EE10FA0CBF0127002764
:106558000FA8FDF7C3FBB0EE4B0A83460CA8FDF766
:10656800BDFBB0EE6A0A059009A8FDF7B7FBB0EECF
:106578004A0A049006A8FDF7B1FB059B049A03900C
:106588000292CDE900B34A46334639464046FFF702
:10659800DBF8B0EE480A0FA8FDF7A0FBB0EE690AD9
:1065A80007460CA8FDF79AFBB0EE490A834609A8EE
:1065B800FDF794FBB0EE680A049006A8FDF78EFB81
:1065C800049B0390CDE901B3009733464A46002166
:1065D80040460136FFF7D0F8082E05F1100504F102
:1065E800100487D113B0BDEC088BBDE8F08F0027ED
:1065F800AEE700BF729603082DE9F0474B4FDFF86E
:106608004881DFF8489104462046F9F71BFE064604
:1066180028B1002246490120BDE8F0475EE705227F
:1066280039462046FDF7A5FA58B9414B00221A60B1
:106638001A611A621A631A641A651A661A67BDE83B
:10664800F087042241462046FDF793FA0546204686
:1066580015BBFAF791FB06460028F0D02DF064FE32
:106668002C465FFA80FA59F8245025B93148BDE81C
:10667800F047FDF7A3BD524629463046FDF779FAA3
:1066880040B920462CF0DCFB29462B482B4CFDF763
:106698001EFEB9E70134E6E7FDF730FA072805469C
:1066A8003BD82046FAF768FB064648B3F9F7BCFE24
:1066B8001F4B03EB051383ED000A01243046FAF75C
:1066C8005BFB064638B1F9F7AFFE194B03EB051330
:1066D80083ED010A01343046FAF74EFB064638B11D
:1066E800F9F7A2FE124B03EB051383ED020A0134FE
:1066F8003046FAF741FB28B9BDE8F047FDF7D6BDAB
:106708000446DBE7F9F790FE094B032C03EB05156C
:1067180085ED030A3FF47DAFEEE7324607230849CB
:106728000848BDE8F047FDF749BD00BF949303084A
:10673800AC6A00207891030817960308E9930308C8
:106748007F950308328F030812960308CC53030879
:106758002DE9F04F834689B092460D46144600262F
:106768004FF019094FF46178BAF1000F45D00A22A9
:10677800214628462EF064FC23890793E388069374
:1067880023790593E3780493A3781D4A19FB0383BF
:106798000393637819FB0383029323780193B0FA78
:1067A80080F7637900937F09334639465846FEF7E8
:1067B800CBFF2B890793EB8806932B790593EB780E
:1067C8000493AB780E4A19FB038303936B7819FB88
:1067D800038302932B7801936B79009339463346F0
:1067E80058460136FEF7C8FF1E2E05F10A0504F1CA
:1067F8000A04B9D109B0BDE8F08F5746D9E700BF00
:1068080086960308F0B58BB00746F9F71BFD0446DA
:1068180030B100225B490120FFF79AFF0BB0F0BDB1
:106828003846FDF76BF91D28054600F3A3800A26B4
:106838004643781C8DF82740FAF79EFA514C0746D4
:1068480050B1FDF75BF9032806D8A31958719DF8D4
:10685800273001338DF827303846FAF78DFA074686
:1068680058B1FDF74BF90D2807D80A236B43E054BC
:106878009DF8273001338DF82730711C0DF1270260
:1068880021443846FDF73DF9FAF776FA074660B134
:10689800FDF734F9222808D80A2303FB0543D870EA
:1068A8009DF8273001338DF827303846FAF764FA17
:1068B800074660B1FDF722F90D2808D80A2303FB23
:1068C800054318719DF8273001338DF827309DF85E
:1068D8002730062B07D0A2190023A3515360138138
:1068E800FDF7E4FC9AE70A2606FB0546002338462E
:1068F800F3803381FAF740FA074638B1FDF7FEF81E
:106908009DF82730F08001338DF827303846FAF7A4
:1069180033FA50B1FDF7F2F80A2303FB0543188157
:106928009DF8273001338DF82730174B4FF0FF3291
:106938001A600A226A43A3184FF4617619890791ED
:10694800D988069119790591D978049198781921EF
:1069580011FB00600390587811FB00610291A25C62
:1069680001925B79009300212B46084A0846FEF7FE
:1069780003FF53E71D23224605490648FDF71EFC81
:106988004CE700BF44370020040E00208696030819
:106998007F950308328F03082DE9F04F2E4EDFF85C
:1069A800C0A087B0814690460D46144602F1200BE0
:1069B80095F9022000232949591891F906109142A6
:1069C80045D00833202BF6D108345C4505F108057D
:1069D800EED107B0BDE8F08F0822214628462EF0F8
:1069E8002FFB627994F9023056F822200492A2799A
:1069F80056F822200392227956F822200292E27851
:106A080056F822200192B0FA80F7228800927F0976
:106A1800524639464846FEF797FE6A7995F902309C
:106A280056F822200492AA7956F8222003922A794D
:106A380056F822200292EA7856F8222001922A88F3
:106A48000092394652464846FEF796FEBCE7B8F132
:106A5800000FC1D14746E0E71C6C0308186C002002
:106A6800AA9603082DE9F04188B00346F9F7EAFB36
:106A7800044630B147490022012008B0BDE8F04182
:106A88008AE7CDE9060018465D1CFDF737F8414B4B
:106A980040B203EBC40696F90220824275D0013455
:106AA800042CF6D1002634462846FAF765F907463D
:106AB80028B1FDF723F80134ADF81800E4B2DFF887
:106AC800D88000253846FAF757F9074600B3FDF78E
:106AD80015F8002258F822108842D3B203D00132A8
:106AE800102AF7D1002358F82320904210D1022D04
:106AF8001AD0032D1DD05A1E012DD2B20FD00B2A49
:106B080003D88DF81B300134E4B20135042DD9D1F6
:106B1800052C14D808B0BDE8F041FDF7C7BB042A1E
:106B2800F3D88DF81C30EEE7052BEED88DF81E3023
:106B3800E9E79A1E0D2AE8D88DF81D30E3E706AB81
:106B480003CB154A71609DF81D10306052F8211072
:106B580004919DF81E109DF91A3052F821100391E6
:106B68009DF81C1052F8211002919DF81B1052F844
:106B7800212001920021BDF8182000920846074AFA
:106B8800FEF7FAFD08B0BDE8F0818DF81A0001247F
:106B98008AE700BFF46B00201C6C0308AA96030860
:106BA8002DE9F04FDFF8DCA087B0814690460D460E
:106BB80014460026B8F1000F61D006222146284667
:106BC8002EF03EFAB0FA80F7207825F095F9834642
:106BD80060797F0925F090F9BBF1000F1DD09BF873
:106BE8000810A27894F803B094F801C04FF4617EBD
:106BF800192313FB02E213FB0BE394F804E000B142
:106C0800007ACDE90223CDE904E0CDE9001C334642
:106C1800524639464846FEF797FD287825F06CF924
:106C28008346687925F068F9BBF1000F1DD09BF801
:106C38000810AA7895F803B095F801C04FF4617E62
:106C4800192313FB02E213FB0BE395F804E000B1F0
:106C5800007ACDE90223CDE904E0CDE9001C3346F2
:106C6800524639464846FEF787FD0136142E05F18F
:106C7800060504F106049DD107B0BDE8F08F47462C
:106C8800CBE700BFC79603082DE9F04186B0074659
:106C9800F9F7D8FA044638B1002253490120FFF722
:106CA8007FFF06B0BDE8F0813846FCF727FF1328C0
:106CB800054600F3918006264643781C8DF8174058
:106CC800FAF75AF8484C074660B1FCF717FFC0B20C
:106CD80025F0F6F830B10378A3559DF81730013345
:106CE8008DF817303846FAF747F8074660B1FCF7D1
:106CF80005FF0D2808D8062303FB054358709DF8A7
:106D0800173001338DF81730B11C0DF117022144EB
:106D18003846FCF7F6FEFAF72FF8074660B1FCF79D
:106D2800EDFE012808D8062303FB054318719DF8DA
:106D3800173001338DF817303846FAF71DF878B157
:106D4800FCF7DCFEC0B225F0BBF848B1062303FB14
:106D5800054302785A719DF8173001338DF81730C2
:106D68009DF81720042A4FF0060327D103FB05439B
:106D780000221A715A711BF0CBFA06236B43E618EE
:106D8800E05C25F0B9F8F278B778192380464FF41B
:106D98006174707913FB074713FB024425F0ACF8C4
:106DA800017A737898F80820039131790F48009791
:106DB800CDE901412946FDF78AFA72E7052A04D18F
:106DC80003FB054300225A71D5E7062AD3D0A2193E
:106DD8000023A3519380CEE7132322460449054894
:106DE800FDF7ECF95DE700BFF01E0020C796030829
:106DF8007F950308328F03080EB400B584B005AB45
:106E0800019053F8042B0649039301A8FDF7E0F815
:106E1800019B00221A7004B05DF804EB03B07047C0
:106E2800C906000810B44C09012250F8243001F0BA
:106E38001F0102FA01F123EA010340F824305DF84A
:106E4800044B704710B44C09012250F8243001F06B
:106E58001F0102FA01F10B4340F824305DF8044B9E
:106E680070474B0901F01F0150F82320012303FA52
:106E780001F1114214BF18460020704770B54488CC
:106E88000546C4F30B042246084600212EF00BF9F0
:106E98002969094A9142034602D3084A914204D318
:106EA80041B11846BDE8704008472246BDE8704029
:106EB8002EF0D5B870BD00BF90D50308A0D6030842
:106EC80038B5064C064DAC4206D2616820461434EB
:106ED800FFF7D4FFAC42F8D338BD00BFE0D00308B9
:106EE80090D5030810B50346F9F7ACF9044628B95C
:106EF800062209491846FCF73CFE58B9FFF7E0FF9F
:106F0800064B00201870064B18701CB1BDE81040E5
:106F1800FDF763B910BD00BF21970308184500208D
:106F2800052700202DE9F04F0F468DB0C2490646CF
:106F3800FCF774FE0546002840F01B82BF49304626
:106F4800FCF76CFE0546002840F01582BC49304627
:106F5800FCF764FE0546002840F00F82B949304628
:106F6800FCF75CFE0546002840F00982B649304629
:106F7800FCF754FE002805460ABF012408243546BC
:106F88000FB144F01004B1492846FCF747FE002829
:106F980000F0F78144F02004F9F746FFFFF790FF6F
:106FA800AB4B002514F0090F1D7000F062822846D3
:106FB800FDF7CAFC14F48073039340F0EC81A548F4
:106FC800FCF790FA04F01803182B40F0E681A24869
:106FD800FCF788FA0123029304F48473082B02D186
:106FE8000020FDF79FFB14F080050BD19B4B1A780E
:106FF800002A9B4A06BF012113460021994A2046D0
:10700800FEF7BAFB2046FEF7CBFB002D40F042828C
:10701800954F964B3E781B78954D964AF01A464206
:1070280005EB83034641D3F8743231462046FEF718
:107038008BFB3B788F4A05EB83053146D5F87432D4
:107048008D4D2046FEF798FBD5ED007A8B4AF5EE7C
:10705800407AF1EE10FA0CBF012100212046FEF71C
:107068008BFB2A468649874D2046FFF737FA864A22
:1070780086492046FFF788F895F90210844AB1FA44
:1070880081F149092046FEF777FB2A4681492046C7
:10709800FEF7D8FE804B1F68804B93F8662002B13C
:1070A8009F6E7F4BDFF8FCA1D3F80090DFF850B259
:1070B80000265AF82650002D40F07281DFF844A2CD
:1070C8002E4669EA070B774B53F82650002D40F0FF
:1070D8008781754F754E6FF07F4300933A6831682A
:1070E800734B2046FEF71AFD40F202230093BA685C
:1070F800B168704B704F2046FEF710FD6F48DFF8FF
:1071080008C201262B5CEA5D0CA919440DF1300E6A
:1071180001F8202C15F80C108E440EF8102C16B11E
:10712800591A4E424E410135082DEBD13146002502
:1071380008AB634A8DF8185020468DF82850FEF7A2
:1071480003FB04AB31465E4ADFF8C0B1DFF8C091FB
:107158002046FEF711FB5B4A5B492046FFF71CFC03
:107168005A4A5B492046FFF71BFD5A4A5A492046AE
:10717800FFF7EEFA594A5A492046FFF70FF9594ADC
:1071880059492046FEF76EFD0126584B5848DFF84E
:10719800E0800222991930442DF052FF1BF8153077
:1071A8004344B0FA80F793F8A12019F81530022B60
:1071B8004FEA571740F0388116F80B304FF0190A8C
:1071C80040F2EE211AFB0313CDE9002339462B4682
:1071D800484A2046FEF7B8FA16F80930454A40F200
:1071E800EE211AFB0313019319F815309844394618
:1071F80098F8A130009320462B46FEF7BDFA0135DA
:10720800122D06F10206C0D1144B3B4E13F8112F74
:10721800002A134A06BF012113460021374A204697
:10722800FEF7AAFA21460020FEF7FBF914F0080F32
:10723800214600F016816DE0E0960308E796030802
:10724800EF960308F59603085F950308FE96030872
:10725800184500200C97030818970308D02E002023
:1072680087CB0308D7950308E4200020D41B00200F
:107278005451030828970308AC6A00203197030883
:10728800BC6C0020F033002070360020383C002011
:1072980040970308C83B0020606D0020300F002095
:1072A800B85B00203854030830370020A43B002086
:1072B800649703086B97030890700308B02F0020A9
:1072C800D18F0308F46B0020946C0020F01E00207E
:1072D8006420002044370020783A00200C20002049
:1072E800FC1F002068390020443A00203F2000207D
:1072F8001B200020EC8F0308FC2E0020CF950308EC
:107308004D97030859970308E82D002040200020D6
:107318001C2000200020FEF701FA21460120FEF77C
:10732800FDF95F4D21460220FEF7F8F933782B70FE
:10733800039B13B95B48FDF705F8FF232B70002763
:10734800F8B221460137FEF7D3F9062FF8D1737842
:107358006B70039B002B7BD15248FCF7C7FF524848
:10736800FCF756F8FF236B70F9F748FD0DB0BDE840
:10737800F08F012404E6022402E6042400E68124B6
:10738800FEE54A492846FCF749FC00283FF404AECC
:1073980044F4807400E602951EE6012302931BE67E
:1073A8002B78DBB14FF0010808FA06F869EA070301
:1073B80013EA080F14BF012100212B465A46204624
:1073C800FEF7C2F967EA090313EA080F5A462B4683
:1073D80014BF012100212046FEF7CEF9013668E6E8
:1073E8002B78FBB14FF0010808FA06F819EA080FE4
:1073F8000BD067EA090313EA080F52462B4614BF5D
:10740800012100212046FEF79FF918EA070F09D04D
:107418001BEA080F2B46524614BF012100212046C3
:10742800FEF7AAF901364EE600922B463946204A65
:107438002046FEF789F919F815301D4A984439464F
:1074480098F8A130009320462B46FEF795F9D6E62A
:10745800FF236B70029B002B86D01648FCF742F87E
:1074680082E73078FEF75AF921467078FEF740F93E
:10747800F0E7A20705D5104B21461878FEF74EF91C
:1074880072E763077FF570AF0B4B21465878FEF71C
:107498002FF969E721461820FEF7C3F8DAE700BF9D
:1074A80000000020E99303082397030807970308BF
:1074B800FC8F030872970308FC2E0020012131E598
:1074C80000212FE52DE9F74F3B4B3C4D1A785B78AF
:1074D8006B7000902A70F9F7A7FCFFF7F1FC384BA6
:1074E800DFF8E0B000241C70A0460D27354B00994A
:1074F8006743DE19D6F800904846FCF75EFB002883
:107508003DD0B8F1000F01D0FBF7D8FF49462E480F
:107518005F44FDF7A5F900213046FEF777F8FBF741
:10752800CDFF3B7903F01803082B3AD0102B3CD041
:107538003046FDF735FF0D2303FB04B3B3F809000C
:10754800F9F733F90746C0B13046F8F783FED7E9B3
:1075580001218246024401443046F8F7B3FE60B97F
:10756800019049461948FDF77BF97968019A514419
:107578003046FDF783FFFBF7A1FF08F1010801344E
:10758800B4F5B37FB1D1F9F739FCFF232B706B70D9
:10759800B8F1000F0DD10E4803B0BDE8F04FFCF76D
:1075A8000DBE0C48FCF7CEFEC2E70A48FCF79EFE6B
:1075B800BEE703B0BDE8F08F5C2900200000002082
:1075C8001845002080580308219503087C97030874
:1075D80078910308E99303082DE9F74F81462CF0C9
:1075E800A3FE054628B1012821D199F800302A2B9D
:1075F8001DD17C48DFF804827B4FFBF773FF002422
:107608004FF00D0909FB048638463168FDF728F963
:10761800291C18BF012130460134FDF7F7FFFBF79D
:107628004DFFB4F5B37FEDD103B0BDE8F08F3D2138
:1076380048462DF04FFD002800F0CF80074617F888
:10764800013C202B07F1FF3232D0A7EB09070130AC
:10765800054601302B78202BFAD0DFF8A0A14FF097
:107668000008D346FFB20D2303FB08A42668304662
:107678002CF05AFE3146024601904846FCF779FA4A
:107688000646002840F09D80019BBB4240F099804F
:10769800237903F06001202951D00BD8F1B1534868
:1076A800FCF78CFD204603B0BDE8F04FFDF778BE2F
:1076B8001746C4E7402958D06029F0D14C4A02EB5C
:1076C800C606002796F878A3B9463B46574502D226
:1076D800B9F1000F35D0002BE1D00EE003F007061A
:1076E800042E284618D12CF015F9D4F80530834219
:1076F8000146D4D32046F9F785F80D2303FB08B8D3
:107708003C48D8F80010FDF7ABF80021204603B03C
:10771800BDE8F04FFDF77ABFFCF7F0F9B4F8055073
:107728000146B4F80700AAB283B21EB1022E1CBFEC
:107738002AB203B29142B2DB9942B0DCDAE7667949
:10774800BCE7D6F8742352F8270060B129460193A4
:10775800FCF74AFA019B30B9394620464FF0010937
:10776800F9F750F84B460137B0E74FF00D0994F898
:1077780005A009FB08B95645BFDA002DBDD02F4634
:1077880001353B78202BFAD02046F9F725F899F8EF
:10779800043003F00703022B05460CD0032B0AD054
:1077A8003846FCF7ABF9A8552C2138462DF092FC49
:1077B8000136451CDFE73846FCF7A0F925F8160026
:1077C800F2E708F10108B8F5B37F7FF44CAF0A4837
:1077D80003B0BDE8F04FFCF7F1BC484603B0BDE884
:1077E800F04F6FE68C97030821950308AA970308C2
:1077F800545103089F970308789103088058030899
:1078080008B5FAF7BFFB0A200EF050FD012008BDAD
:10781800F8B50E4C456862731646027A0F4642F078
:10782800800225212846FFF7EBFF3A462621284605
:10783800FFF7E6FF46F0800227212846FFF7E0FF22
:107848000DF0EEFE206101202073F8BD300F0020FE
:1078580070B50478032C0E46154603D0BDE8704079
:10786800FAF7A2BC4468027A25212046FFF7C8FF30
:10787800324626212046FFF7C3FF2A4663212046C9
:10788800FFF7BEFF812227212046FFF7B9FF01201D
:1078980070BD028822F040021204120C0280038894
:1078A80010B4002991FAA1F4B4FA84F49BB208BF89
:1078B8004FF0FF34013C23F0380343EAC4039BB282
:1078C800038003885DF8044B43F04003038070474E
:1078D800074A00235168814202F11C0204D0013397
:1078E8000C2BF7D100207047581CC0B2704700BF5E
:1078F800B00B002038B504460123002002212C22B9
:107908003E252070A5706170E2702371E371024812
:10791800FFF7DEFF607138BD5800024000F1FF3C00
:107928004FEACC002DE9F043A0EB0C04A400374F3C
:10793800DFF8FCE03E59364DDEF81490DFF8F480AD
:107948003C44AE420CBF01260226656846EA090699
:107958004545CEF8146083B0A16023613ED02D4B1D
:107968009D423DD014339D423CD014339D4232D0C9
:1079780014339D4239D014339D4239D014339D427B
:1079880039D003F562739D423AD014339D4239D001
:1079980014339D4232D014339D4235D01E491F4BBB
:1079A8008D420CBF1D460025A0EB0C0007EB8000A4
:1079B8009209447B85610021012301A88DF80440C8
:1079C8008DF805208DF806108DF8073013F040FC6F
:1079D80003B0BDE8F0834FF40055E5E70225E3E77F
:1079E8002025E1E74FF40075DEE74FF40035DBE7CB
:1079F8004FF40015D8E74FF00075D5E7084DD3E7E9
:107A0800084DD1E7084DCFE7084DCDE7B00B002072
:107A1800000002401C00024058040240000002100E
:107A280000020010020000102000001000200010CA
:107A380000100240080002400138C0EBC000094BAA
:107A48008000F0B4084D1C58084F6E691844BC42B9
:107A58000CBF0123022333436B6101754275F0BCEF
:107A6800704700BFB00B0020001002400000024029
:107A78002DE9F04F544C54F8204083B0002C5FD0CF
:107A8800E56DA1601F469046504B6A6862652360A9
:107A980004F1620204F1E2036261A36180224FF4FF
:107AA8008073C4E903238146287E27F077FDE868C0
:107AB80060B1FFF70DFF09F10102D2B20C21FFF707
:107AC800BBFF636DEA68A26324332365A86898B195
:107AD800FFF7FEFE09F101020646D2B20B21FFF7BD
:107AE800ABFF2346EA7E3A493046FFF717FF636D3E
:107AF800AA68E2632833E36494F86100F9F728FC84
:107B0800064694F86000F9F723FC3A07824695F890
:107B180019B019D5C6B117F0110F4FF00B0309F1C1
:107B28000100F07114BF4E213E21B3715A46304610
:107B3800F9F7D4FCFB0743D5A36B6BB3E36B5BB3DB
:107B4800204603B0BDE8F08F17F0010F0CBF2E27B9
:107B58004E2718F0020F0AD04EB10B2209F101038B
:107B6800B271F37130465A463946F9F7B7FC18F046
:107B7800010FE1D0BAF1000FDED00C2309F10100AA
:107B88008AF807008AF806305A4639465046F9F707
:107B9800A5FCA36B002BD1D12B7FAA7E8DF80420E6
:107BA8009B090021012201A88DF805308DF80610E7
:107BB8008DF8072013F04CFB204603B0BDE8F08F8A
:107BC8003046F9F793FFB7E7E8440020F05503087B
:107BD800290B00080348D0F83C3113B100F59A701E
:107BE80018477047B00B00200348D0F8203113B174
:107BF80000F58C7018477047B00B00200348D0F888
:107C080004310BB1FC301847704700BFB00B00209F
:107C18000348D0F8E8300BB1E0301847704700BF90
:107C2800B00B00200348D0F8CC300BB1C430184753
:107C3800704700BFB00B00200348D0F8B0300BB13C
:107C4800A8301847704700BFB00B00200348D0F891
:107C580094300BB18C301847704700BFB00B002030
:107C68000248836F0BB1703018477047B00B002083
:107C78000248C36D0BB1543018477047B00B002051
:107C88000248036C0BB1383018477047B00B00201E
:107C98000248436A0BB11C3018477047B00B0020EC
:107CA8000248836803B11847704700BFB00B002033
:107CB8002DE9F8430501744C63596119002B00F054
:107CC8009A80724A6719934204BF01230B730646D0
:107CD800387A27F063FC3B7A03F01F015B09012225
:107CE800022B02FA01F200F0A880032B00F0A0801A
:107CF800012B03D1664B996A0A439A6263190136CC
:107D08001879F9F725FBF6B2074610B11223C671A8
:107D1800837163195879F9F71BFB10B11323C671E6
:107D2800837163199879F9F713FB10B11423C6719D
:107D3800837166190E21F2793846F9F7CFFB70790D
:107D4800F9F706FBF2790E21F9F7C8FBB079F9F7D4
:107D5800FFFAF2790E21F9F7C1FB63594D4A9342B4
:107D680070D04A4A934200F083804B4A934274D0C1
:107D78002C44227B002A40D000252E469988474A69
:107D880021F480510904090C958156819980B3F832
:107D980004E0D788B2F808C0B2F80E90B2F81080A4
:107DA800508A94884EF4805EB7F5827FA3F804E089
:107DB80026D0998821F470610904090C4CEA010164
:107DC80099802743198849EA070448EA040401F41A
:107DD800415120430843304345EA00011980998BFB
:107DE800908A21F400621204120C9A8318821A886D
:107DF80042F040021A80BDE8F88301250226BDE75B
:107E080044EA0904198844F4827448EA04040443DF
:107E180001F44150044346EA040028431880998835
:107E280021F470610904090C4CEA01019980D6E734
:107E3800174B19690A431A6160E7154BD9680A4359
:107E4800DA605BE702F56042D16841F48051D160A5
:107E5800D16821F48051D1608AE702F5EA321169CC
:107E680041F400411161116921F4004111617FE77A
:107E780002F5EC32116941F480411161116921F474
:107E88008041116174E700BF1029002000380040CC
:107E98000010024000300140003C0040000000207B
:107EA800F0B44C4C049D00EB800004EB8004606847
:107EB80000285FD0484F4E004FF42041F6B2396693
:107EC8008469240401F1FF314BD44168DFF814C1FF
:107ED80046F4903401EA0C010C434FF4204144600D
:107EE800396602E0B1F1FF3F52D0846914F0020410
:107EF80001F1FF31F6D04FF42041826239660A461B
:107F080002E012F1FF324CD3816911F04001F8D040
:107F180032494468DFF8CCC03A6641EA0342013B83
:107F28001643DBB204EA0C02013316432B444660C5
:107F380082694FF4204112F0040201F1FF3107D1A8
:107F48004C1C36D0826912F0040201F1FF31F7D0DF
:107F5800426A05F8012BAB42EAD14FF420423A6657
:107F68000DE04C1CACD11E4A3966138801339BB214
:107F780013800020F0BC704712F1FF3221D38369CF
:107F880013F02003F8D02023C3613A660120F1E7FB
:107F9800134A3966138801339BB220461380F0BC1C
:107FA80070470F4C3A66238801339BB208462380FA
:107FB800E0E70B4C3966238801339BB210462380D7
:107FC800D8E707493A660A88013292B218460A8009
:107FD800D0E700BF20450020300F00200024000219
:107FE80060240020009800FCF0B50E4601780129B5
:107FF80085B0044653D0022957D11D46836846F000
:10800800800113B118689B880385606840F2E933E2
:10801800868901E0002B57D00689013B16F0020F34
:108028009BB2F7D0017340F2E93301E0002B4BD04B
:108038000189013B11F0010F9BB2F7D0037B606807
:108048004FF0000C83894FF6FF764FF47A734FF0A8
:10805800FF0E03E0013B9BB2B34229D001898F0791
:10806800F8D580F80CE04FF47A7302E0BBB2B34263
:108078001ED00189C90703F1FF37F7D5017BC9B2C3
:108088000AB1117001320CF1010CAC45E6D1A368BC
:10809800C3B11A689B889361012005B0F0BD90F9BF
:1080A8000400411C01D0022805DD002005B0F0BD08
:1080B800F9F78EFEEBE7617900923246FFF7F0FEA2
:1080C80005B0F0BD0120F1E70392F9F781FE039AAC
:1080D800B5E72DE9F0410478032C884617461E467B
:1080E8001FD14468027A252142F080022046FFF71A
:1080F80087FB424626212046FFF782FB46F0800296
:1081080027212046FFF77CFB04200EF0F3FE72B611
:10811800C92133463A462046F9F7C5FE62B6BDE89E
:10812800F081BDE8F0415FE737B500F10C04054682
:1081380000220A212046FFF78BFB0F220A21204646
:10814800FFF786FB01AA032310212046FFF7C1FF92
:108158009DF8043080336B839DF805308033AB8302
:108168009DF806308033EB8300220A212046FFF772
:108178006FFB0DF10302012302212046FFF7A9FF3F
:1081880001230DF1030209212046FFF7A2FF112266
:108198000A212046FFF75CFB012003B030BD2DE922
:1081A800FF47037B0546884600F10C061BB1022BEE
:1081B80003D9032B37D000245AE001230DF107021D
:1081C80002213046FFF785FF0028F4D09DF80730DC
:1081D800D907F0D5072302AA03213046FFF779FF14
:1081E8000446002CE7D09DF80E7011220A21304673
:1081F800FFF72EFB3B07DED4B5F91A1002A8F8F7F3
:108208004CFBA8F80000B5F91C100DF10A00F8F7AE
:1082180044FBA8F80200B5F91E1003A8F8F73DFBC7
:10822800A8F8040024E0264F4FF0020A0024B946BB
:1082380097F86C30012B1FD00FD3022BD1D1F8F750
:108248002FFC81460028B6D102A905F11000F9F7E4
:1082580082FE87F86C900446C3E73B7B23B9012272
:1082680002213046FFF7D4FA012389F86C30002444
:10827800204604B0BDE8F087F8F712FC00289AD130
:1082880002A905F11000F9F766FE9DF808300446CA
:1082980008B1DA0708D40023BAF1010F89F86C3065
:1082A80089D04FF0010AC3E73B7B23B9072203219A
:1082B8003046FFF7ADFA022389F86C300024D7E77F
:1082C800300F00201FB54B4C237C012B5BD0022BB9
:1082D8005DD1A36913B11A689B881385F52160697C
:1082E800F9F7C3FD01230DF10F0200216069F9F7C9
:1082F8008BFDA36913B11A689B8893619DF80F10D1
:108308003D48FBF7E4FF237C012B4ED0022B50D1D4
:10831800A36913B11A689B8813859A216069F9F7D4
:10832800A4FD01230DF10F0200216069F9F76CFD2E
:10833800A36913B11A689B8893619DF80F102F48A1
:10834800FBF7C5FF237C012B41D0022B43D1A36946
:1083580013B11A689B8813859B216069F9F785FD1D
:1083680001230DF10F0200216069F9F74DFDA369A2
:1083780013B11A689B8893619DF80F102048FBF78A
:10838800A6FF04B010BD94F91400421C01D10021CD
:10839800B6E70228FBDC0DF10F020092617D752221
:1083A800FFF77EFD0028A9D1F1E794F91400411CDC
:1083B80001D10021C3E70228FBDC0DF10F02009276
:1083C800617D1A22FFF76CFD0028B6D1F1E794F918
:1083D8001400421C01D10021D0E70228FBDC0DF17A
:1083E8000F020092617D1B22FFF75AFD0028C3D1BE
:1083F800F1E700BFF0540020B8970308CB970308B3
:10840800DE970308F0B5037C012B85B004464DD0F8
:10841800022B51D1836913B11A689B88138560694F
:1084280040F2E933828901E0002B74D00289013BD4
:1084380012F0020F9BB2F7D0C323037340F2E93363
:1084480001E0002B67D00289013B12F0010F9BB2BB
:10845800F7D0037B60698389038999074FF0050783
:1084680002AE4FF47A724FF0FF0C4FF6FF7506D448
:10847800531E9BB21AB31A4603899907F8D580F898
:108488000CC04FF47A7302E08BB2AB4217D002896A
:10849800D20703F1FF31F7D5027BD2B20EB13270A9
:1084A80001367A1E6FB117461A46E5E790F91400AF
:1084B800431C01D0022824DD002005B0F0BDF9F7E7
:1084C80087FCA36913B11A689B8893619DF80C0017
:1084D8009DF808609DF809109DF80A509DF80B203A
:1084E8009DF80D3041EA062143EA002342EA0522BD
:1084F8000120A4F85010A4F85220A4F8543005B074
:10850800F0BD02AB617D009343220623FFF7C8FC50
:108518000028DBD1D0E7F9F75BFC9BE7F0B5037BDC
:10852800012B85B004464DD0022B51D1436913B1BC
:108538001A689B881385206940F2E933828901E033
:10854800002B71D00289013B12F0020F9BB2F7D0C9
:10855800BB23037340F2E93301E0002B64D00289A6
:10856800013B12F0010F9BB2F7D0037B206983898E
:10857800038999074FF0050702AE4FF47A724FF05E
:10858800FF0C4FF6FF7506D4531E9BB21AB31A465A
:1085980003899907F8D580F80CC04FF47A7302E084
:1085A8008BB2AB4217D00289D20703F1FF31F7D55E
:1085B800027BD2B20EB1327001367A1E6FB1174605
:1085C8001A46E5E790F91000431C01D0022821DD86
:1085D800002005B0F0BDF9F7FBFB636913B11A6819
:1085E8009B8893619DF80C009DF808609DF8091020
:1085F8009DF80A509DF80B209DF80D3041EA0621A0
:1086080043EA002342EA052201206183A283E3832F
:1086180005B0F0BD02AB617C00933B220623FFF757
:108628003FFC0028DED1D3E7F9F7D2FB9EE71749D4
:10863800174B184A184810B4D1F8884044F470040D
:10864800C1F888401C6844F001041C605C68224042
:108658005A601A6822F0847222F480321A601A680A
:1086680022F480221A605A6822F4FE025A60DA6AFA
:1086780022F00F02DA621A6B002410404FF00062F9
:1086880018639C608A605DF8044B704700ED00E059
:10869800001002400CC07FF8CCFC00FF90F860305E
:1086A80043B942690121072082F84430A2F8460004
:1086B80082F84810704700BF0120704700207047BB
:1086C800027A407A02FB00F07047037913F0020344
:1086D80008D00369D0E90920013B101A1840C0B23C
:1086E800181A704718467047017170477047037928
:1086F8009B070AD5436A8269D154436A01690133E9
:10870800B3FBF1F201FB123343627047037913F0B4
:10871800010306D0D0E90732C0689B1A0138184017
:1087280070471846704710B5037913F001030146E6
:108738000ED0FFF7EBFF50B10B6A4A69CC68D05CEA
:108748000133B3FBF4F204FB1233C0B20B6210BD69
:108758001846FCE790F84B3830B53BB990F8491803
:1087680090F84A380124DAB2914200D830BDB0F806
:10877800525804FA03F22A43A0F852280133F2E7C8
:10878800D0E90920131A584258417047F0B5564CA1
:108798002378002B38D06378002B35D1A17AE57A7D
:1087A800C1F1FF0189B200292FD125716571A57129
:1087B80023796279A179A589E68901280BBF12027C
:1087C8001B0242EA034343EA02430B434749172289
:1087D800012707FA02F0184214BF3046284612F162
:1087E800FF3201F8010FF4D201236370A36A182243
:1087F8005A60E26A00215162118841F0010111803A
:108808001A6842F001021A60F0BDC1F1FF036B4320
:108818003C212289B2FBF1F61B120F46052EC7D860
:10882800DFE806F0030E1F2F4251D9B2EB1A5A4364
:108838003C23B2FBF3F20A4425716271A171B7E7D8
:10884800B2FBF7F107FB112291B2DEB2C1F13C0293
:10885800E91A5143B1FBF7F1314421716571A671F1
:10886800A6E73C27B2FBF7F107FB1122DEB292B272
:10887800EB1A5343B3FBF7F3334426716571A371C5
:1088880096E7B2FBF7F607FB162292B25FFA83FC73
:10889800C2F13C02E91A5143B1FBF7F1614484F893
:1088A80004C06171A57183E7B2FBF7F107FB1121E1
:1088B800DEB289B2EB1A5943B1FBF7F131442171A9
:1088C8006671A57174E73C27B2FBF7F107FB11222B
:1088D80092B2DEB2BA1AEB1A5343B3FBF7F333443E
:1088E80025716671A37163E7001000200F10002046
:1088F800064A074B1068074A9860002193F836002B
:1089080083F83010FF23137040E700BFB06A0308F4
:10891800001000202C000020034B5A780AB90122CD
:108928005A700020704700BF2C000020144B154AD5
:1089380093F8401001B314490978D1B91349D160AB
:10894800134A144912685964117983F84810D16898
:10895800D96411491965517983F8541011699965D9
:108968000E49D9659179D26983F860105A6600205A
:1089780070470B49D160E3E70A49D160E0E700BFDF
:10898800001000202C000020EA2A0020E86A0308D2
:10899800AC290020E22A0020E32A0020E62A002051
:1089A800746B0308E46B0308034BB3F86820034BAC
:1089B8004FF0FF301A80704700100020E82A00208E
:1089C800034B1A88034B0020A3F86820704700BFA8
:1089D800E82A002000100020074B93F90030012BF3
:1089E80006D0064BB3F86C20A3F86A200020704725
:1089F8004FF0FF30704700BFA00B00200010002090
:108A080008B5064B1A782AB1054A1278012A1CBF04
:108A180000221A70FFF78AFF002008BDEA2A00200A
:108A2800E02A0020064B93F90020064B12B91A7071
:108A3800002070471A78002AFAD10122F7E700BF10
:108A4800A00B0020E62A0020104B114A93F86E1064
:108A5800517293F86F109172B3F87010118093F8F7
:108A6800772083F87420B3F87C20A3F87820B3F833
:108A78007E20A3F87A20B3F88420A3F88020B3F8E6
:108A88008620A3F882200020704700BF0010002035
:108A98001C280020104A114B517A83F86E10917AE5
:108AA8001288A3F8702093F8742083F87720B3F81D
:108AB8007820A3F87C20B3F87A20A3F87E20B3F8B6
:108AC8008020A3F88420B3F8822083F86F10A3F8DD
:108AD80086200020704700BF1C28002000100020BE
:108AE8000020704700207047084A0949B2F88830CA
:108AF8004B8292F88A3092F88B2003EB83035B0059
:108B08000B82044B00209A70704700BF00100020B1
:108B1800A85D00205C290020084A094B518AA3F867
:108B28008810128A0A21B2FBF1F283F88A20054ADA
:108B3800927883F88B200020704700BFA85D002042
:108B4800001000205C29002030B1007910F1FF30BE
:108B580018BF4FF0FF3070474FF0FF307047144A8E
:108B6800144B528802F0010283F88C2093F83720C6
:108B780083F88D2093F8382083F88E2093F83920D5
:108B880083F88F205A8FA3F8902093F83C2083F81D
:108B9800922093F83D2083F8932093F8342083F8AB
:108BA800942093F83E2083F895200020704700BF5A
:108BB800B85B0020001000200A4B0B4A1B68B2F873
:108BC80096105980B2F89810A3F84C10B2F89A1081
:108BD8009980B2F89C10B2F89E20D9801A800020A3
:108BE800704700BF58290020001000200D4B93F853
:108BF800A020762101FB02320020B2F8A610A3F8CB
:108C08009610B2F8F010A3F89810B2F8A810A3F8CC
:108C18009A10B2F8AA10B2F8A420A3F89C10A3F8EE
:108C28009E207047001000200A4A0B4BB2F806122B
:108C3800D980B2F808121981B2F80A125981B2F82B
:108C48000C129981B2F80E12B2F81022D9811A8248
:108C58000020704700100020805B00200A4A0B4B60
:108C6800D188A3F806121189A3F808125189A3F82C
:108C78000A129189A3F80C12D189128AA3F80E124C
:108C8800A3F8102200207047805B0020001000200D
:108C9800184B194993F8122230324A7493F8A020DD
:108CA800762101FB0232002092F8EB1083F81312B0
:108CB80092F8BE1083F8141292F8BF1083F81512B8
:108CC80092F8C01083F81612B2F8D810A3F8181248
:108CD800B2F8D610A3F81A1292F8F31083F81C12FF
:108CE80092F8171192F8182183F81D1283F81E22A2
:108CF800704700BF001000202C0000200F4B1049C7
:108D080093F8122230320A7593F81F2230328A758E
:108D180093F8D8221A2101FB023202F50F7103F5EC
:108D2800087302F5157251F8040B43F8040B9142CD
:108D3800F9D10A881A800020704700BF001000206F
:108D48002C0000200A4A92F8D8321A2101FB03238A
:108D580003F50F7302F5087102F50E7251F8040B52
:108D680043F8040B9142F9D10A881A800020704711
:108D78000010002010B5124A124992F8123292F8E7
:108D8800A00030334B7402F1A401762300FB0313D7
:108D980002F2D921002002F2E2221C7A0C705C7ADD
:108DA8004C709C7A8C709C8922F810400130032802
:108DB80003F1060301F10301EFD1002010BD00BF4C
:108DC800001000202C0000200749084B0A7883F87F
:108DD800A020013283F812224A7883F8D82201327F
:108DE80083F81F22002070475C2900200010002013
:108DF8000A4930B50A4C002201F53A70135DA3F117
:108E08006105052D9CBF203BDBB283540132072A44
:108E1800F4D1002081F8EF0230BD00BF001000201F
:108E28007D900308084B93F8F022012A074A06D8D8
:108E380093F8F112881E012888BF03219170B3F8B6
:108E4800F232138000207047001000203C2A0020D6
:108E580010B5044623790E2B00D110BD032B04D185
:108E6800D4F809309868FFF7F3FF0E34F2E70B499E
:108E7800D1F8F4329A68134618790E280CD19B1A47
:108E88005A10074B5343013B91F8FD2293FBF2F331
:108E9800013381F8FC3270470E33EDE700100020F3
:108EA800B76DDBB60C4BD3F80023824210DA0B4ABD
:108EB8009278022A0AD0032A0CD1D3F804331B690A
:108EC80023B19842B4BF01200220704701207047A7
:108ED8000020704702207047001000203C2A002024
:108EE800054B30B11A69186001321A6105221A75EA
:108EF800704704221A757047442A0020194BB3F8AA
:108F08001023D3F80803D3F80C1310B40132B3F9C3
:108F1800124392B201300131A242C3F80803C3F8E8
:108F28000C13A3F810230FDAB3F81623B3F91813A8
:108F38005DF8044B013292B28A42A3F81623A4BF0B
:108F48000022A3F816237047B3F814235DF8044BE6
:108F580000210132A3F81423A3F81013A3F8161361
:108F6800704700BF0010002030B44FF498714FF0E4
:108F78009615114C114B016040F29E71104AC0F8D1
:108F8800065044614FF4E17503240183C0F81A3098
:108F980008210023C58380F8204080F82110C0F8FC
:108FA80022200371C0F80A30C0F80E30438280F8DE
:108FB800263030BC704700BF020100017D009600DA
:108FC8007800960000230322027183700380C37027
:108FD80043718371C37103724372704700230A227D
:108FE8000360436083608381028070472DE9F84302
:108FF800784C94F8232394F824339A4200F088801C
:1090080094F8232394F82333C2EBC20204EB8202C0
:10901800C3EBC30304EB830392F8471393F82C6361
:109028008B1E9E422FD06C4AB4F880331278D4F845
:10903800281301339BB21C2AA4F880336CD0002576
:1090480094F82333654A0133A2FB0302520802EB6A
:1090580042029B1ADBB284F8233300293DD00CF07E
:10906800DFFAD4F8B433C01AB0F5FA7F04DB002372
:1090780045F0040584F8B233D4F8AC33002B34D16E
:109088002846BDE8F88394F8233304F54B77C3EBFF
:10909800C30307EB830361B11944002213F8015B92
:1090A8002A44994292B2F9D1D3B203EB1222FF2A91
:1090B8003AD0494AB4F880331278D4F828130133E7
:1090C8009BB21C2AA4F88033B9D1454BB4F880234D
:1090D8005A8004229A800025B2E794F8B233002B14
:1090E800BDD1D4F8AC33002BCAD03E4A1268D31A8B
:1090F800B3F5FA7FC4D994F88233032B04BF002355
:10910800A4F8A8330023C4F8AC332846BDE8F88394
:10911800D4F828130025A0E7314BB4F880235A80EF
:1091280003229A8000258BE794F8233301221C211F
:1091380001FB0323FA18FD5C6DB3012D16D1082E2F
:109148003FD0254AB4F880331278D4F82813013375
:109158009BB21C2AA4F880337FF471AF204BB4F87B
:1091680080235A8006229A80002569E71A4AB4F8B3
:1091780080331278D4F8281301339BB21C2AA4F840
:1091880080337FF45CAF164BB4F880235A800522F5
:109198009A80002554E7192ED4F8281324D00E4AB3
:1091A800B4F88033127801339BB21C2AA4F88033B8
:1091B8007FF446AF0A4BB4F880235A8006229A807F
:1091C8003EE794F8B033002B40F0EB801D46D4F80E
:1091D800281335E70010002070270020ABAAAAAAA0
:1091E80074270020A44E002092F802C05578036925
:1091F80092F8038092F804909679D77992F808E06B
:109208000CF0070C45EA0C2508F03F0892F80AC054
:109218001D8095784FEA481848EAD508957BA3F849
:10922800028092F803804FEA890040EA981092F889
:10923800058008F0010840EA8820988006F00F06AB
:10924800507992F80780F60146EA5000567AD8809D
:109258004FEA4E0E4EEAD81E06F0030692F8068034
:10926800D07A07F07F074EEA462E3F01567BA3F8D7
:109278000AE047EA18171F8106F00707967A92F85E
:1092880009E0C00040EA5610167B0CF01F0C46EAB5
:10929800072605F03F05577BD8816D014FEA8C1CE6
:1092A80045EAD7004CEA9E0CA3F80CC01E825882EF
:1092B800D07B92F80EE0D77C92F8128092F811C019
:1092C800967C557D800040EA9E1092F810E07F0061
:1092D8000EF0010E47EAD8170CF00F0C92F8108028
:1092E80040EA8E204FEACC1C92F814E098824CEAAF
:1092F800580C907DA3F816C006F07F0692F811C0AE
:109308000EF0030E47EA4E27360146EA1C165F8325
:1093180092F814C0577D1E8305F01F05AD01C000EB
:1093280045EA9C0540EA5710D8839D83D57D40F2D5
:10933800147015F0010F14BF0646AD2615F0020F84
:1093480008BFAD201E8458842B075FD415F0040F86
:109358000CBF0125092594F88233032B1CD1137EF9
:1093680094F883032E4ED4F8A423C3EB8323A6FBDF
:10937800036304EB40065B09B6F88473A6F88433EC
:10938800DB1B1344013000F00F02180984F8832313
:10939800C4F8A433A4F8A803224B1B68C4F8AC3360
:1093A8004EE65378102B15D020D8DBB994F8B1339A
:1093B800D4F82813002B7FF442AE94F8B333012B72
:1093C80026D919B10A78303A012A21D9002584F81A
:1093D800B35335E694F8B1330BB984F8B15301238C
:1093E80084F8B233D4F82813002529E6303B012B42
:1093F800F8D852F8010F0C49C4F81C0393799088E7
:1094080088808B71C4F82813002519E60325A2E784
:109418000133012284F8B33384F8B22300250FE620
:109428001F85EB51A44E00201C13002010B50446E4
:109438000CF0F6F8544B002283F8B82393F8B923BC
:10944800012A19D9D3F8BC2340F6AC51821A8A42B2
:1094580012DD4E49B3F880230978013292B21C29F3
:10946800A3F8802305D14A4AB3F88013518001211B
:109478009180002283F8B923E2B27E2A29D093F89A
:10948800B91329B393F8B9131B295CD893F8C813F7
:10949800002972D0002182F0200283F8C81393F8C3
:1094A800B913022903D1012A08BF83F8C02393F80E
:1094B800241393F8B94393F8B903C1EBC10103EB43
:1094C800810121440130C0B281F82B2383F8B9030C
:1094D80010BD93F8B923012A2FD993F824232D49D5
:1094E80093F823430132A1FB02C1490801EB410172
:1094F800521AD2B294420CD093F8B94393F8241379
:1095080083F82423C1EBC10103EB8101621E81F8BA
:10951800472393F8C0233AB10121002283F8B813F6
:1095280083F8C023C3F8B403184A12781C2A1ED043
:109538000022C3F8C40383F8C823012283F8B9239F
:10954800C3F8BC0310BD002283F8B9230F49B3F850
:1095580080230978013292B21C29A3F88023B7D15D
:109568000B4AB3F8803353800223938010BDD3F89D
:10957800C4230749821A0A80DAE77D2A8FD101229B
:1095880083F8C82310BD00BF0010002070270020FA
:1095980074270020ABAAAAAA034B03EB4101B1F838
:1095A800CC03C008704700BF001000201D4B93F883
:1095B800F0239AB370B493F8F143B3F8F25303EB82
:1095C8004401002091F8F76391F8F82383F8F00339
:1095D80042EA0622954202D0002070BC704793F8F8
:1095E800F533032B03D0812B1AD0012BF5D10120A1
:1095F800122C2546A8BF1225002CEED00A4B03EBEF
:109608004505A3F12801DC781A79023342EA0422DD
:109618009D4221F8022BF6D170BC7047002070479C
:109628000320E5E700100020F413002038B50446B5
:109638000BF0F6FF444AD2F83C34C31AB3F57A6FFC
:1096480016D892F84034C2F83C04B3B1022B1FD0AC
:10965800442B92F8F11375D901330231DBB249007A
:109668008B4282F840341BDB01318B4263D038BD1A
:109678000023C2F83C0482F84034A82CF7D1002318
:1096880082F8F033A2F8F23392F8F113204603E09F
:10969800E0B282F8F1030146D51885F8F403DBE758
:1096A800B2F8F233E4B283EA042424B2002CB8BF3F
:1096B80041F22101A3B2B4BF81EA43035B009BB22C
:1096C8001C0446BF41F2210181EA43035B009BB2BF
:1096D800180446BF41F2210181EA43035B009BB2B3
:1096E800190446BF41F2210181EA43035B009BB2A2
:1096F8001D0446BF41F2210181EA43035B009BB28E
:109708001C0446BF41F2210181EA43035B009BB27E
:10971800180446BF41F2210181EA43035B009BB272
:10972800190446BF41F2210181EA43035B009BB261
:10973800A2F8F23338BD0021012382F8401482F8E0
:10974800F03338BDE0B2A7E70010002078B310B5B9
:1097580082B040F25514AA2200238DF80210ADF809
:1097680000408DF803208DF80430694655220DF12C
:1097780003045340082213F0800F4FEA430318BF35
:1097880083F03103013ADBB2F5D1A14202D011F8DE
:10979800012FEEE702688DF80330536AAA228DF88C
:1097A8000420694605221BB1984702B010BD7047D6
:1097B800F7F7C6FBF9E700BFF8B5134D95F859243C
:1097C8000AB90120F8BD114B1C6823685E6A46B1CE
:1097D800204605F24441B047002385F8593401205A
:1097E800F8BD05F24447BE1800E023689B68204690
:1097F80098470028F9D0236817F8011B1B682046F2
:109808009847B742F1D1E7E700100020A02E0020CA
:1098180003788B4210D9094B03EB810193F88C3400
:10982800D1F85C041BB900F5777080B27047400826
:1098380000F5777080B27047002070470010002054
:10984800F8B50BF0EDFECC4B93F88D24002A00F010
:10985800938093F89C5493F89D2493F89E1493F85E
:109868009F44120442EA0562224342EA012202F0BE
:10987800F0220021B2F1E02F83F88D1400F00A8164
:109888001025D3F8AC2493F89244117893F8A824BF
:1098980093F8B07493F8B164144104F00F04002FE6
:1098A8007DD1A1420DD90B2C0BD893F892C493F813
:1098B800937403EB840406EA0C0C07EB0C27C4F83A
:1098C8005C7493F89444144104F00F04A1420DD938
:1098D8000B2C0BD893F894C493F8957403EB840479
:1098E80006EA0C0C07EB0C27C4F85C7493F8964452
:1098F800144104F00F04A14200F2E58093F8984463
:10990800144104F00F04A14202D90B2C40F2FD804F
:1099180093F89A44144104F00F04A14202D90B2C85
:1099280040F200810D2D14DD93F89C44144104F09D
:109938000F04A14202D90B2C40F21181102D08D13D
:1099480093F89E4444FA02F202F00F02914200F2A8
:10995800CD8093F8A024002A00F0C58093F89224C3
:10996800120600F1C08093F85914C3F8A404052422
:10997800012231B91046F8BD042493F8591400297E
:10998800F8D0D3F8A4140029F4D0411AB1F57A7F9D
:10999800F0DB00212246C3F8A4141046F8BDA1420A
:1099A8000FD90B2C0DD8A7420BD093F892E493F85B
:1099B80093C403EB840406EA0E0E0CEB0E2CC4F8D9
:1099C8005CC493F89444144104F00F04A1420FD9E5
:1099D8000B2C0DD8A7420BD093F894E493F895C4B8
:1099E80003EB840406EA0E0E0CEB0E2CC4F85CC4E0
:1099F80093F89644144104F00F04A14252D893F806
:109A08009844144104F00F04A1420FD90B2C0DD82F
:109A1800A7420BD093F898E493F899C403EB840415
:109A280006EA0E0E0CEB0E2CC4F85CC493F89A44AC
:109A3800144104F00F04A14201D90B2C7FD90D2D3C
:109A480087DD93F89C44144104F00F04A1420FD918
:109A58000B2C0DD8A7420BD093F89CE493F89DC427
:109A680003EB840406EA0E0E0CEB0E2CC4F85CC45F
:109A7800102D7FF46EAF93F89E4444FA02F202F080
:109A88000F0291427FF665AF0B2A3FF662AF97420D
:109A98002FD15EE793F8922412F0800F14BF10259F
:109AA8000C25EEE60B2CAAD8A742A8D093F896E48A
:109AB80093F897C403EB840406EA0E0E0CEB0E2C05
:109AC800C4F85CC49BE70B2C3FF618AF93F896C418
:109AD80093F8977403EB840406EA0C0C07EB0C2745
:109AE800C4F85C740AE70524012246E70B2A3FF60E
:109AF80030AF93F89E4493F89F1403EB82022640FC
:109B080001EB0621C2F85C1423E793F898C493F894
:109B1800997403EB840406EA0C0C07EB0C27C4F8D1
:109B28005C74F5E693F89AC493F89B7403EB840489
:109B380006EA0C0C07EB0C27C4F85C74F2E6A742A3
:109B48003FF47DAF93F89AE493F89BC403EB840445
:109B580006EA0E0E0CEB0E2CC4F85CC46FE793F803
:109B68009CC493F89D7403EB840406EA0C0C07EB81
:109B78000C27C4F85C74E1E600100020344B5B68E5
:109B8800C3F3080370B4CBB9EFF31183B3B9314A07
:109B9800314E324D1368AC6811688B42FAD1316886
:109BA8008C42F7D82E4A15684FF47A7101FB05F2FA
:109BB800141BB4FBF5F401FB034321E0EFF311811F
:109BC800102383F3128803F1E023C9B29D681A6851
:109BD80012F4803F234A1EBF012414609D681D4B68
:109BE8001E68136881F311881D4A14684FF47A714E
:109BF800334401FB04F2521BB2FBF4F201FB0323D2
:109C0800194AD2F8B414C2F8B4345B1A41F2883154
:109C18008B420AD9C0B2012382F8900482F8B83482
:109C2800002382F88D3470BC704792F8B8340F2B3B
:109C3800F9D8D1180133DBB2C0B2102B81F89004E7
:109C480082F8B834ECD1012382F88D3470BC7047A7
:109C580000ED00E0A44E00203C53002010E000E09E
:109C6800385300203453002000100020036933F8D3
:109C7800110000EB8000C01000F55C7080B27047E6
:109C8800436993F82120002A00F0AF80F0B5594AC3
:109C980093F802E01278DC7D5F78DD7893F806C0EF
:109CA800DE791B2A04BF544A148002690EF00700AB
:109CB80047EA0027002183F82110187A19791780BC
:109CC80005F03F059F7893F805E06D0145EAD70553
:109CD8009F7A5580DD78890041EA95110EF0010ED2
:109CE80041EA8E219D7B91800CF00F0C59794FEA47
:109CF800CC1C4CEA5101D18006F07F06997993F883
:109D080007C0360146EA1116597A1681400040EA22
:109D1800DC1001F0030140EA41205E7BD97A5081D2
:109D280007F01F07587ABF0147EA900090819F7A91
:109D3800187B93F80EC006F0070640EA062005F0E7
:109D48003F055E7B1082C90041EA57116D01D18140
:109D580045EAD6015182D97B5F7CDD7C9E7C587DAB
:109D6800890041EA9C1193F810C00CF0010C41EAFB
:109D78008C2107F00F0793F812C09182197C6D00AF
:109D8800FF0147EA510145EADC1C5F7C1D7DD18259
:109D980006F07F06360146EA171605F00305997D99
:109DA8001F7D16834CEA45255E7D558340F214736A
:109DB80014F0010F14BF1D46AD2500F01F0014F06C
:109DC800020F08BFAD238001C90040EA970041EAAD
:109DD8005611538423079083D183158407D414F034
:109DE800040F0CBF01200920F0BD10467047032066
:109DF800F0BD00BF70270020742700203B4B5B6834
:109E0800C3F30803F0B42BBBEFF3118313BB384A39
:109E1800384F394E1368B5681468A342FAD13C68C4
:109E2800A542F7D8354A16684FF47A7404FB06F24F
:109E3800551BCA69B5FBF6F504FB03539A1A40F69D
:109E4800AC54A2422EDC91F8204074B3182C38D9B7
:109E5800F0BC7047EFF31184102383F3128803F1E9
:109E6800E023E4B29E681A6812F4803F244A1EBFB9
:109E7800012515609E681E4B1F68136884F31188BE
:109E88001E4A15684FF47A7404FB05F23B44921B92
:109E9800B2FBF5F204FB0323CA6940F6AC549A1AE4
:109EA800A242D0DD002281F820200F28D0D1012243
:109EB800CB61087081F82020002381F82130F0BCA4
:109EC8007047631CDBB2192B81F820300855F3D199
:109ED8000C4B1B781B2B08BF0B4B4FF0010081F874
:109EE800210008BF9A80F0BC704700BF00ED00E079
:109EF800A44E00203C53002010E000E0385300201E
:109F08003453002070270020742700200A4BDFED0F
:109F18000B6ADFED0B7A03EB8101D1F8BC3407EE55
:109F2800103AB8EE477AE7EE267AFCEEE77A17EEB3
:109F3800903A98B2704700BF0010002001F11F3F0F
:109F480000405C44714A92F8FC3433B192F802350F
:109F58000021162B82F8FC1401D00020704792F8DB
:109F68000135022BF0B440F2CE8002F5A06018440F
:109F780002F20251D32311F8014F634013F0800F0E
:109F88004FEA430318BF83F0D503DBB213F0800F09
:109F98004FEA430318BF83F0D503DBB213F0800FF9
:109FA8004FEA430318BF83F0D503DBB213F0800FE9
:109FB8004FEA430318BF83F0D503DBB213F0800FD9
:109FC8004FEA430318BF83F0D503DBB213F0800FC9
:109FD8004FEA430318BF83F0D503DBB213F0800FB9
:109FE8004FEA430318BF83F0D503DBB213F0800FA9
:109FF8004FEA430318BF83F0D5038842DBB2BAD1D6
:10A0080092F81915994202D00020F0BC704792F8D6
:10A01800080592F8076592F80C1592F8103592F831
:10A02800144592F80455B2F804C5D2F8047500F046
:10A038000F00C00140EA560001F01F0192F80B65BD
:10A04800C2F8C804890141EA960103F03F0392F877
:10A058000F6592F81305C2F8D4145B0143EAD603DE
:10A0680092F80315C2F8E03404F07F04B2F808351A
:10A07800D2F80865240105F0070544EA101041EA02
:10A088000521C3F30A13C2F8EC04B2F80C55C2F860
:10A09800BC14B2F80E45D2F81005B2F81215C2F881
:10A0A800CC34D2F81435C0F38A10C1F34A01C3F393
:10A0B800CA13CCF3CA0CC7F38A37C6F3CA366D097C
:10A0C800C4F30A04C2F8E404C2F8E814C2F8C0C42D
:10A0D800C2F8C474C2F8D064C2F8D854C2F8DC44D8
:10A0E800C2F8F03492F8183592F81705B2F8161538
:10A0F800DB0043EA5013C1F38A01C2F8F834C2F80E
:10A10800F414012081E7D3237AE700BF0010002070
:10A11800F8B5624B624C1D68E907064615D594F8F8
:10A12800403594F841259A4239D1D4F84435B342A0
:10A138009CBF002384F84C35D4F88405301A0028D5
:10A1480020DD012084F88805F8BD15F4005564D198
:10A15800D4F8703504F5AD609847C20719D5514A4F
:10A1680094F88233C0F3400110F00A0F117600F022
:10A17800040125D0052B33D00029D6D0012384F83B
:10A188008035D2E794F888050028DDD194F8800559
:10A19800F8BD4307C9D5012384F88035C5E7D4F84D
:10A1A8004805404A84F84135304400210123C4F869
:10A1B80044050120117684F84C3584F88805C3E7F6
:10A1C800D4F84825052B3244C4F844255DD000292D
:10A1D80060D10123012084F84C3584F88805B3E761
:10A1E8002B46AC4694F88323D4F8A40304EB420727
:10A1F8000132B7F884E3A7F884C3A3EB0E03034442
:10A2080002F00F02180984F88323C4F8A433A4F8D1
:10A21800A803A1BB002DDCD187E7B4F8503513BBE8
:10A22800B4F85235FBB9B4F85435E3B9B4F8563537
:10A23800CBB9B4F85835B3B9B4F85A359BB9B4F8B2
:10A248005C3583B9B4F85E356BB9B4F8603553B989
:10A25800B4F862353BB9B4F8643523B9B4F8663557
:10A26800002B3FF462AFD4F848350E493344002040
:10A278000122C4F84435087684F84C255CE70123AC
:10A2880084F88035002DA4D14FE740F2FF339C4677
:10A298000125A7E7012384F880359AE7B85B0020F9
:10A2A800001000202C00002000207047002070477C
:10A2B80001207047024B03EB8101B1F88C05704710
:10A2C8000010002030B40246002305251E2400E0BB
:10A2D8000232032BD4BF0021012100F813100133EF
:10A2E800042B04D0122B5470F2D130BC7047557037
:10A2F800EEE700BF024B036043608360C3607047B2
:10A30800E803D007024B03EB4101B1F85005704751
:10A3180000100020024B03EB4101B1F850057047D3
:10A3280000100020DD4B93F8C4250AB900207047BF
:10A338002DE9F04F93F8C62593F8C5450021012A69
:10A348008BB083F8C41500F0EF8093F8CC55023D2C
:10A3580015F0FF0500F09D8103F2CC5005444FF63F
:10A36800FF7210F8011B521AA84292B2F9D1110AD1
:10A378001C4494F8CB05884240F0878194F8CA15AC
:10A38800D2B2914240F0818193F8EC25202A40F026
:10A398007C8193F8C705821C0192821D029200F10C
:10A3A8000802039200F10A02049200F10C020592DD
:10A3B80000F10E02069200F11002079200F1160257
:10A3C800089200F1180200F1040A00F1120800F1E5
:10A3D8001407099200F11A0B019A53FA82F1029AB2
:10A3E80053FA82FC039A9CF8CD959CF8CCC553FA95
:10A3F80082F20192049A53FA82F6059A53FA82F588
:10A40800069A53FA82F4079A53FA82F2029253FA9E
:10A4180088F20392089A91F8CD8591F8CC1553FAF1
:10A4280082F218440592099A53FA8AFE53FA87F77A
:10A4380090F8CDA590F8CC05049753FA82F29EF8CF
:10A44800CD7506929EF8CCE5019A00EB0A2001EB47
:10A4580008210EEB072E92F8CD8592F8CC75C3F83B
:10A468008C0596F8CD2501920CEB0920C3F89805C8
:10A4780095F8CDC596F8CC6595F8CC55019AC3F8F2
:10A48800901506EB0226049A0299C3F894E592F80F
:10A49800CDE592F8CC2591F8CD9591F8CC050399A6
:10A4A800019602EB0E22C3F8B425059A94F8CDA5BF
:10A4B800019E94F8CC45C3F8A06507EB082700EB8C
:10A4C800092091F8CD8591F8CC1592F8CD65C3F89F
:10A4D800AC0553FA8BFB92F8CC05069AC3F89C7529
:10A4E80005EB0C2504EB0A2401EB0821C3F8A4555D
:10A4F800C3F8A84592F8CD55C3F8B0159BF8CD45DB
:10A5080092F8CC159BF8CC2500EB0620C3F8B805CB
:10A5180001EB052102EB04220120C3F8BC15C3F8A6
:10A52800C0250BB0BDE8F08F93F8C705B3F8C88510
:10A538001D18821C019253FA82F295F8CC6595F8A1
:10A54800CD7592F8CDC592F8CCE500F1040A53FA1E
:10A558008AF2851D464429460295B64492F8CD559F
:10A5680092F8CC6553FA81F20EEB072E00F108073A
:10A578000397764453FA87F792F8CCE592F8CD25FD
:10A5880006EB0C2600F10A0197F8CDC50491B644F4
:10A5980097F8CC6553FA81F70EEB052500F10C010D
:10A5A80097F8CD8505912E4497F8CC5553FA81F745
:10A5B80006EB022600F10E0197F8CC2506913544EA
:10A5C80053FA81F605EB0C2500F1100153FA81FED0
:10A5D800154496F8CC2597F8CD7596F8CDC59EF814
:10A5E800CC65079105EB082500F112082A4453FAB7
:10A5F80088F502EB072200F1140795F8CD959EF82F
:10A60800CDE5324495F8CC6553FA87F500F116018B
:10A6180002EB0C22324495F8CCC5089153FA81F626
:10A6280002EB0E2200F1180195F8CD55099162440C
:10A6380096F8CCE596F8CDC502EB092253FA81F6D7
:10A64800724400F11A0B96F8CCE596F8CD6502EB4A
:10A65800052253FA8BF51C44724495F8CCE594F81E
:10A66800CB9595F8CD5594F8CA4502EB0C22964443
:10A678000EEB062E0EEB052E04EB09291FFA8EFEB3
:10A688001FFA89F9F1453FF4A7AE00200BB0BDE8E9
:10A69800F08FFF214FF6FF726AE600BF001000201E
:10A6A800504B5B68C3F3080370B4CBB9EFF3118365
:10A6B800B3B94D4A4D4E4E4D1368AC6811688B4284
:10A6C800FAD131688C42F7D84A4A15684FF47A7142
:10A6D80001FB05F2141BB4FBF5F401FB034321E075
:10A6E800EFF31181102383F3128803F1E023C9B239
:10A6F8009D681A6812F4803F3F4A1EBF0124146007
:10A708009D68394B1E68136881F31188394A1468AB
:10A718004FF47A71334401FB04F2521BB2FBF4F29A
:10A7280001FB0323354AD2F8F015591AB1F5FA7F1F
:10A7380014D90021C2F8F03582F8F41582F8F5151D
:10A74800C3B2042B26D0202B24D092F8EC1509B9DB
:10A75800552838D0814216D1002109E092F8F51524
:10A7680099B992F8F415C2F8F035C3B20029E8D0C7
:10A7780092F8C50554180138814284F8CC351DD0AB
:10A78800013182F8F41570BC7047013982F8F5156B
:10A7980070BC7047002102244FF6FF7082F8C7454D
:10A7A800A2F8C8055418581E814282F8EC3582F880
:10A7B800C53582F8C61584F8CC35E1D1012382F875
:10A7C800C43570BC704701241F2582F8EC05A2F837
:10A7D800C81582F8CC3582F8C64582F8C74582F894
:10A7E800C555CDE700ED00E0A44E00203C53002005
:10A7F80010E000E0385300203453002000100020FF
:10A8080038B500F166020446831EEA2123F8021FC8
:10A818009A42FBD140F649136385274B63600025B4
:10A82800CE2323810320E56713F0F0FB052013F006
:10A83800EDFB082013F0EAFB092013F0E7FB0A20E0
:10A8480013F0E4FB0C2013F0E1FB0D2013F0DEFB0A
:10A85800022013F0DBFB0121184A84F86D10506FB9
:10A868002B4601FA03F501330D2B40EA0500F8D118
:10A878004FF420635067A4F86E3040F60123A4F823
:10A8880070300F4BA366142384F86C30802384F84F
:10A89800803042F61403A4F878304FF6FF73A4F81A
:10A8A8008230A4F884304623A4F8863040F201238D
:10A8B800A4F8883038BD00BFCD004E0034280020F1
:10A8C8009808640038B50446002101234FF4FA7053
:10A8D80032220325E080257122812170E1706371A5
:10A8E800A37210200AF046F8607038BDF8B5354CF0
:10A8F800354D3C22002120462AF0D5FB334B95F8F4
:10A908000F66B3F858202284103393E8070095F8AF
:10A91800FA3595F8FB7584F822600C2B04F10C06C7
:10A9280084F8247086E8070009D801229A4041F685
:10A9380001510A4204D11846002B3FD1F8BD00232B
:10A9480094F82020042A34D0053A042AF3D8204A5F
:10A95800204BC4E90123204A61681368194843F071
:10A96800020313604FF4807323838847238B07EE19
:10A97800903AF8EEE77AF7EE006A86EEA77AB5F82D
:10A9880010364FF47A72A26284ED007A7BB1134ECE
:10A9980006F16C07B5F81036A16A00EE103A304699
:10A9A800B8EE400A2436F8F711FFB742F2D1012079
:10A9B800F8BD0B4A074BC4E90123CCE7012BBED1F4
:10A9C8000020F8BD702B002000100020F05400205B
:10A9D800D10A0008258500087029002014160020D7
:10A9E800C90A000870B590F8603044699AB073B924
:10A9F8004268537884F84430D1789378012243EA46
:10AA08000123A4F8463084F848201AB070BD0546E2
:10AA180002E02068F6F7D7FA2068F6F7DAFA002895
:10AA2800F7D1014662220DF106002AF03CFB154AD7
:10AA38001549D2F884360968144C92F88026039395
:10AA48000B4417920493124A6B69A6781148029036
:10AA580040F2FF51ADF80410CDE905235EB96078E6
:10AA6800642202FB004001A904302AF0F8FA01220E
:10AA78006B696670A2701868FF211AB0BDE8704053
:10AA8800FEF764BE00100020A44E0020B45300203E
:10AA9800A58600087453002090F8603063B910B59B
:10AAA8000278032A0DD0042A19D0022A1C4C0FD090
:10AAB800002384F8903610BD194B002283F89026A5
:10AAC8007047174C84F89136002384F8903610BDEF
:10AAD800012384F89136002384F8903610BD42682B
:10AAE800017E52780E4C0120814202F00F0284F858
:10AAF800910609D00229DBD1002AD9D0162084F882
:10AB080092360BF077FCD3E72AB1152084F8921619
:10AB18000BF070FCCCE716200BF06CFCC8E700BF0C
:10AB28000010002070B50B4C4FF0FF3504F525766A
:10AB38002368DC34184643B193F83430142B04D01E
:10AB4800F6F744FA854228BF0546A642F0D12846C2
:10AB580070BD00BF9416002038B51B4B9B78022BA4
:10AB680018D0032B194C10D00020D4F8003394F8D7
:10AB780028291344B3F5807FA8BF4FF4807383421C
:10AB8800A8BF0346C4F8003338BDD4F80403F6F769
:10AB98001DFAEAE700200E49034641F2264503F56F
:10ABA800A17201EB021205EB0314D279D20703F16B
:10ABB800010304D40A5D012A98BF00F500700A2B2E
:10ABC800EDD1024CD1E700BF3C2A00200010002044
:10ABD800BC6D002010B50C4B0C4C93F82D1993F854
:10ABE8002C29237882B00D311E320424017242725E
:10ABF8008DF804402BB901220DEB0401B62020F09A
:10AC0800B5FF02B010BD00BF00100020B029002021
:10AC180000B5094B83B01B7804228DF804201BB1C2
:10AC2800002003B05DF804FB012201A9B62020F042
:10AC38009DFF03B05DF804FBB029002000B5094B67
:10AC480083B01B7802228DF804201BB1002003B0CA
:10AC58005DF804FB012201A9B62020F087FF03B0AC
:10AC68005DF804FBB029002000B5094B83B01B78C0
:10AC780001228DF804201BB1002003B05DF804FB0D
:10AC880001A9B62020F072FF03B05DF804FB00BFF5
:10AC9800B029002000B5074B83B01B7800208DF841
:10ACA800040023B9012201A9B62020F05FFF03B0F8
:10ACB8005DF804FBB0290020ECE700BF70B504463E
:10ACC8000AF0AEFC6E4AD2F8343903F24C438342A0
:10ACD8000BD392F8383943B1022B8ABF92F8010599
:10ACE8000520023098420BDC70BD0121002382F858
:10ACF8003819C2F8340982F8004582F8FC3470BD6E
:10AD0800591CC9B288421344D4BF0125002582F8D2
:10AD1800381983F8004582F8FC54E5DC92F80255AE
:10AD28000023162D82F83839DED06B00290648BF7B
:10AD380083F0D503DBB213F0800F4FEA430318BF4B
:10AD480083F0D503DBB213F0800F4FEA430318BF3B
:10AD580083F0D503DBB213F0800F4FEA430318BF2B
:10AD680083F0D503DBB213F0800F4FEA430318BF1B
:10AD780083F0D503DBB213F0800F4FEA430318BF0B
:10AD880083F0D503DBB213F0800F4FEA430318BFFB
:10AD980083F0D503DBB292F8014513F0800F4FEA38
:10ADA800430318BF83F0D503022CDBB247D93549DA
:10ADB8000C44023111F8016F734013F0800F4FEA11
:10ADC800430318BF83F0D503DBB213F0800F4FEABB
:10ADD800430318BF83F0D503DBB213F0800F4FEAAB
:10ADE800430318BF83F0D503DBB213F0800F4FEA9B
:10ADF800430318BF83F0D503DBB213F0800F4FEA8B
:10AE0800430318BF83F0D503DBB213F0800F4FEA7A
:10AE1800430318BF83F0D503DBB213F0800F4FEA6A
:10AE2800430318BF83F0D503DBB213F0800F4FEA5A
:10AE3800430318BF83F0D5038C42DBB2BAD1024476
:10AE480092F8FF249A427FF44FAF7A2D02D07C2DDE
:10AE58007FF44AAF0C4A136E572B3FF745AF0B49A7
:10AE68000B480D684C680821995413440121C3F814
:10AE78000150C3F80540136E01700933136670BDA5
:10AE88000010002000150020382E00200515002095
:10AE98002E2E0020F0B518468BB01C460E461746DD
:10AEA80029F042FA1E2828BF1E2003232146024605
:10AEB8000546002402A88DF804308DF805708DF839
:10AEC80006608DF807402AF0CAF8064B1B7813B1C4
:10AED80020460BB0F0BD2A1D01A9B62020F046FE81
:10AEE8000BB0F0BDB029002010B582B000248DF859
:10AEF800043001AB8DF80540FFF7CCFF02B010BD60
:10AF080038B5A0F6640423796579DB0722D594F86F
:10AF1800483803B3D4F844341A68D36A5B085362D8
:10AF280094F84C3823B1B4F856380133A4F856389D
:10AF3800E94301F00101206C27F0B4FF012384F8F4
:10AF48004B38002384F8493884F84A38A4F8523832
:10AF580084F8483838BD94F84B38012B04BF94F86E
:10AF6800493884F84A382046FDF7F4FB94F84B3802
:10AF78004BB90123E94384F84B381940206CBDE8EC
:10AF8800384027F08FBF002384F84B3805F00101C3
:10AF9800206CBDE8384027F085BF08B5074B93F80B
:10AFA800391921B9012283F83929002008BD4B1E1F
:10AFB80059425941492010F005FEF6E700100020DB
:10AFC80010B5044B044C1A8804492046FBF714FFBB
:10AFD800204610BDE82A00203A19002052BA03087A
:10AFE80010B5054B0549B3F86C2003F63F1420460D
:10AFF800FBF702FF204610BD0010002052BA0308DC
:10B0080008B5044BB3F86A0040F4004010F0FEFFA6
:10B01800002008BD0010002008B50C4B93F9003043
:10B02800012B0B4B04D1002283F84429002008BDD2
:10B0380093F8440918B9012283F84429F6E701284E
:10B0480018BF022010F08EFFF0E700BFA00B002011
:10B058000010002070B5124C124B94F900401A7879
:10B06800012C05460E4605D1012A01D001221A708D
:10B07800002070BD012A03D1002010F073FFF7E70C
:10B08800022AF3D1084B002483F84449FFF7C4FF90
:10B09800064B314628461C70FDF7B2FCE8E700BFB6
:10B0A800A00B0020E02A002000100020EA2A00203F
:10B0B80038B5194D95F8A040762303FB045495F84C
:10B0C800133284F8EB30154B186815F027FA95F809
:10B0D800143284F8BE3095F8153284F8BF3095F8EC
:10B0E800163284F8C030B5F81832A4F8D830B5F85C
:10B0F8001A32A4F8D63095F81C3284F8F33095F853
:10B108001D3284F8173195F81E3284F8183115F07D
:10B11800D1FE002038BD00BF0010002058290020B3
:10B1280038B50D4B0D4A18680021034602F1090590
:10B1380014781C7254785C7294789C7235F81140BB
:10B148009C810131032902F1030203F10603EFD1C7
:10B1580015F0E4F9002038BD58290020D912002044
:10B1680008B5054B93F81F020138C0B283F8D8021E
:10B1780020F0DAF9002008BD0010002008B5054BC2
:10B1880093F812020138C0B283F8A0000BF043FA1A
:10B19800002008BD0010002010B5054C94F8A00050
:10B1A8000BF039FA94F8D80220F0BEF9002010BD4F
:10B1B80000100020F8B52E4DAB78022B4FD10FF0C0
:10B1C8003BFB0446D8B92B492B482C4EFBF714FE01
:10B1D80022462B4F2B49334607F64D10FBF70CFE42
:10B1E80033462246274907F65510FBF705FEAB788C
:10B1F80087F8F1322B88A7F8F2320020F8BD0FF05B
:10B2080011FB044630B920491B481C4EFBF7F4FDDE
:10B218002246DEE71D4C6378022B16D0032B1CD187
:10B228001B491548154EFBF7E7FD41F29853E458C2
:10B238004FF47A23B4FBF3F40FF0ECFA4FF4FA630B
:10B248000268B2FBF3F2121BC3E712490A480B4E1D
:10B258000024FBF7D1FD2246BBE70B49F6E70E4970
:10B2680005480E4E0024FBF7C7FD2246B1E700BF94
:10B278003C2A002059BA03084519002056BA030889
:10B288000010002072BA030861BA0308BC6D0020E0
:10B2980067BA03086DBA030885CB0308E1CA030837
:10B2A8002DE9F0411E4600238B55074608460C46FB
:10B2B800904629F039F8751E301A21182544404265
:10B2C8006A1A002AA5EB040312DA234420211A1B68
:10B2D800002A11DA0023A355094B93F85D19891B3D
:10B2E800234642463846C9B2BDE8F041F6F72ABDC2
:10B2F8002B5C05F80139E3E703F80119E7E700BF1C
:10B30800001000204B1E032B2DE9F04104460E4689
:10B31800274F0ED8274B586AFDF79AFDD7F8F43215
:10B328005B680BB100209847F31E012B30D90BF056
:10B3380069F9236800255B6887F8B0592046984763
:10B34800E37BC7F8F452013B022EE37301D0042ECD
:10B3580016D12046F6F719FD03220521164B204683
:10B36800F6F7F0FC236820465B6A984715F078FBEF
:10B3780015F0E0FAC8200BF0BDFD104B104ADA605A
:10B38800104A136823F4005313600020BDE8F081CD
:10B3980097F85E59DFF83080013D6B1CC7D058F82C
:10B3A80035305B680BB100209847013DF5E700BFD9
:10B3B800001000202C00002078BA030800ED00E0FF
:10B3C8000400FA050C2B002060190020F0B4214A73
:10B3D80092F9FC42D2F8F452214491FBF4F304FBB5
:10B3E800131192F8FD4282F8F812CBB2A9686343B0
:10B3F8000E2505FB03130021C2F8B43982F8B819E9
:10B408001D462F790E2FCEB201F101011AD1B44297
:10B41800214628BF3146102982F8B81984BF102167
:10B4280082F8B81992F8B8190139C9B282F8B8196E
:10B43800C1EBC101084A03EB4101994204D2F0BCB7
:10B44800F6F7A3BC0E35DCE75C7B02F8014F0E3340
:10B45800F3E700BF00100020B819002038B5164BDC
:10B46800D3F8F422526805461C46BAB994F85E0926
:10B4780098B10138C0B284F85E0904EBC00000F549
:10B48800166003C80D4B83E80300FDF7F0FC28465F
:10B4980094F9F812FFF79AFF002038BD93F9F902E2
:10B4A800D3F8B439C0EBC00003EB40009047002844
:10B4B800DCDA4FF0FF30F0E700100020F412002033
:10B4C80038B505460C4641B31D4BD3F8F4228A42E1
:10B4D80025D093F85E29082A1FD8511C83F85E19D5
:10B4E80003F53D7103C903EBC20202F5166282E857
:10B4F80003000022C3F8F44283F8F922236833B129
:10B508009847013003D12846BDE83840A6E7FDF743
:10B51800AEFC00212846FFF759FF002038BD93F9FB
:10B52800F91293F8FD2291FBF2F402FB141283F84E
:10B53800F922FDF79CFC21462846FFF747FFECE778
:10B5480000100020424A92F8B01970B5D2F8CC59D0
:10B558001446002947D115B9C2F8D05970BD3D4BE2
:10B568009A6A002AB8BF99629B6A04EB8303D3F8EE
:10B57800D439C4F8D039002BF0D0012384F8B0397D
:10B58800354BC4F8F4320023A4F8F8324FF40050D5
:10B5980084F85E3907F0EEFBD4F8D009F6F7E8FB3B
:10B5A800D4F8D009437A027A112B4FF001013FD821
:10B5B80084F8E419022184F8E519002184F8E619D1
:10B5C800510884F85D3984F8FD12017B31B10021FE
:10B5D80084F8E61984F85D3984F8FD22D4F8F41269
:10B5E800BDE870406CE75DB11A48816A013191FB92
:10B5F800F5F205FB1213836204EB8303D3F8D459E5
:10B60800D4F8D069AE42A9D094F8F92294F8F81287
:10B6180094F8FD3201FB032384F8F932336830468D
:10B628005B689847F37BC4F8D059013BF373B3E7E1
:10B6380084F8E519022184F8E619991E002584F892
:10B648005D19911E84F8E45984F8FD12BDE700BF26
:10B65800001000202C00002048000020F8B5BF4B47
:10B66800D3F8F42206460D461C460AB9FA2005E02E
:10B67800062904D1FFF766FF4FF4FA70F8BD0529D3
:10B688000ED193F8E7292AB1002283F8E7294FF46D
:10B69800FA70F3E73046FFF7E1FE4FF4FA70EDE792
:10B6A800072908D10022AE4983F8E729FFF708FFE8
:10B6B8004FF4FA70E2E7022945D193F8E7795FB9C8
:10B6C80093F9F93294F8B829934233DA013384F8BC
:10B6D800F9326B1E012B03D894F8E739002BC5D03B
:10B6E80094F9F932D4F8B419C3EBC30201EB42015F
:10B6F8000A79013A0C2AB9D801A050F822F000BF03
:10B7080003B80008E9B70008AFB70008C5B70008D4
:10B7180015B80008FFB800088DB8000845B900083A
:10B728007FB9000875B600088DB8000839B8000858
:10B73800BBB8000894F8F812013149B2FFF746FE89
:10B7480084F8F972C5E70129C3D193F8E739002BCA
:10B75800C2D194F8F912D4F8B4294B1E5BB2C3EBEA
:10B76800C30002EB400084F8F932007920B9002BBD
:10B77800C4BF023984F8F91294F9F932581C06D07A
:10B78800C3EBC30302EB43031B79002BA4D194F84A
:10B79800F812013949B23046FFF718FE94F8B83963
:10B7A80084F8F93295E7042D7FF460AFD1F80910D9
:10B7B8003046FFF785FE4FF4FA705FE7D1F80530A1
:10B7C800002B3FF453AF042D7FF450AFD1F809108C
:10B7D8003046984701303FF45DAF4FF4FA704DE7BB
:10B7E800D1F80530002B3FF441AF042D7FF43EAF74
:10B7F800D1F8091030469847EFE73046FFF72EFE9C
:10B80800002384F8E7394FF4FA7037E7D1F80920B4
:10B81800002A3FF42BAF291F4D424D4115701C449F
:10B82800FA2094F8B92942F0010284F8B92925E7E9
:10B83800D1F8091000293FF419AF042D94F8E7292D
:10B8480007D1002AEBD14749012284F8E7298A6306
:10B85800E5E7002AE3D0012D07D1424A926B0A326C
:10B8680095400A8815430D80D9E7022DD7D13D4A66
:10B87800906B01220A3002FA00F00A8822EA0002DC
:10B888000A80CCE7D1F8090000283FF4EFAE07683A
:10B89800042D3A7806D1457995423AD980790244FF
:10B8A8003A7036E00579954233D28079121A3A70A7
:10B8B8002FE0D1F809000268042D137816D1007919
:10B8C800984201D901331370D1F805301BB1D1F872
:10B8D80009103046984794F9F9321C44FA2094F834
:10B8E800B93943F0010384F8B939C7E6002BEBD026
:10B8F800013B1370E8E7D1F8090000283FF4B6AE21
:10B9080007683A78042D55B213D190F905C0AC45B3
:10B91800C4DC1C4494F8B92942F0010284F8B9291E
:10B92800D1F80530002B3FF4A1AE30469847FA20F5
:10B93800A4E690F904C0AC45EBDAB6E7D1F8090003
:10B9480000283FF493AE0768042D3A880CD1C588C7
:10B958009542DED9008902443A80DAE700100020D7
:10B96800580000202C00002085889542D1D20089FB
:10B97800121A3A80CDE7D1F8090000283FF476AED4
:10B988000768042DB7F9002012D1B0F90650954286
:10B9980002DD008902443A801C4494F8B93943F026
:10B9A800010384F8B939D1F80530002BBDD15DE623
:10B9B800B0F904509542EFDA0089121A3A80EBE7A1
:10B9C8002DE9F04F734BD3F8CC29002A89B0814672
:10B9D8001D4632DBD3F8E82902F543425032904243
:10B9E8002BD393F89266C3F8E80936BB93F8B0896D
:10B9F800B8F1000F24D1684BDA88A2F2E342B2F51D
:10BA0800F97F15D8B3F9041040F2E14291420FDCF6
:10BA1800B3F9022040F2D6639A4209DD5F4B1B78E6
:10BA2800DD0705D4FFF78EFD5D4B4FF4FA729A8758
:10BA38005C4B1A68574BC3F8F42909B0BDE8F08F7E
:10BA480095F8EC49D5F8D0B9554F4FF47A73B0FB57
:10BA5800F3F30293DCB121465846FFF7FFFD85F862
:10BA6800EC69B887D5F8B439002B40F09D80494C73
:10BA7800029AD4F8F83903F5FA739A42D8D9D4F867
:10BA8800D009F6F753F9029BC4F8F839D0E7424BCE
:10BA9800D988B3F90220A1F2E341B1F5F97F19463B
:10BAA80013D8B3F9040040F2E14398420DDC40F2A8
:10BAB800D6639A420DDD394B1B7813F0010F0CBF8A
:10BAC800062401247B6C01331AE040F2D6639A42C3
:10BAD80022DC40F2E1439A4220DDB1F900009842AD
:10BAE8001EDD40F2D66290421CDCB1F90410994286
:10BAF8001ADD91421ADC012300223B64C5F8F029C3
:10BB0800B7F93C207B64002A12DDD5F8F4391344D8
:10BB1800029A9B1ABB87A5E70124D3E70224D1E741
:10BB28000324CFE70424CDE70524CBE70724C9E79E
:10BB3800002C97D04FF0000A3B6C5046534520DC50
:10BB4800033C00B2012CB8878CD87B6C142B89DDA0
:10BB5800A3F1140290FBF2F03228B88782DCD5F802
:10BB6800F0290AB9C5F8F039D5F8F0299B1A3A6CCA
:10BB7800052193FBF1F313448B42C8BF0B463B648A
:10BB880070E72146584601930AF1010AFFF766FD5E
:10BB9800019BD3E700100020402B0020FF28002045
:10BBA8002C000020A44E002095F8E439D5F8D0796F
:10BBB800002B40F0CE8095F8B8293B7A9B1A0222D8
:10BBC80093FBF2F3DBB20193D5F8FC3903F5C333E9
:10BBD800A03399453B6888BFC5F8FC99DB6A3846AD
:10BBE80088BF464698477A7B1FFA80F9002A00F0FA
:10BBF800BE8095F8B839D5F8B419C3EBC30301EB87
:10BC080043030022994202F1010440F2A580002377
:10BC18007B73D5F8B40995F8F93259B2C1EBC10272
:10BC280000EB420201331279DBB2002AF5D097F912
:10BC38000E2085F8F912002A0FDB8A4228D095F8E1
:10BC4800E539019903FB0212D2B2B44B95F8E61913
:10BC58003846F6F777F8A9EB0009B9F11D0F7FF61A
:10BC680006AF95F9F92297F90E30934214D095F85A
:10BC7800E539019903FB0212D2B2A94B95F8E619EE
:10BC88003846F6F75FF895F8F932BB73A9EB000967
:10BC9800B9F11D0F7FF6EBAE0023D5F8B489DFF8B4
:10BCA8009CA2039395F8B839D5F8B4299DF80C40AF
:10BCB800C3EBC30302EB430398453FF6D8AE2E19F6
:10BCC80096F8B93998071ED5019B95F8E52995F896
:10BCD800E61902FB043298F80430002B18BF013132
:10BCE800D2B2D8F80030C9B23846F6F72BF896F831
:10BCF800B939A9EB000923F00203B9F11D0F86F841
:10BD0800B9397FF6B4AE2B1993F8B929D10740F1A8
:10BD18008980019B95F8E56906FB043695F8E439B6
:10BD2800F6B20BB10136F6B298F804300D2B00F2DA
:10BD38005681DFE813F039015401540145004500EC
:10BD48007D00DD00D200E800E800380005019B0016
:10BD58008E000123019337E755FA82F20E3192F8EB
:10BD6800B90940F0030082F8B90922464AE7002ED3
:10BD78003FF44FAF95F8B839D5F8B419C3EBC303FE
:10BD880001EB430399423FF644AF487B440707D58C
:10BD980055FA82F494F8B90940F0010084F8B90919
:10BDA8000E310132EEE7D8F80910002900F01781AA
:10BDB8000C2204A829F0B5F90C23324604A921E085
:10BDC8000DF1200B4FF00001032B0BF8101D0AD1C9
:10BDD800D8F805303BB1120705D598470C22014623
:10BDE800584629F09EF94E49584629F064F99AF8C0
:10BDF800E4390BB1013EF6B2584628F095FA3246BE
:10BE0800C3B2594654443846FFF74AFA94F8B93948
:10BE180023F0010384F8B939A9EB0009B9F11D0F22
:10BE28007FF625AE039B013308F10E08039339E72B
:10BE3800D8F809000028EFD003782BB1394904A8B5
:10BE480029F055F90323B8E7374904A829F04FF931
:10BE5800F8E7D8F809301A689B68117804A853F8ED
:10BE680021100C2229F05DF90C23A6E7D8F8090067
:10BE78000028D1D02D4A0088D2F800C09AF9F932AA
:10BE88004FF47A710005BCFBF1F201FB12C29AF87B
:10BE9800E71913D569B1B2F5FA7F0AD29C4208D1E5
:10BEA800234B9B6B012B04D11C4904A829F01FF9D3
:10BEB800C8E7204904A829F01AF9C3E741B1B2F547
:10BEC800FA7F05D29C4203D1194B9B6B012BEBD017
:10BED800194904A829F00BF9B4E7D8F80900002893
:10BEE8009AD0036804A9187826F0C8FE052364E7E9
:10BEF800D8F8090000288FD0036804A993F9000036
:10BF080026F0BCFEF2E7D8F80900002884D00368C0
:10BF180004A9188826F0B2FEE8E700BF32960308A5
:10BF280004CB030885BA030889BA0308A44E002085
:10BF38002C000020DC97030887CB030800100020A2
:10BF4800D8F8090000283FF467AF036800891B7818
:10BF5800584300F5C33004A9A03026F08FFE9DF8A1
:10BF680012209DF811308DF811202E228DF8122004
:10BF78009DF815208DF81030302A01D02E2A0DD1C9
:10BF88004FF000028DF815209DF81420302A01D0BA
:10BF98002E2A03D14FF000028DF81420302B04BF55
:10BFA80020238DF81030A1E7D8F809B0BBF1000FB5
:10BFB80017D0D8F8000028F0B7F995F8E61901313C
:10BFC80001442C445B463246C9B23846F5F7BAFEFE
:10BFD80094F8B93923F0010384F8B9391CE7002033
:10BFE8001AE7584618E700BF10B9074A1075704796
:10BFF80010B5054C606027F03BFA4FF6FF7202233C
:10C00800A281237510BD00BF442A00200B4B9B78EA
:10C01800022B08D0032B04D1094BD3F80403F4F7FF
:10C02800CFBF00207047074A41F2BC43D358002BCA
:10C0380001DD0DF0D3B90120704700BF3C2A002074
:10C0480000100020BC6D0020F0B5184E002383B00E
:10C0580004460821D6F8000A86F8B93302ADF4F789
:10C06800BBFFD6F8000A8121F4F7B6FF8923D6F87A
:10C07800006A25F8023DE71D14F8010B32462946EF
:10C0880011F0C6FCBC42F7D1BDF806301A0A52FAC4
:10C0980083F3C3F1FF039BB23246D8B20021ADF857
:10C0A800063011F0B5FC03B0F0BD00BF0010002051
:10C0B8000FB400B583B004AB054953F8042B0193C2
:10C0C8000020F7F785FF03B05DF804EB04B0704774
:10C0D800DDDE00082DE9F04FA14DAB789A1E012A4C
:10C0E80089B040F2AB800321A970802006F014FECD
:10C0F8000746002800F0A980802106F003FE7E791B
:10C10800984B994C97F9027084F8040A03EB86035C
:10C118000222D3F86C310093B3F5613F0CBF11468E
:10C1280000210023CDE9012138461A46802106F076
:10C1380081FC0C3E032EC4F8040300F2F380402374
:10C1480084F82839002800F08180884AE978166840
:10C15800874A884B52882D88A4F8D02B003118BF05
:10C16800012116F0020F14BF0A46002294F8820338
:10C1780093F80AC0079215F1FF354FF0000293F8C3
:10C1880009B094F8D47BDFF8FCE17B4B9EF800A063
:10C19800DFF8F481DFF8F4E1C4F80C2A18BF0125B0
:10C1A800801A18BF01201CF0FD0F14BF4FF0010CBE
:10C1B8009446BBEB0201A7F1190BBBFA8BFB18BF26
:10C1C80001214FEA5B1B012F059103F1200914BFE0
:10C1D80059460121C3E90122C3E9032203F1AC074F
:10C1E8000491BAEB020AC6F3C001C4F8209A03F519
:10C1F8009C79C6F3800B0691C4F8247AC4F8289A6F
:10C20800D8F800709EF800900799079418BF4FF06F
:10C21800010A164690464FF0010EF3B25A1E152A2F
:10C228001CD8DFE802F03939393939393939352933
:10C2380025312D1F194848485444581F032B3FF4F3
:10C2480054AF4E4B5A78012A7CD8474C002384F8C7
:10C25800F03209B0BDE8F08F02463AB10EFA06F2A4
:10C2680048EA02080133DBB2162B38D80136D4E786
:10C278005A46002AF2D1F9E7069A002AEED1F5E7E4
:10C288006246002AEAD1F1E7059A002AE6D1EDE7ED
:10C29800049A002AE2D1E9E7994534BF0022012235
:10C2A800002ADFD00EFA06F248EA0208DAE70A4660
:10C2B800002AD3D1DAE706EB460207EB420212F86E
:10C2C800562C003218BF0122002AEBD1CAE72A46B1
:10C2D800002AC3D1CAE75246002ABFD1C6E7079C45
:10C2E8001320C4F8D88B16F0A3F8D4F8E45BD4F87C
:10C2F800EC1B84F8DC0B00230222C4F80C33A4F8EE
:10C308001033A4F81433A4F81633C4F8083384F8A7
:10C31800F43BC4F8E05BC4F8E81B84F8F02209B0E9
:10C32800BDE8F08FD4F8083A154A03EB4303A2FBA3
:10C3380003235B0911D0402BA8BF4023DBB284F84C
:10C348002839FFE641F2D5529B5C002B7FF47DAF84
:10C35800054C402384F82839F7E60123EFE700BFAE
:10C368003C2A0020B06A0308001000207029002031
:10C37800502900201C2800200C1A0020BC6D002029
:10C38800D34D621070270020582900205127002023
:10C3980008B5084B9B78032B06D0FFF79BFE064B8E
:10C3A800012283F8F52B08BD27F098F80028F4D06F
:10C3B80008BD00BF3C2A0020001000202DE9F04FE6
:10C3C800AD4CAE4D237D012B83B000F06882022B6B
:10C3D8000CBF0723002385F8F63BA94B19780022E8
:10C3E800CB1E85F8F72B85F8F82B2A2B1AD8DFE80F
:10C3F80003F04A19194A19191919191919194A1951
:10C408004A19194A1616161619191919191919193E
:10C418001919191919191919191919194A0001237A
:10C4280085F8F83B0023227985F8F93B232085F825
:10C43800FA3B85F8FB2B0AF05DFD95F80936002BD1
:10C4480040F0E18195F8FA0BB0B903B0BDE8F08F80
:10C458008C4A8D4B8D49F161C6E900238C4995F8CA
:10C46800FA3B0A6842F001020A60072286F8632054
:10C4780043F0010385F8FA3B95F8FB3B13F0FD0305
:10C4880004D00120E1E785F8F71BCBE7E278814E7D
:10C49800A17894F8260086F88C06003218BF01228D
:10C4A80095F80F0686F85D20012995F80E2686F87E
:10C4B800612086F85A0096F8582000F047820A2A28
:10C4C800637800F0F0810C2A40F04B8202229FED45
:10C4D800727A86F85B2007EE903AF8EEE77A6F4FAB
:10C4E80086F85E1067EE877A013BFCEEE77A86F8FD
:10C4F8006030C7ED007A33686648984796F863302D
:10C508000F2B07D8012202FA03F34CF2FF110B425A
:10C5180040F02482002386F8623024F0FFFE94F86D
:10C528002120638CDFED5E6A5E49B4F824B0D7F849
:10C538000080A5F80CBC07EE102AB8EEC76AB7EE63
:10C54800007A07EE903AF0EE475AE6EE665A0B4646
:10C558004FF47A70A6EE267AA5F8FC0B524FE3EC5E
:10C56800015AF8EEE77A83ED007A67EEA67A94F836
:10C578002030C1ED027A0AB987F84820032B00F071
:10C58800CE81002B00F0D981012B04BF40F2355336
:10C59800A5F8FC3B07EE908A9FED440A444CF8EE60
:10C5A800677A80EE270A28F0FFFCB5F8FC9B032386
:10C5B80090FBF3F39945A8BF99461FFA89FAA5F8A5
:10C5C800FCAB07EE90AAFBEEED7A17EE903AB0EED0
:10C5D800670A44F8083B28F0E7FC4FEA5A019BFB3E
:10C5E800F0F09FED345ADFED345ADFED343A9FED29
:10C5F800342ADFED342A9FED343A9FED341ADFED0B
:10C60800341ADFED346A85F8140CA5F8161C0023DB
:10C6180007E00133B6EE007A202BA4EC017A00F093
:10C628008C8007EE903AF8EEE77A67EE857A37EE77
:10C63800A57ABDEEC76A16EE102A2032402AE8D83D
:10C64800F4EEE57AF1EE10FA40F33E819FED226AAE
:10C6580001E0B0EE677AB4EEC67AF1EE10FA77EE42
:10C66800667AF6DCF4EEE37AF1EE10FA40F129810D
:10C678009FED1A6A36E000BF805B002000100020A2
:10C6880070270020832300080D84000890C1793D9D
:10C6980070290020F054002000009C43A85B002073
:10C6A8000AD7233C001C00202C00002000247449D9
:10C6B800101C00203C8C4F3EDB0FC93FDB0F49C0EC
:10C6C80092E741B99730083C15A82ABEDB0FC9BFCD
:10C6D800DB0F4940DB0FC940E4CB1641E4CB16C160
:10C6E800F0EE477AF4EEC67AF1EE10FA37EEA67A53
:10C6F800F6D4B4EEE57AF1EE10FA40F3DA8031EED2
:10C70800C77A27EE076AB0EE624AA6EE024A0133FC
:10C71800202BF0EE430AE6EE040AF7EE007A67EE05
:10C72800464A37EEC77AF6EE007AA4EEA07A27EEEC
:10C73800277AA4EC017A7FF474AF974AB2FBF8F039
:10C7480080B2B0FBFAF0C0B207EE900AB2FBF9F281
:10C75800F8EEE77AF7EE006A86EEA77A0C2404FB77
:10C7680008F8424538BF42468C4CA6F80C3504F10F
:10C77800A80E4FF0100C142304F12808C6F810E591
:10C78800A6F8FCC4A6F8801607EE902AF8EE677A99
:10C7980086EDD97AFCEEE77AA6F8861686F8610364
:10C7A80017EE901A9FED7E0A7E48A6F80835C6F85F
:10C7B8000445C6F80085CDED017AF7F707F8B5F816
:10C7C800163C01999FED760A7748A6F88236A6F8B6
:10C7D8008836F6F7FBFFB5F8163CA6F88436A6F8B7
:10C7E8008A369FED6F0A71480199F6F7EFFF97F8BF
:10C7F800493023B196F86230003318BF012387F817
:10C808004930012021E695F80A36694E013B5BB2B2
:10C818000222591C32743FF415AE93423FF712AE10
:10C828001B01644AD358002B3FF40CAE95F80B0655
:10C8380000283FF407AE7361F4F78AFDB06128B1B0
:10C8480095F908361C220133C37182710D21F4F762
:10C85800D3FFB069F5F74FF95748F5F7D9FB074605
:10C86800A8BB95F80B06DFF88481F4F771FD534BEC
:10C878003E4681461F6800E0013606EB4603BE428D
:10C8880003EB080ABFF6DEAD18F80300F4F760FD05
:10C898008145F1D131465046F5F781FAD2E50423B6
:10C8A80085F8F63B99E5042286F85B209FED447AEB
:10C8B80011E6B4EEC17AF1EE10FA48BF33EEC77A4A
:10C8C8001FE7B0EE677A14E7F0EE477ACAE6042865
:10C8D80086F858003FF4BCAD092833D801238340BB
:10C8E80013F4587F49D0374BF361BB1FDBB236498D
:10C8F800364A032BC6E900123FF6B0AD344A354933
:10C908001A440B6892F8AC2186F8632043F00103BF
:10C918000B6095F8FA3B002A7FF4AAAD92E5E38B09
:10C92800B3F5A77FFFF436AE40F2622240F23551EC
:10C938009342A5F8FC1B7FF62DAE4FF4FA63A5F8D9
:10C94800FC3B27E6002386F863307BE50A2A0ED0F5
:10C9580086F85B309FED207A0B46BCE586F86220AE
:10C96800DBE5032286F85B209FED1C7AB3E586F8A9
:10C978005B100B469FED1A7AADE51B06E2D596F8DB
:10C988005D30DFED187A9FED187A002B18BFF0EEB6
:10C99800477AC6ED077AA8E740420F00606C0308A3
:10C9A80000004842045B0020285B00204C5B00200C
:10C9B800F05400201029002000550020405300208A
:10C9C800E438DE4290C1793DA9310008F920000819
:10C9D800B06A03087029002000007A440000FA4277
:10C9E800D145634490C1793D90C1F93D445300203D
:10C9F80038B5394B5B68C3F30803CBB9EFF3118340
:10CA0800B3B9364A364D374C1368A06811688B4263
:10CA1800FAD129688842F7D8334A11684FF47A72F4
:10CA280002FB01F4241AB4FBF1F402FB034421E0F5
:10CA3800EFF31181102383F3128803F1E023C9B2C5
:10CA480098681A6812F4803F284A1EBF01201060B7
:10CA58009868224B1D68136881F31188224A11686F
:10CA68004FF47A7404FB01F22B44121AB2FBF1F270
:10CA780004FB03241E4DD5F8B433E31AB3F5FA6F5B
:10CA8800C4BF002385F8B83395F8B83323B9002319
:10CA9800C5F82833012038BD00221649D5F82803E7
:10CAA80010F084FD95F8B8337BB9134B1B781C2B19
:10CAB80004D1D5F8983C114AE31AD3800023C5F86D
:10CAC800984CC5F82833012038BD0D48FFF7BCFA4B
:10CAD800002385F8B833E8E700ED00E0A44E002015
:10CAE8003C53002010E000E038530020345300206D
:10CAF80000100020B81300207027002074270020A1
:10CB0800886D030870B50446CC2582B04430617145
:10CB1800A11D2571CDE90010251D9AB16E4611465B
:10CB280030461A46F6F786FD30462946F7F7B8F933
:10CB3800009A019220680095521B2946F4F720FAC2
:10CB480002B070BD6E46EFE72DE9F04F9E4DDFF85D
:10CB580088B2AB7887B005F104084FF0640ADBF8B7
:10CB680000604BB32C780AFB045214461369043452
:10CB7800002B54D09E4252D9D36D002B00F38C80E9
:10CB880002274FF000090BE0AB7085F800909BB1CD
:10CB98002B69002B42D0B34240D2EB6D002B7BDCDB
:10CBA800236984F860702046444603B19847AA7800
:10CBB800531EDBB2002AE7D1844C854FDFF814827C
:10CBC80004F69C4604F54A6900255FFA85FA0AF1DD
:10CBD800180B5FFA8BFB584615F050FC00286ED0F6
:10CBE800735D002B40F0D780BBF1190FB4F8E63C19
:10CBF80000F0D680BBF11A0F40F09F805B077CD510
:10CC08003B78D90700F18580D8F800209206434682
:10CC180000F161814FF01B0A0221C6E044466369B6
:10CC28001868F4F7D6F90028C6D063691868F4F7CD
:10CC3800CAF9A37853B994F85720012A04D02AB91D
:10CC4800552803D0AB788AE7CC28FBD16268D0544A
:10CC5800A37862780133DBB29A42A370F2D194F8D8
:10CC68005730012B35D0002B43D1626811785529F4
:10CC780073D02369012284F86020002BE2D020467B
:10CC8800984794F86020AB78002A7FF468AF002BAF
:10CC98004ED1DBF800308FE794F85730012B3BD0AA
:10CCA80023B9636921781868FCF750FDA268A36D61
:10CCB8001644013B0022E660A365A2707CE70AF1F6
:10CCC800190A70555FFA8AFABAF11B0F1AD00135A2
:10CCD8007BE762B16668013EB718002016F8011FAD
:10CCE800F7F71AF9BE42F9D1021C18BF012284F8DD
:10CCF80060202369002BC2D1C3E7D4F888365807CF
:10CD08003FF57EAF94F8B0391BB9314B1B78DB0780
:10CD180064D507B0BDE8F08F60690368002BC5D003
:10CD280094F85630217804F11802FFF7EBFEBDE7BE
:10CD3800013BDBB2AB702A7011E70AF1190A9A07B6
:10CD48005FFA8AFA77D53B78D807BDD4D8F800308F
:10CD580013F02003B8D1194627E05178012988D16A
:10CD68009178FF2985D11179AA2982D1D678D170F5
:10CD780061680F1D11F8012B5340082204E05B0085
:10CD8800DBB2013A00F0AD801806F8D5580080F003
:10CD98003100C3B2F5E70AF1190A5FFA8AFA93E794
:10CDA800D9074ED54FF01A0A012194F8E43C8DF8C2
:10CDB8001610012B4AD023B90131D4F8A00CFCF786
:10CDC800C5FC012373557FE7B453002000100020F1
:10CDD800FF2800200C2B0020A44E0020774B1B6856
:10CDE80013F0200395D194F89126002A39D0744A7B
:10CDF8009188A1F24751B1F5957F8AD85188A1F25F
:10CE08004751B1F5957F84D81288A2F24752B2F5FE
:10CE1800957F3FF67EAF6B4A029202214FF4C872AB
:10CE2800CDE9002168481A46032123F00CFE0123AE
:10CE380084F890366DE7D4F888369B077FF544AFC1
:10CE480081E7D4F88836DA07ACD440E7D4F8A02CC8
:10CE5800002AB6D019460DF116024846FFF752FED1
:10CE6800AFE794F89036002B7FF453AF544B94F807
:10CE78009216D888A0F2475080B2B0F5957F39D87D
:10CE8800B3F90020A2F24755ADB2B5F5957F67D842
:10CE98005D88A5F24755B5F5957F43D8B3F9045099
:10CEA800B5F5876F3EDA00293FF433AF06AA0223AF
:10CEB80002F8013D434901934FF4C873029100936E
:10CEC80004210123404823F0BEFD012384F8913654
:10CED80084F890361DE794F8B029002A3FF47FAF14
:10CEE80017E7B9427FF446AFF31A18BF012384F855
:10CEF8006030FEE600293FF40CAFB3F90020B2F52C
:10CF0800876F30DA022306AA2E4802F8013D022173
:10CF18004FF4C873CDE9011000932B48012323F087
:10CF280092FDD2E7F9B95A88A2F24752B2F5957F35
:10CF38003FF6EFAEB3F90430B3F5F06F7FF7E9AE23
:10CF480006AA01231F4902F8013D022002914FF46D
:10CF5800C871CDE9001004211B4823F074FDB4E723
:10CF68000029CCD1D5E6B3F90210B1F5F06F1FDC7A
:10CF7800B2F5F06F1EDCB1F5876F1DDBB0F5957F5C
:10CF88003FF6C7AEA2F2475292B2B2F5957F3FF68E
:10CF9800C0AEA1F2475292B2B2F5957F3FF6B9AE54
:10CFA800B3F90430B3F5F06F7FF7B3AE0123AAE706
:10CFB8000423A8E70323A6E70523A4E70C2B0020F6
:10CFC800402B0020A1AA0008A01C002030B51B4C53
:10CFD80085B000254FF4804084F8E85C05F09CFE9D
:10CFE80018B34FF4E133032290F902000295CDE91A
:10CFF80000324FF480412B462A4605F01BFD94F879
:10D008008C36C4F8A00C84F8E43C70B10C4994F850
:10D018008026D4F884360093CDE901212B462A4690
:10D02800294604F54A6023F00EFD012384F89C3C50
:10D0380084F89D3C84F89E3C05B030BD001000206B
:10D04800EDA9000838B50B4C0B4BC4F8EC3C04F6C2
:10D05800EC452846FDF7F2FD00210122FF23284672
:10D0680084F8F81C84F8F92CA4F8FA3CFDF7B2FD12
:10D07800284638BD00100020906D030888B10029AB
:10D088000EDD03798B420BDB002A09DD43799342DD
:10D0980006DB02EBC102093A836833F812007047D5
:10D0A8000020704708B5074B93F84A1049B193F828
:10D0B8004B2032B1044B1868FFF7E0FF034BA3F88D
:10D0C800FC0C08BD2C000020AC290020001000201A
:10D0D80008B5064B93F84B2022B9012283F84B2060
:10D0E800002008BDFFF7DEFFFAE700BF2C00002094
:10D0F80008B5064B93F84A2022B9012283F84A2042
:10D10800002008BDFFF7CEFFFAE700BF2C00002083
:10D1180008B5054B1A78054B1978054B1868FFF7C1
:10D12800ADFF044B188008BDE32A0020E22A002046
:10D13800AC290020E42A002008B5074B93F9002009
:10D14800064B12B91A70002008BD1A780AB90122D4
:10D15800F8E7FFF7DDFFF6E7A00B0020E22A002042
:10D1680008B5074B93F90020064B12B91A70002036
:10D1780008BD1A780AB90122F8E7FFF7C9FFF6E7F0
:10D18800A00B0020E32A002070B5384B86B01A782F
:10D198008DF80C205A788DF80D2000269A78CDF855
:10D1A8000E608DF80E209A88ADF810201A7ACDF806
:10D1B800126003AD8DF8142095E807006C4603C48F
:10D1C80022802B4A1278022A1C4632D1294B197820
:10D1D800294B8DF800101A78284B8DF80120186813
:10D1E800FFF74CFF264BADF8040093F84439E3B938
:10D1F80005200EF0B7FE234B0A221E788DF8026038
:10D208006946284627F01CFF58B19DF80030237066
:10D218009DF801306370BDF80430A670A38009F052
:10D22800F1F94FF0FF3006B070BD06200EF09AFEFF
:10D23800E1E7154B1B7873B90E4B19780E4B8DF837
:10D2480000101A780D4B8DF801201868FFF716FFAB
:10D25800ADF80400CFE730460EF084FE0B4B8DF896
:10D2680000601B88ADF80430C5E700BF78290020AE
:10D27800E02A0020E22A0020E32A0020AC2900202E
:10D2880000100020E62A0020EA2A0020E82A0020D0
:10D2980003685B6A184703681B6A1847F8B5214F8B
:10D2A8003E68002E3BD0204B1B7813B11F4A82F8F2
:10D2B8004A301F4B1B7813B11C4A82F84B30FFF7DA
:10D2C800F1FE1C4B1C4C1B78013384F839391B4B7D
:10D2D8001B883BB1154D3868691CFFF7DCFF08B99E
:10D2E80001236B703279164B84F8042DF268C4F868
:10D2F800082D5A1CC4F80C2D727984F8102D326947
:10D30800C4F8003DC4F8142D493BC4F8183DB3795E
:10D3180084F81C3DF369C4F8203D0020F8BD4FF0A7
:10D32800FF30FBE7AC290020192700202C00002043
:10D338001A2700201427002000100020162700209C
:10D348007600002003685B69184730B405798D4280
:10D3580006D34579954203D3036830BCDB68184788
:10D3680030BC704770B5134E134C356894F84A10AA
:10D3780094F84B202846FFF7E8FF6178AB798B4299
:10D3880003D32B6828461B6998470C4D0EF0BEFB4B
:10D3980094F84A1094F84B206378306829706A70C2
:10D3A800AB70FFF76BFEA88009F02CF94FF0FF3047
:10D3B80070BD00BFAC2900202C0000207829002077
:10D3C80010B50C4658B1F3F7C3FF18B103238371A6
:10D3D8000023C3712146BDE81040F4F70DBA10BD13
:10D3E80010B5044601210079FFF7EAFF6379216847
:10D3F8009A0802239340C868DB439BB20340CB6082
:10D4080010BD10B5044622210079FFF7D9FF6379D2
:10D418002268990802238B40D94389B21161D168E7
:10D428009BB20B43D36010BD73B590F85B38032BE8
:10D4380005460C462AD100231D4E8DF807309DF86D
:10D44800073095F85C289A4201D802B070BD9DF863
:10D45800073006EBC3031B797BB184F0010373B17A
:10D468009DF8073056F83300F4F745FB9DF8073070
:10D478000133DBB28DF80730E1E72346EFE79DF88B
:10D48800073056F83300F4F731FBEFE7036CC06B55
:10D49800DB79DB0748BF81F0010424B102B0BDE8A5
:10D4A8007040F4F728BB02B0BDE87040F4F71EBB2B
:10D4B800346B002010B5A0F5066494F84D381BBBFA
:10D4C80094F84C288ABBD4E9091399421CD0591CFA
:10D4D800A069A162C35C2069DBB25B0043F40073FE
:10D4E800A4F850380A2384F84E38012384F84C38BD
:10D4F80094F85B38814228BFA262012B01D0042B2B
:10D5080002D1206CFFF76CFF94F84838002B6FD1DC
:10D5180094F849380133DBB2092B84F8493827D10C
:10D528002046BDE81040FBF715B994F94E387BB199
:10D53800B4F850184B08A4F8503801F001012046FF
:10D54800FFF772FF94F84E38013B84F84E38DBE75A
:10D5580084F84C38D4E909239A42D5D194F85B3839
:10D56800012B01D0042BCFD1206CFFF74AFFCBE76A
:10D578000A2B3DD194F84B382BB9B4F8523843F004
:10D588000103A4F852382379D9070AD5B4F8520808
:10D59800820501D4C30718D4B4F858380133A4F865
:10D5A8005838012284F8482894F84B280023012A87
:10D5B80084F849381CD1617984F84B38206C01F023
:10D5C8000101BDE8104025F06DBCE36AC0F34700D7
:10D5D80013B1216B9847E4E7E3696269D054E369C2
:10D5E800E1680133B3FBF1F201FB1233E361D8E7E1
:10D5F80010BDF0B56C4C277895B0002F40F0C68070
:10D6080094F8246D002E00F0C180304607F0D6F95A
:10D618000546002800F0BA800368E362C368A36285
:10D62800002B00F0B3803046F3F792FEC4F8280DC3
:10D6380010B129238371C7712A7A2E21F3F74EFF7F
:10D64800E06A07F051F921F0A9FFE06A038823F0A6
:10D6580001031B041B0C03801E23E3810F230026F8
:10D66800A38101A92D230127CDE90173039622F097
:10D6780063F96023CDE90436CDE906660896EB79AF
:10D68800990740F18580DB00042203F00803ADF818
:10D698001620ADF81E300023069304AA6979E06AC3
:10D6A80006F061FB08226979E06A06F037FBE36A55
:10D6B800A06A5A6C42F400425A641A8842F0800206
:10D6C8001A80EA79697912F0020F14BF0422012244
:10D6D8008A40196A21EA02011962196A0A431A6220
:10D6E8001A8842F001021A80FAF7F2F8002229217A
:10D6F800FAF7A2F9A06AFAF7EBF860222B4900239F
:10D70800FAF70CF9A06A0DF01BFEA06A036823F073
:10D7180001031B041B0C03600DF012FE09A80DF099
:10D72800E1FDE36A6A79A06A343313440993182344
:10D738000026ADF830308023CDE90D631C4B0A93E9
:10D7480010230B934FF40073CDE90F364FF40053B9
:10D75800CDE9123609A9202311930DF0D1FD6A797C
:10D76800E36A0C2A9CBF134931F81260DA68164341
:10D77800A26ADE60136843F00203136001200023ED
:10D7880023816381FBF702F80123237015B0F0BDF4
:10D798005B004FF4807203F00203ADF81470ADF82B
:10D7A8002020ADF81C3076E700100020230D00087B
:10D7B80010100020C0890308F8B5444C23780BB139
:10D7C800637803B1F8BD94F8306005460C2014F076
:10D7D80055FE002E3DD000283ED1FFF70AFF012359
:10D7E80084F8303094F83760012EEBD80B2014F011
:10D7F80045FE002837D0364A364B126894F83E600A
:10D80800A3FB02131B09FA2101FB13237D2B28BF5D
:10D818000026314F3B78B34203D1D4F82C3D9D42CA
:10D82800D0D32E4B53F82600A06094F83600FAF7B0
:10D83800ADFF07EE905A9FED2A7A3E70F8EE677AB0
:10D8480077EE877AFCEEE77A17EE903AC4F82C3D2B
:10D85800F8BD0028C1D0F8BDFBF74AF894F830307D
:10D86800002BBFD1F8BD1F4BDB78002BC3D1012E95
:10D8780013D194F83D309BB11B4B1B7813F0010377
:10D888000ED11E4694F83430002BC2D0174B1B78AB
:10D89800002BBED094F83E60BBE794F83860F1E7FF
:10D8A8000B4A618F94F83C301068114EB0FBF1F2CE
:10D8B80001FB03F301FB1202A6FB0313B2EB531F98
:10D8C80094F8396028BF0026DCE700BF001000206C
:10D8D800A44E0020D34D62102C000020B06A03082B
:10D8E8000024744984290020FF280020212B0020CF
:10D8F8001F85EB5110B51C4C94F88C3063B31B4A50
:10D90800136843F480331360FFF773FE012384F830
:10D91800303094F88D30012B98BF84F8373094F864
:10D928008E3084F8383094F88F3084F83930B4F871
:10D938009030638794F8923084F83C3094F89330B0
:10D9480084F83D3094F8943084F8343094F8953065
:10D9580084F83E30002010BDFAF7CAFF4FF480303B
:10D96800F5F7C6FDD5E700BF00100020B85B002022
:10D97800F8B55A4C94F90020002A63D0584B93F814
:10D98800401009B983F84020B3F86C1019B9E18840
:10D9980009B1A3F86C105349088810B9A08800B1E0
:10D9A8000880022AE17805D111F0080218BF012287
:10D9B80083F844294C4B4D4A1B784D4DD35C85F870
:10D9C8004C304C4B4C4E1B783068002B3FD194F9AF
:10D9D8000130082293FBF2F20132002833D0476964
:10D9E800BA5C85F84E2080B35A4202F0070203F071
:10D9F800070358BF53420133026952F823301B789A
:10DA080085F84F3001F00A030A2B3C4F26D1E288F3
:10DA18003B493846F9F7F0F9202385F85530E37883
:10DA28009A073AD513F0040F0CBF4F23492385F802
:10DA380057305223502285F85830002385F8562055
:10DA480085F85930F8BD3F22CBE72E4BD7E7552351
:10DA580085F84E30462385F84F30D3E7C90705D5FA
:10DA6800A28827493846F9F7C7F9D5E794F901108C
:10DA780030684B4203F0070301F0070258BF5A42CF
:10DA88000132082391FBF3F10131FFF7F7FA1C4942
:10DA980002463846F9F7B0F9BEE794F9002094F940
:10DAA8000230022A07D0272B11DC182B11DC0F2B90
:10DAB800D4BF0023012332686AB10133D26952F816
:10DAC800232011491148BDE8F840F9F795B9032317
:10DAD800F1E70223EFE70B4AF3E700BFA00B0020B2
:10DAE80000100020E82A0020E02A00208FBA03084E
:10DAF8002C000020E12A0020AC2900207D00002015
:10DB080052BA03088DBA03089891030882000020CE
:10DB180008B50F4B9B78022B08D0032B09D10D4B6E
:10DB2800D3F80403003018BF012008BD0CF084FEB0
:10DB380008B9002008BD0CF075FE0028F9D0064B86
:10DB48005878A0F10300B0FA80F0400908BD00BF82
:10DB58003C2A002000100020BC6D002070B5144B3A
:10DB68009B78022B05460ED001780446E9B1114E88
:10DB7800D6F80403F3F730FA15F8011F0029F7D196
:10DB88002C1B204670BD26F0CFFB0B4B04461868B3
:10DB9800037E13F0060FF4D090F82830002BF0D154
:10DBA8002946224625F0BCFDEBE70C46204670BD11
:10DBB8003C2A002000100020442A002010B51A4BEF
:10DBC8009B78022B82B007D0184B0146D3F8040388
:10DBD800F3F702FA02B010BD154B8DF807001B6869
:10DBE80093F91A104A1C0FD05A6840F2FF14C2F376
:10DBF8000802A24208D002EB41220E4950545A684A
:10DC080001325A6002B010BD1A7E12F0060FE1D040
:10DC180093F82820002ADDD1184601220DF10701CA
:10DC280025F07EFDD6E700BF3C2A0020001000202A
:10DC3800442A0020D46D00202DE9F04100F11002A3
:10DC48000746002452F8043DA40003F10801E4B299
:10DC58002BB10F2903F180033BD844F0010497420C
:10DC6800F0D12046FFF7AAFF00252E46A84604F06B
:10DC78000303022B24D0032B14D0012B09D0013528
:10DC8800042D4FEA9404F2D1B8F1000F4AD1BDE84F
:10DC9800F08157F82500B8F1000F3BD10001C6B25A
:10DCA8009846ECE757F82500B8F1000F18D1C0F3F3
:10DCB8000720FFF783FF17F82500FFF77FFFDEE750
:10DCC80057F82500B8F1000F1AD1C0B2FFF776FF58
:10DCD800D5E7FF2B94BF44F0020444F00304BEE7E9
:10DCE800C0F303303043FFF769FF57F82500C0F34E
:10DCF8000710FFF763FF57F825603601F6B2BEE755
:10DD0800C0F303103043FFF759FF57F82560360179
:10DD1800F6B2B4E700F00F003043FFF74FFF4FF0C3
:10DD28000008ACE73046BDE8F04147E7F8B5061F04
:10DD38000446324600F10807002152F8043F03F177
:10DD480020003F2803F1080503F102033DD80F2DF9
:10DD580018D8032B02D9002908BF01219742ECD11A
:10DD6800012921D002290FD1206800F03F0040F09E
:10DD78008000FFF723FF2079FFF720FF207ABDE816
:10DD8800F8401BE70221E9E7D4E90030A2681B014B
:10DD9800800000F00C0003F03003034302F003009E
:10DDA8001843BDE8F84009E7206800F00F0040F08C
:10DDB8004000FFF703FFD4E9013000F00F0040EA0C
:10DDC8000310C0B2BDE8F840F8E604F10C020025E3
:10DDD80052F8043D03F18001FF2903F500404FEAA2
:10DDE800850506D9B0F5803F03F500031BD245F041
:10DDF8000105A242ECD165F03F00C0B2FFF7DEFE9C
:10DE080056F8043F05F00302022ADBB227D0032AA2
:10DE1800184616D0012A0ED0FFF7D0FEB7424FEAB7
:10DE2800A505EDD1F8BDB3F1807F34BF45F00205FB
:10DE380045F00305DDE7FFF7C1FE7078FFF7BEFE8A
:10DE4800ECE7FFF7BBFE7078FFF7B8FEB6F9020003
:10DE5800C0B2FFF7B3FE96F90300C0B2DCE718467C
:10DE6800FFF7ACFE7078FFF7A9FEB6F90200C0B262
:10DE7800FFF7A4FED2E700BF0EB470B583B007ACBD
:10DE88000646482054F8045BFFF798FE2020FFF769
:10DE980095FE3046FFF762FE3A20FFF78FFE2A46CE
:10DEA80023460A4901940020F6F792F804460A200E
:10DEB800FFF784FE064AD2F8003303341B1BC2F86E
:10DEC800003303B0BDE8704003B07047DDDE0008E2
:10DED80000100020084671E62DE9F04F5C4DD5F89A
:10DEE800344D85B0904600290CBF04220622661CDA
:10DEF800DDF838900F9F009260D0A1453BDDA3EB81
:10DF0800080A57B1109BDA1B04FB02F20123B95C23
:10DF1800D5F8D82B8B40134226D0D5F8306D04FBAA
:10DF28000AF408EB040B96BB58F8040026F0FCF939
:10DF3800411D0846FAF7B6FF78BBD5F8000395F8F7
:10DF4800382D401AC5F8000392BB012285F8382DF8
:10DF58003EBB58F80400FFF701FE9BF904104B1C68
:10DF680002D03C48FEF7A4F8D5F8344D01344C45AE
:10DF7800C5F8344DC5DBA14553D0D5F8300D009B0D
:10DF8800834294BF0020012005B0BDE8F08F032133
:10DF98000846FAF787FF0028CFD0012005B0BDE872
:10DFA800F08FB3442C489BF80410FEF781F8DBE7A8
:10DFB8002C20FFF703FED5F8306DC9E7D5F830AD52
:10DFC800924503D3002005B0BDE8F08F234A02EB49
:10DFD8008A020646D2F8102301921046CDE90213B0
:10DFE80026F0A2F90B30FAF75DFFDDE901210446BE
:10DFF800039B0028D1D1BAF1030F98BF31461848C6
:10E008000193FEF755F8D5F80013D5F8342D85F8A7
:10E01800384D091A541CC5F80013C5F8344D019B36
:10E028006BE70120FAF73EFF0028A6D1D5F80033A8
:10E038000A20013BC5F80033FFF7C0FDD5F8300DC5
:10E048004FF0FF330130C5F8300DC5F8343D96E781
:10E0580000100020A4BA0308ACBA0308B06A030889
:10E0680094BA03087F2810B5044607D964F07F00E6
:10E07800C0B2E409FFF7A2FD7F2CF7D8E0B2BDE8F3
:10E0880010409BE538B5044600EB410534F9023BE6
:10E09800D81780EA4300FFF7E5FFA542F6D138BD5F
:10E0A800C31783EA4000DDE7F8B50F4BD3F8205AD1
:10E0B800D3F8244AD3F8286AA9B1831E00EB410794
:10E0C80027441E4404441D4434F9022B36F9023F08
:10E0D80035F9020F134403EBD373A0EB6300FFF78A
:10E0E800DFFFA742F0D1F8BD00100020F0B52B4C9F
:10E0F8002B4DD4F80873D4F83C6D2A48D4F8EC3B7F
:10E1080094F8392D94F84C152D7890F82000B742E2
:10E1180085B027DB84F8445DC4F8403D84F8450D9C
:10E1280084F8461D84F8472D01AD5320FFF746FDBE
:10E13800D4F8400DFFF796FF94F8440DFFF792FFCF
:10E1480094F8451D94F8462D94F8473D03932846C6
:10E15800CDE90112FFF7EAFD0023C4F808330120D6
:10E1680005B0F0BDD4F8406D8DF80850B3428DF875
:10E178000B2001938DF809008DF80A1001AD04F504
:10E18800546204D095E8030082E80300CDE769688B
:10E1980053689942F6D10020E2E700BF0010002042
:10E1A80000290020842900201E4BD3F8081A0022D9
:10E1B8001F29C3F80C23A3F81023A3F81423A3F8EA
:10E1C8001623C3F8082324D03F291DD04FF4FA4260
:10E1D800B2FBF1F1A3F812131348B3F91223018823
:10E1E80029B1914201DD1F2A18DC92FBF1F1A3F855
:10E1F8001813817800314FEA022218BF012183F8F1
:10E20800F012C3F83C2D70474FF40072A3F81223A4
:10E21800E2E74FF48062A3F81223DDE70121A3F8B7
:10E228001813E6E7001000203C2A0020F0B585B05E
:10E23800FEF7C4F8054618B1CA4B1868FCF756FB38
:10E24800C94C94F87C3D94F8811D84F8711D04F63E
:10E2580048560022022BF26000F0BF80032B00F02A
:10E26800AC80012B3DD0C14B1A785E79012A00F0B1
:10E278008980022A32D15978013949B2481C2DD0F7
:10E2880002292BDC0901BA48415839B3987884F837
:10E298008C2DC4F8901DF3F75BF8C4F8940D7AE060
:10E2A80094F8912D1AB976221F4684F8912D94F985
:10E2B800900D431C09D0022807DCAE4B009394F85C
:10E2C800911D0123D022F9F7EBFD94F8BC3D582BA2
:10E2D80000F0058117B1002384F8913D284605B068
:10E2E800F0BD94F87D2D94F87E1D84F8643D531E8E
:10E2F80084F8683D84F8691D94F87B3D0022062B5C
:10E3080084F8702DAFD8012202FA03F313F05D0FE1
:10E31800A9D094F8643D934204BF94F87E3D84F8F4
:10E32800693D954B93F85820062A00F04A8194F8E5
:10E33800643D0022012B8DF80F2000F0EF80032BA5
:10E3480000F03A8101220B218C48F9F781FA042068
:10E3580008F0D0FD01230DF10F0200218748F9F7DD
:10E36800B8FE18B19DF80F30482B51D094F8643D91
:10E37800032B7FF478AF10223721D4F8680DF9F712
:10E388003FFA70E7D978187984F88C2D4B1E84F8F9
:10E39800903D84F8910D062E09D80123B34013F05F
:10E3A80042079BD113F03D0F71D1012E96D0744ACC
:10E3B800136843F00403136090E76F4A92F858100B
:10E3C80006297FF450AF103294F87E1DC4F8682DEA
:10E3D80084F8643D84F86C1D8EE794F87F2D013A2B
:10E3E80052B2571C3FF43FAF022A3FF73CAF12012D
:10E3F8005F498A58002A3FF436AF94F8800D84F8B4
:10E40800643DC4F8682DF2F7A3FFC4F86C0D73E7F8
:10E41800B4F9781D9FED5B6A594F642291FBF2F3C2
:10E4280002FB131212B207EE902AB8EEE77A07EE53
:10E43800903AF8EEE77A3B68534AC4F8582DE7EE6D
:10E44800067A012143F00803F2EE046A67EEA67A21
:10E458004E4A3B6008460823C4F85C2DC6ED037A93
:10E4680084F8703DF3F754FBD4F8583D4848984772
:10E4780000210120F3F74CFB94F87A3D012284F83F
:10E48800882D002B3FF4EFAE84F8703DEBE61420A6
:10E4980008F030FD94F88C3D012B3FF401AF022BBE
:10E4A8007FF413AFD4F8943D13B11A689B88138591
:10E4B800D021D4F8900DF3F7D8FC01232D4AD4F8D5
:10E4C800900D0021F3F7A0FCD4F8943D13B11A681D
:10E4D8009B88936194F8BC3D582B7FF4FFAE2D4A7E
:10E4E8002D4E1823A2F134008821F9F77DFD312241
:10E4F800F4212A48F3F758FE294B2A482A492B4A7F
:10E50800C4F8A03D2A4BC4F89C6DC4F8A40DC4F807
:10E51800A81DC4F8982DC4F8AC3D48E794F86C2DB4
:10E52800002A7FF40FAF0C22032B84F86C2D7FF4A4
:10E5380009AF204BD4F8680D46F2A811C3F87C1334
:10E5480012223721F9F75CF90D222421D4F8680D3D
:10E55800F9F756F930226A21D4F8680DF9F750F91D
:10E56800F0E600BFA85B002000100020A42F0020C8
:10E5780010290020BC1D0020F0540020641D00203C
:10E58800702900208988883C31810008A78100080B
:10E59800581D0020C01D0020A50A00088C1D002061
:10E5A800A70A00087D230008E10A00080000D859DE
:10E5B800BF0800082C00002094F86C2D002AB2D067
:10E5C800B7E71033032194F87E2DC4F8683D84F82A
:10E5D800641D84F86C2DAAE610B50C4C94F80B0653
:10E5E80021F046FF94F87C3D022B04D0084B1A78A2
:10E5F800022A05D010BD94F8800D21F039FFF5E707
:10E608009878BDE8104021F033BF00BF001000200B
:10E61800A42F002000B5ADF2946D68464FF4D26285
:10E62800064926F01CFD029B1BB168460DF15601F8
:10E6380098470DF2946D5DF804FB00BFF05400207C
:10E64800023990ED007AD0ED017AD0ED026A062900
:10E6580013D8DFE801F0424D56616A790400B1EE43
:10E66800676AF1EE666AF1EE477A80ED006AB0EE0D
:10E67800467AC0ED017AC0ED026A384B93F86C36E1
:10E6880053BB374B93ED036A93ED005AD3ED065A0B
:10E6980027EE866AA5EE076AA5EEA66A80ED006AEF
:10E6A80093ED046A93ED015AD3ED075A27EE866A73
:10E6B800A5EE076AA5EEA66A80ED016A93ED055AF4
:10E6C800D3ED025A93ED086A67EE857AE5EE877A0C
:10E6D800E6EE267AC0ED027A7047B1EE476AC0EDE1
:10E6E800007AB0EE677A80ED016AF0EE467AC4E708
:10E6F800B1EE477AF1EE677A80ED007AC0ED017AE3
:10E70800BBE7B1EE676A80ED017AF0EE477A80EDFB
:10E71800006AB0EE467AB0E7B1EE477AF1EE666A83
:10E7280080ED007AC0ED026AA7E7B0EE476AF1EE25
:10E73800666A80ED017AC0ED007AB0EE677AC0EDC6
:10E74800026AF0EE467A98E7F1EE677AF1EE666AC9
:10E75800C0ED017AC0ED026A8FE700BF2C000020EF
:10E76800DC1D00202DE9F843634C0546D4F85C3DD8
:10E7780004F5606104F658509847B4F9003E94F8DF
:10E78800701D06EE903AB4F9023E07EE103AB4F95D
:10E79800043E07EE903A04F64852F8EEE66AB8EE00
:10E7A800C77AF8EEE77A1046C2ED006A82ED017A80
:10E7B800C2ED027AFFF744FFDFF84CE19EF8000053
:10E7C800430777D4D4F8083E94F8881D19B3B4F9F0
:10E7D800821D92ED005A92ED016A92ED027A05EEE1
:10E7E800901AB4F9841D06EE901AB4F9861D07EE46
:10E7F800901AF8EEE55AF8EEE66AF8EEE77A75EE62
:10E80800655A76EE666A77EE677AC2ED005AC2ED0F
:10E81800016AC2ED027A002B4AD0384AED1A9542B5
:10E8280018D9374A002302F10800A2F18A01951D80
:10E83800C4F8083E32F9023B30F9024B234403EB9B
:10E84800D3735B10AA4221F8023BF3D1BDE8F84329
:10E8580007F0D8BE0020F2F7C7FB2A4B03F1C2012C
:10E8680003F1CA0203F10C0031F9024FF3EC017A0B
:10E8780007EE104AB8EEC77AFDEEE76AF4EEC77AFB
:10E88800F1EE10FA44BF16EE904A0C8032F9024FAE
:10E8980007EE104AB8EEC77AFDEEE76AF4EEC77ADB
:10E8A800F1EE10FAC4BF16EE904A14808342DBD111
:10E8B800BDE8F883C4F8085E04F6825C114604F6E5
:10E8C8000C6704F6146604F654594FF00008F1EC8E
:10E8D800017A2CF8028BFDEEE77A494517EE903A5B
:10E8E8001BB227F8023B26F8023BF0D120F00400C7
:10E8F8008EF800002B4667E7001000207FC3C9018F
:10E908000C1E0020481D002000290020944B954A29
:10E91800996AB2F8F835A2F81036002900F00D818E
:10E9280007EE903AB8EE676A07EE901AF8EE677A43
:10E938009FED8D7A9FED8D0ADFED8D2A9FED8D3A43
:10E948009FED8D1ADFED8D1A9FED8D2A9FED8D5A63
:10E9580026EE276AF0EE400A26EE076A2DED028BB6
:10E96800FDEEC67A36EE000A17EE900AFDEEC07A82
:10E9780002F2146317EE901A2030203102F5D062AB
:10E98800F7EE004A402800F2A580B4EEE26AF1EE04
:10E9980010FA40F3DC80B0EE467ADFED7B5ADFED0B
:10E9A8007B6A01E0B0EE677AB4EEE67AF1EE10FA2F
:10E9B80077EE657AF6DCF4EEC37AF1EE10FA40F100
:10E9C800BD80DFED715ADFED726A01E0F0EE477A43
:10E9D800F4EEE67AF1EE10FA37EEA57AF6D4B4EE54
:10E9E800E07AF1EE10FA00F3A280DFED6A7AB4EE75
:10E9F800E77AF1EE10FA48BF33EE477A67EE077A06
:10EA0800B0EE614AA7EE814A4029F0EE423AE7EEBD
:10EA1800843A67EE275ADFED606AA5EEA37AB0EE76
:10EA2800644AF0EE647AA7EE264AE7EE667AC7EE05
:10EA3800843A55D8B4EEE06AF1EE10FA40F38A80D1
:10EA4800B0EE407ADFED505ADFED506A01E0B0EEEB
:10EA5800677AB4EEE67AF1EE10FA77EE657AF6DCCC
:10EA6800F4EEC37AF1EE10FA77D5DFED475ADFED11
:10EA7800486A01E0F0EE477AF4EEE67AF1EE10FA31
:10EA880037EEA57AF6D4B4EEE07AF1EE10FA51DC5E
:10EA9800DFED407AB4EEE77AF1EE10FA48BF33EED4
:10EAA800477A67EE077AF0EE616AE7EE816AF0EE80
:10EAB800428AE7EEA68A67EE275AB8EE008AA5EEE4
:10EAC800A87AF6EE006A74EEC75A27EE087A65EE61
:10EAD800A66A0BE0F7EE003A4029B0EE634AA9D9DE
:10EAE800B0EE457AF6EE006AF7EE005AC4EE847A84
:10EAF800243343ED053A67EEA66A67EEA55A27EE7A
:10EB0800877A43ED096A43ED076A43ED085A03ED36
:10EB1800067A03ED035A03ED045A03ED015A03ED97
:10EB2800025A9A427FF42EAFBDEC028B704732EE48
:10EB3800C77A63E732EEC77AB3E77047B0EE677A11
:10EB4800B4EEE07AF1EE10FA7FF74FAFEFE7F0EEB0
:10EB5800467A30E7F0EE407A82E7B0EE677A92E7DD
:10EB6800702B00200010002027D4D236DB0FC93FBD
:10EB7800DB0F4940DB0F49C092E741B99730083CA9
:10EB880015A82ABE00000000DB0FC940E4CB1641DF
:10EB9800E4CB16C1DB0FC9BFF304353F154B164A4A
:10EBA800197CB2F8A82393F92430DFED145A9FEDAD
:10EBB800146A07EE101A07EE903AF8EEC76A07EEE5
:10EBC800102AF8EEE77AB8EEC77A67EEA57A26EE4D
:10EBD800877A0C4BE7EE067A6422FCEEE77A17EEAA
:10EBE800901A88B202FB00F283FB02301044C0F393
:10EBF80047207047E82D0020001000200AD7234145
:10EC08000AD7233C03082080114B124A197C93F938
:10EC18002430DFED115A9FED116A07EE101A07EE46
:10EC2800903AB2F8A833F8EEC76A07EE103AF8EE51
:10EC3800E77AB8EEC77A67EEA57A26EE877AE7EE26
:10EC4800067AFCEEE77A17EE903A98B2704700BF62
:10EC5800E82D0020001000200AD723410AD7233CC2
:10EC68002DE9F84F4A4FDFF850A1D7F8206ADFF8AE
:10EC78004C91354606F1440845F8040B07F61C6428
:10EC880007F6485B94ED006AD4ED016A94ED027AC8
:10EC9800D4ED037ABAEC010ABDEEC66AFDEEE77A56
:10ECA800FDEEE66ABDEEC77AA5EC016AC5ED087A05
:10ECB800C5ED026A85ED057A26F076F9B9EC010A08
:10ECC80028F8020B26F070F9FBEC017AA8F804008A
:10ECD800FDEEE77A143417EE903AA8F83E302D4B43
:10ECE8009C42CFD11D4606F1340406F13C08B5EC30
:10ECF800010A26F059F924F8020B4445F7D1264DAC
:10ED080006F14208B5EC010A26F04EF924F8020B88
:10ED18004445F7D1214BDFED227A93ED000A20EE2E
:10ED2800270A26F041F91F4B1F4AA6F8420011781E
:10ED38001A885888A6F850209A88DB88A6F85200C6
:10ED4800A6F85420A6F8563071B106F15803174AB0
:10ED580003EB4101F2EC017AFDEEE77A17EE900A37
:10ED680023F8020B9942F5D1114A124B51885A687F
:10ED7800D7F8B03DA6F87810C6E91F23FFF744FF7F
:10ED8800B7F8823EA6F88A00A6F87230BDE8F88F78
:10ED980000100020581E0020681E0020741E00204D
:10EDA80000007A447427002051270020182A0020E8
:10EDB8005029002040290020AC5B00209C2B00201B
:10EDC8002DE9F043854CB4F810338DB00546002B7F
:10EDD80040F01281824B1B88002B00F0A38028464C
:10EDE800FFF73EFFD4F8205A49202E46FEF7E6FEEC
:10EDF800D4F80C03FFF736F956F8040BFFF732F98D
:10EE0800304624F08FFB05F1100024F08BFBD4F87A
:10EE1800D83BDE0300F19280D4F8D83B980300F188
:10EE28008480D4F8D83B590300F1D38005F1280039
:10EE380024F078FB032105F13400FFF723F9B5F935
:10EE48003A00FFF70FF9042105F13C00FFF71AF922
:10EE5800D4F8D83BDA0400F1AD809F0400F1A1801A
:10EE68005E0500F19380180500F1868019047ED4B0
:10EE7800032105F14400FFF705F9D4F8D83BDA027D
:10EE88006BD49F0263D4B5F9583007EE903A554BCE
:10EE9800F8EEE77A93ED007A77EEC77AFCEEE77A38
:10EEA80017EE900AFFF7DEF84F4B1B78012B0ED9AF
:10EEB80005F1580707EB430705F15A0636F9020B27
:10EEC800B5F95830C01AFFF7EBF8B742F6D1D4F8C5
:10EED800D83B9E051FD4D4F8201A444D444B454ACC
:10EEE800C4F8241A481B801003FB00F3013382FB8B
:10EEF8000302A2EBE37202EB42029B1A8C2202FB92
:10EF080003530122C4F8281AC4F8203A84F8F42BD1
:10EF18000DB0BDE8F083B5F97200A0F2DC50FFF740
:10EF2800BFF8D8E7FFF7E2F859E7286AFFF7B8F81B
:10EF3800D4F8D83B59037FF579AF4AE0E869FFF781
:10EF4800AFF8D4F8D83B98037FF56BAFEDE7042111
:10EF580005F15000FFF796F895E7032105F14A00FF
:10EF6800FFF790F8D4F8D83B9F028CD5EFE7B5F8B7
:10EF78008A00FFF777F87BE7D5F88000FFF790F86D
:10EF8800D4F8D83B19047FF573AFF0E705F1840096
:10EF98000321FFF777F8D4F8D83B18057FF566AF5B
:10EFA800EAE7E86FFFF77CF8D4F8D83B5E057FF511
:10EFB8005AAFEBE7B5F87830B4F8D00BC01AC0F305
:10EFC8000D00FFF74FF8D4F8D83B9F047FF548AF02
:10EFD800E7E7686AFFF764F828E700BF0010002039
:10EFE8003C2A0020142A0020512700202C1A002037
:10EFF8008BAFF88A56555555D4F8E46BD4F8E03BF6
:10F00800B34207D094F8F032C4F8E06B093B012B07
:10F0180040F24E81D4F8EC6BD4F8E87BBE4207D0BE
:10F0280094F8F032C4F8E86B093B012B40F23381C5
:10F03800B4F81633002B7FF46BAFA84B1B88002B5A
:10F048003FF466AFFFF752F82846FFF709FE502055
:10F05800D4F8205AD4F8246AFEF7B0FDD4F8203A40
:10F06800D4F8282AD4F8241A12681B6808681344AC
:10F07800A3EB4000FFF714F8321D291D04A823F064
:10F08800EDFD04A824F04EFA06F1100205F1100176
:10F0980004A823F0E3FD04A8FEF748FE10274FF06C
:10F0A8000108D4F8D83B08FA07F21A4240F0D58094
:10F0B8000137132FF5D106F1280205F1280104A81C
:10F0C80023F0CCFD04A824F02DFA04AFEC4605F19A
:10F0D800340306F1340005F13C0933F9021B30F919
:10F0E800028BB3F90620B0F906E0A1EB0801A2EB08
:10F0F8000E02994547F8041B4CF8042BEDD104A8DF
:10F10800FEF79AFD6846FEF797FDD4F8D82B12F45F
:10F11800805306D0B5F87830B6F878105B1A0493A7
:10F128000123900408D5E96FF76F0CA800EB830062
:10F13800C91B40F8201C0133510513D504A905F15A
:10F14800840006F1840C01EB830705F18A0830F985
:10F15800021B3CF902EB8045A1EB0E0147F8041BAA
:10F16800F5D1033302F40041120540F18180D5F84E
:10F178008020D6F880700CA800EB8300D21B40F8E2
:10F18800202C03F10108002977D1B8F1010F22D012
:10F1980004AB03EB8802002008F1FF3352F8041D8A
:10F1A8004000013BC0B209B140F001005F1CF5D13D
:10F1B800FEF704FD0DF10C09002701E0474510DAC0
:10F1C80059F8043F0137002BF8D0D81780EA4300DC
:10F1D800FEF748FFF2E7049BD81780EA4300FEF7E2
:10F1E80041FF03214420FEF75FFFD4F8D83BD90242
:10F1F8006DD49A0266D43A4B58201978FEF754FF1A
:10F20800D4F8D83B9B0506D5B5F97200B6F972302B
:10F21800C01AFEF745FFD4F8200A324D324B334A64
:10F22800411B891003FB01F3013382FB0312A2EB9C
:10F23800E37202EB42029B1A8C2202FB0353D4F8BE
:10F24800242AC4F8203A0123C4F8240AC4F8282A36
:10F2580084F8F43B0DB0BDE8F083BB00EA183344F2
:10F2680052F8240C53F8243CC01AFEF719FF1FE784
:10F2780021B9002BB5D0984687E74346B5F88A20D0
:10F28800B6F88A000CA901EB8301121A41F8202C68
:10F2980003F1010879E74520FEF790FC1E20FEF7F0
:10F2A8008DFC3046FEF7DEFE3846FEF7DBFEBFE695
:10F2B8004520FEF783FC0020FEF780FC3046FEF771
:10F2C800D1FEA7E604215020FEF7EEFE93E70321C6
:10F2D8004A20FEF7E9FED4F8D83B8AE73C2A00200A
:10F2E800512700202C1A00208BAFF88A5655555507
:10F2F8002DE9F047A34C94F8F032013B8AB005465B
:10F308000A2B16D8DFE813F03E0055000B00670003
:10F318001500150086009E0008012C015401FBF71A
:10F328001BFC994AD4F8343D126864339342C0F008
:10F33800E881964DAB78022B11D02B79012B00F088
:10F348008581022B08D194F8F032012B04D194F86E
:10F35800F53B002B00F0D2810AB0BDE8F0878C4B5A
:10F3680041F2D5529B5C002BE7D094F8F53B012283
:10F3780084F8F022002BEFD0002384F8F53B0AB084
:10F38800BDE8F087834B1B78DB07D2D524F0A6F8BD
:10F39800064648B1804F00257B599E4200F087867B
:10F3A800DC35B5F5257FF7D1784DFCF793FEAB78C2
:10F3B800C1E7764DAB78022B00F05D85724A126882
:10F3C800C4F8342D00230322C4F80033C4F8303DB8
:10F3D80084F8F022B1E7FBF7BFFB704A0292A2F172
:10F3E8000C03302101930091A2F10A035021163A2F
:10F3F8004920FEF771FD654D002840F072814FF0FD
:10F40800FF310722C4F8300DAB78C4F8341D84F8F6
:10F41800F02290E7FBF7A0FB614B5C4D0021052033
:10F428000090A3F10802CDE901115320FEF754FD25
:10F43800002840F056810822C4F8300DAB7884F8D3
:10F44800F02278E7FBF788FB564B93ED000A25F08E
:10F45800ABFD554B93ED000A054625F0A5FD014689
:10F468004020F9F71FFD00287FF463AF4F4AD4F816
:10F47800303D52784C2B00F20A86DFE813F0630225
:10F488009F029702900289028102790272026A023F
:10F4980026031E0316030E0339032E030603FF0279
:10F4A800F702EF02E702DC02D102C602BB02AB029E
:10F4B80062045204420437042B041F041304090491
:10F4C800FF03F603EC03E203D9035E0355034B0382
:10F4D800B704AD04A3049A04910487047B0472045E
:10F4E800DB04D204C904C104EC04E404F4044303B7
:10F4F8005B0253024A0241022D02ED01E501DD01E2
:10F50800D501CD01C501BD01B501AD01A5019D0123
:10F5180095018D0185017701132012F0AFFFD0B15D
:10F52800B4F81033BBB94520D4F80C63FEF746FB9A
:10F538000E20FEF743FB3046FEF794FD2846FEF703
:10F5480091FDD4F83C3DC4F8083328460A2384F8D2
:10F55800F032FFF735FC0D4DF9F7D0FCAB78EAE651
:10F5680094F8DC3B002B6DD0132012F087FF0028A5
:10F5780068D194F8F53B002B64D1092384F8F03264
:10F58800E9E700BF00100020A44E00203C2A00201C
:10F59800BC6D0020FF280020941600203E6E030852
:10F5A80070700308142A0020382A00205C290020E3
:10F5B800AD4DAB78022B32D1AC4E94F8F43B3768A2
:10F5C800002B40F0CB8037B33B7823B397F8283033
:10F5D800002B7FF4C4AEBB6387F83C3004233A7E2B
:10F5E80087F828307B6AC7E90B3312F0080303D089
:10F5F8009F4B41F2B4529B587B634FF00008C7F809
:10F608002480C7E90288384623F032FF0523C7F86B
:10F61800408087F828300022042332603375954AE9
:10F62800D4F8343D1268C833934203D3FCF7EEFC98
:10F63800002856D0AB78032B00F04385012284F8CC
:10F64800F02278E62846FFF7BBFB84E78A4B94F85C
:10F65800F0521B78DB0703D411F020FD002842D1BB
:10F66800844ED4F89C2E33689A4243D8012D3FF437
:10F6780073AE94F8F53B002B3FF46EAE0B2D0ED80D
:10F688000123AB4040F6030213EA02077FF474AE8D
:10F6980013F4C06F03D0093D012D40F2578533683C
:10F6A800C4F8343D0B2384F8F03265E6704B5A7881
:10F6B800032A7FF455AE41F2C4410122595C3275E8
:10F6C800002900F0658541F20851595C002900F0D5
:10F6D800258541F24C529A5C002A00F01E850023D1
:10F6E8003375AB7827E6634B1B6803F59C530833E7
:10F6F800C4F89C3E012D7FF42FAE28E6FCF748FEA7
:10F708002AE64020F9F7CEFB00287FF412AED4F8A1
:10F71800303D5A4D40260EE0FEF750FAD4F800234B
:10F72800D4F8303D013A0133013EC4F80023C4F84F
:10F73800303D00F0E5842B4493F828331846002B1D
:10F74800EAD1494DAB7800204FF0FF310422C4F8CC
:10F75800300DC4F8341D84F8F022ECE53846002159
:10F768000AF0B2F900287FF456AFBAE7444B45498E
:10F778001A6845483C4DFEF77FFBD4F8302DAB782E
:10F788000132C4F8302DD6E5404B3E491A7840483E
:10F79800354DFEF771FBF0E73E4B3A491A8A3E4871
:10F7A800314DFEF769FBE8E73A4B36491A883B4882
:10F7B8002D4DFEF761FBE0E7364B32499A78384821
:10F7C800294DFEF759FBD8E7324B2E491A793548AF
:10F7D800254DFEF751FBD0E7334B2A491A7A3348B7
:10F7E800214DFEF749FBC8E72F4B26491A7F3048C1
:10F7F8001D4DFEF741FBC0E72B4B22495A7E2D4891
:10F80800194DFEF739FBB8E7274B1E499A7E2A485F
:10F81800154DFEF731FBB0E7234B1A491A7E2748EE
:10F82800114DFEF729FBA8E794F8982E15492448AE
:10F838000D4DFEF721FBA0E794F87B2D11492148D7
:10F84800094DFEF719FB98E71F4B0E495A791F48D7
:10F85800054DFEF711FB90E794F8FA2509491C4875
:10F86800014DFEF709FB88E73C2A0020442A0020C6
:10F87800BC6D0020A44E0020FF280020B06A0308B9
:10F88800B85B0020ACBA030878BD030870270020D5
:10F8980070B30308A85D0020C4A003080CA10308E6
:10F8A800F8A00308E4A00308E82D0020789F0308C7
:10F8B8005CBD030840BD030824BD030810BD030850
:10F8C8009CA603080C9E0308A42F0020809E030812
:10F8D800789D03080000C842B4F8F8351FED037A94
:10F8E8009A499B489B4D07EE903AF8EEE77A67EE07
:10F8F800877AFDEEE77A17EE902AFEF7BDFA3CE725
:10F90800954A9649138A96489289924DFEF7B4FA19
:10F9180033E7914A9149D389924852898D4DFEF730
:10F92800ABFA2AE78C4B89491A898F48894DFEF72B
:10F93800A3FA22E7884B85499A7D8C48854DFEF7C6
:10F948009BFA1AE78A4A8B498B48824DFEF794FA4C
:10F9580013E78A4B7D495A8A89487E4DFEF78CFA0F
:10F968000BE77C4D79492A888648FEF785FA04E733
:10F97800B4F9182375498448764DFEF77DFAFCE6FC
:10F98800B4F9122371498148724DFEF775FAF4E60D
:10F998007F4A78497F486F4DFEF76EFAEDE67E4A5A
:10F9A80074497E486B4DFEF767FAE6E67C4B7D4A64
:10F9B8007D497E48674DFEF75FFADEE67C4A7D4B5F
:10F9C8007D497E48634DCDE900327D4B7D4AFEF787
:10F9D80053FAD2E61A2000FB02407B4990F84032E5
:10F9E80090F83F2290F8410200907848594DFEF770
:10F9F80043FAC2E61A2303FB02425449B2F84A22E8
:10FA08007348544DFEF738FAB7E61A2303FB02424F
:10FA18004E4992F848226F484E4DFEF72DFAACE653
:10FA28001A2303FB0242494992F83D226A48494D8C
:10FA3800FEF722FAA1E61A2303FB0242434992F891
:10FA48003C226648434DFEF717FA96E694F8882E4E
:10FA58003E4963483F4DFEF70FFA8EE63E4B3B4961
:10FA68005A7860483B4DFEF707FA86E65E4B374901
:10FA78001A685E48374DFEF7FFF97EE65C4B9B7AC5
:10FA8800012B00F07A83334D77E6B4F8D02B59492F
:10FA98005948304DFEF7F0F96FE6584B55491A8B27
:10FAA80057482C4DFEF7E8F967E68BB2AAB22B4906
:10FAB8005448284DFEF7E0F95FE64FF07E52524970
:10FAC8005248244DFEF7D8F957E62C4B1F499A8A1D
:10FAD8004F48204DFEF7D0F94FE645484D498388F9
:10FAE8004288008800904C481A4DFEF7C5F944E654
:10FAF800D4F8D83BDA0400F137830F23C4F8303D3B
:10FB0800144D3AE6144B1149DA884448114DFEF772
:10FB1800B3F932E6424B0D491B68424893F8272057
:10FB28000C4DFEF7A9F928E63D4B08491B683E48ED
:10FB3800DA88084DFEF7A0F91FE6394B03491B6820
:10FB48003A489A88034DFEF797F916E6ACBA0308C7
:10FB5800889D03083C2A0020805B0020D8BB03084E
:10FB6800FCBC0308ECBC0308409C03082C9C03085D
:10FB7800C0BA030898910308CCBA0308A85D00200E
:10FB8800ACBB0308A4BB030898BB03088CBB0308E1
:10FB9800A42E002080BB030854BB03086CBB0308D9
:10FBA80024BB030830BB03083CBB030844BB030861
:10FBB80014BB03087D900308F0BA030800BB0308D0
:10FBC800DCBA0308E4BA030838BC030844BC0308D9
:10FBD800C8A50308BCA5030830A5030828A5030881
:10FBE800DCA60308F89B0308A85B00202CBC0308CC
:10FBF8001C280020ECBB030814BC0308702B002051
:10FC0800F0BB0308E0BB0308C4BB0308CCBB030874
:10FC1800B8BB0308F8BB030804BC03081C9C030812
:10FC28005829002020A90308BCA70308ACA703088B
:10FC38009B4B9C491B689C481A889C4DFEF71CF9F5
:10FC48009BE5974B97491B689948B3F84C20974D0B
:10FC5800FEF712F991E5924B92491B68954893F883
:10FC68006020924DFEF708F987E58D4B8D491B689A
:10FC780091485A888D4DFEF7FFF87EE5884B8949F3
:10FC88001B688E4893F82620884DFEF7F5F874E532
:10FC9800834B84491B688A4893F82020834DFEF7DC
:10FCA800EBF86AE57E4B87491D688748EB7EAA7E9C
:10FCB8002D7F0095FEF7E0F87C4D5EE5784B814995
:10FCC8001D6882486B7D2A7DAD7D0095FEF7D4F8CE
:10FCD800764D52E5724B7B491D687D48EB7BAA7BCC
:10FCE8002D7C0095FEF7C8F8704D46E56C4B7549BC
:10FCF8001D6878486B7A2A7AAD7A0095FEF7BCF8C9
:10FD0800C1E61A2000FB02406E49B0F85032B0F844
:10FD18004E22B0F8520200906F48644DFEF7ACF8DE
:10FD28002BE51A2000FB0240664990F8463290F80D
:10FD3800452290F84702009068485C4DFEF79CF811
:10FD48001BE51A2000FB02405E4990F8433290F808
:10FD5800422290F8440200906148544DFEF78CF816
:10FD68000BE54F4B4F491B685E48DA8E4F4DFEF747
:10FD780083F802E54A4B53491D685B486B8AAA8998
:10FD88002D8B0095FEF778F8484DF6E4444B45492D
:10FD98001B68564893F84720444DFEF76DF8ECE48D
:10FDA8003F4B40491B6852489A8E404DFEF764F815
:10FDB800E3E43B4B3B491B684E485A8E3B4DFEF7EC
:10FDC8005BF8DAE4364B37491B684B4893F8302028
:10FDD800364DFEF751F8D0E4314B32491B6847489D
:10FDE80093F82C20314DFEF747F8C6E42C4B2D49EB
:10FDF8001B68434893F846202C4DFEF73DF8BCE4B9
:10FE080094F8902E27493F48284DFEF735F8B4E47A
:10FE1800234B24491B683C485A8D244DFEF72CF887
:10FE2800ABE41F4B1F491B6838481A8D1F4DFEF75E
:10FE380023F8A2E41A4B1B491B6835481A8F1B4D3F
:10FE4800FEF71AF899E4334B16499A783248174D59
:10FE5800FEF712F891E494F8912E12492F48134DA9
:10FE6800FEF70AF889E42B4B0E495A7D2C480F4DB2
:10FE7800FEF702F881E42B4E337D052B3FF66FAA7F
:10FE880001A252F823F000BFB5F6000867F3000896
:10FE980031FF0008030001083500010899FF000838
:10FEA80058290020ACBA030860A903083C2A00209E
:10FEB80098A70308B0BC030870A703089CBC0308F4
:10FEC80094BC030838BC030888BC030880BC03083A
:10FED80074BC03086CBC030860BC030858BC030866
:10FEE80050BC03084CA80308D8BC030834A803086E
:10FEF80020A8030808A80308F4A70308C4BC03083B
:10FF0800D0A70308B8A603084CA903083CA903080E
:10FF18005CA80308805B0020E49B0308B4A60308E0
:10FF2800089C0308442A0020DFF89C92DFF89C8292
:10FF3800DFF89CA2706805AA49460AF097F90128DB
:10FF480041464FF003027FF4CCAB059F384677B3A8
:10FF58003B7863B325F0D3F8032251460028E9D152
:10FF680007F1080025F0CBF803460028E2D157F83E
:10FF7800030F06903A798DF81C2006A88DF81D30DD
:10FF8800F3F7BCFD3369984238BF18463061D1E7B2
:10FF9800804A814B1268C4F8342D03210022C4F82A
:10FFA8000023C4F8302D84F8F012FFF7D9B971682E
:10FFB80091F91A20571C0AD0774B02F5A17203EB6E
:10FFC8000213FF20DA796FF30002DA71887691F96B
:10FFD8001B20501C0FD0704B02F5A17203EB0213CB
:10FFE800FF27DA79C2F34500013820EAE07060F3B0
:08FFF8004602DA71CF76032303
:020000040801F1
:10000000337568480378002B7FF46FAB7768002F57
:1000100000F0978097F82830002B7FF466AB2838E3
:100020004422394625F01FF83846002109F050FDDA
:10003000002373605C4B3769DFF8A0E10FCB0DF153
:10004000180CACE807000DF11F018CF800307B1C88
:100050000DF11A07AEFB0302D20802EB8200A3EBFC
:100060004003303301F801398F421346F2D14C4B33
:1000700041F2C4410122595C3275002968D041F235
:100080000851595C81B341F24C529A5C5AB3042333
:100090003375FFF72ABBFBF7BDFF444D00283FF443
:1000A00024ABD4F83C2DC4F808230A22AB7884F89A
:1000B000F022FFF744B9304602F0AAFCDC2200210E
:1000C000781924F0F4FFFFF76FB9D4F8040302F0B5
:1000D0009FFC94F8043A0022022BC4F804231DD09C
:1000E000AB78FFF7AFBA022202EB021203EB8203F6
:1000F00003F5A6502E4B009306A93C232022043082
:100100000DF094FFFFF7F1BA2B44284D93F8282304
:10011000AB78002A7FF413A9FFF718BB1BF072FE1F
:10012000DEE70222442101FB023303F5A650214BF6
:10013000009310221323204904300DF077FFFFF7BE
:10014000D4BA09F023F900283FF4CFAA77686BE707
:100150000A46C9E74520FDF735FDFF20FDF732FDD2
:100160001648FDF7FFFC3846FDF72CFDFFF79BBA5C
:1001700094F87420124913480C4DFDF781FEFFF7E7
:1001800000BBB4F97830B4F97A200F490F48074D15
:10019000FDF776FEFFF7F5BA0A46C3E7A44E002046
:1001A000BC6D0020BC83002090BD03083C2A0020C9
:1001B000E98E0008F1BF0008B0BA030884BD030847
:1001C000ECBB030864A30308D8BB03081CBC0308EA
:1001D0004C2A0020B8BA0308BCBA0308CDCCCCCC5A
:1001E0002DE9F84388460178A9B10C4E04468146B2
:1001F000354606F10807284624F070FF38B1B842AA
:10020000A0EB06003CBFA9EB040308F8003019F886
:10021000011F0029EFD1BDE8F88300BF90700308EB
:100220002B4B1B6842F201021A4200D17047294B46
:100230005B68C3F3080370B4CBB9EFF31183B3B9B0
:10024000254A264D264C1368A06811688B42FAD1C6
:1002500029688842F7D823490D684FF47A7404FB63
:1002600005F1081AB0FBF5F004FB030321E0EFF3FE
:100270001180102383F3128803F1E0231A499D684B
:100280001A68D20344BF01220A60134A48BF9D681E
:1002900016680B68C0B280F3118812490C684FF4DD
:1002A0007A70334400FB04F1491BB1FBF4F100FB0D
:1002B00003130E480E49126882600124022280F85E
:1002C000214081F8A42EC1F8A03E70BC704700BF49
:1002D000B85B002000ED00E0A44E00203C5300205D
:1002E00010E000E03853002034530020842900201F
:1002F000001000202C4B1B6842F201021A4200D170
:1003000070472A4B5B68C3F3080330B4CBB9EFF3F3
:100310001183B3B9264A274D274C1368A06811688A
:100320008B42FAD129688842F7D8244A14684FF4DE
:100330007A7101FB04F2101AB0FBF4F001FB030325
:1003400021E0EFF31181102383F3128803F1E023FE
:10035000C9B29C681A6812F4803F194A1EBF012076
:1003600010609C68124B1D68136881F31188134A52
:1003700010684FF47A712B4401FB00F2121BB2FBA0
:10038000F0F201FB03230F490F488A68022403F5AA
:10039000B71303F5587302F2DC5280F8A44EC0F88C
:1003A000A03E8A6030BC7047B85B002000ED00E0E2
:1003B000A44E00203C53002010E000E03853002001
:1003C0003453002084290020001000202DE9F0473C
:1003D000C34DC44CC449688AC44AC54BC54FC64EB8
:1003E000C4F87415DFF84CE3C4F84835002184F8EC
:1003F000A51E84B00FFA80F9C4F86C75C4F8706556
:1004000004F6A46102F1240CDEF8003022F8029F09
:1004100003F59673944541F8043FF5D1DFF818834E
:10042000DFF818C3D8F800E0B44B1EF4805F08BFB3
:10043000B5F91E90ACF8069003F178010AE01FFAB6
:1004400089F293F8019009F104092CF81920063378
:100450008B421AD01A78002AF9D193F802A0DA78E0
:100460009245F4D20AF1FF3909EB890909EB8909B0
:1004700009F561790132BAF1000FE0D102EB820295
:1004800002EB820202F56172DBE71EF0080F2CD14D
:1004900042F201031EEA030F18D11EF4004F11D1DE
:1004A000EB7B13B1022384F8823395F8222094F871
:1004B0006815131D8B42A8BF0B4684F8D43F04B0C7
:1004C000BDE8F087012384F88233EEE744F6206329
:1004D0001EF4005FA4F86A3500F08B800822884B78
:1004E00084F86825C4F86C35D7E72B7A0C2B79D8BB
:1004F000DFE813F08A008A0028018B017800780079
:100500007800BF017800F8018A0078000D0003012F
:100510000A2293FBF2F3A3F5B0639BB2002263F3CC
:100520000F0263F31F4277497748C4F8B02F1223B4
:10053000C4F8B42FC4F8B82FC4F8BC2FC4F8C02F27
:10054000C4F8C42FC4F8C82FC4F8CC2FC4F8D02FD7
:10055000C4F87815C4F86C0542F6F8216B4A84F8A3
:10056000683540206A4BA4F86A15C4F87025C4F8B1
:10057000743502F0D5FB002834D0AB7A697A90F953
:100580000200644A002B0CBF00230823002918BF77
:1005900043F001034FF0030C4FF4E131CDE901C307
:1005A00000910023402102F049FAC4F8000A78B112
:1005B000DFF88C9199F80030002B00F013820023B3
:1005C00094F8822384F8B03312B9032384F8823379
:1005D000D4F8003A003318BF0123D8F800E0002B0C
:1005E0007FF456AFD8F800E0C4F86C75C4F87065B5
:1005F0004EE71EF0010F3FF450AF0C22464B84F83B
:100600006825C4F86C3548E7444BC4F8AC34402046
:1006100002F086FB81460028E4D04FF0000A84F8FF
:10062000A0A40DF09BFB2A7A012A03460FD0C0F04C
:10063000EA810A2A1BD1D8F8002012F480621CBF7C
:1006400080F00102D2B202F0010284F8A024032259
:10065000072184F8A824012284F8B11484F88C249A
:100660000C2142F6F82284F86815A4F86A25697A04
:100670002B4A2C48C4F86C2500312B4AC4F8742549
:10068000C4F8700518BF01214AB299F9020094F824
:10069000A0C4002B40F08481BCF1000F00F0AC81BD
:1006A000032342F008024FF4E131CDE90132009119
:1006B00000231E4A402102F0C1F91D4B1860EB7B5C
:1006C00094F86825013BDBB29A4284F8B03402D832
:1006D000002384F8B034031C18BF01237DE700BF5A
:1006E000E82D002000100020B9A200083E2B0020B9
:1006F000A0860100B1A20008B5A20008F01E0020EB
:100700001DA30008B01F0020759C0008F58F00088D
:10071000F9C90008359400080DA3000868150020E9
:100720001998000849980008C1970008859B00089F
:10073000A02E0020A44E0020B85B0020402B0020FB
:10074000212E002002010A2392FBF3F2A2F5B062EF
:1007500092B2002362F30F0362F31F43CA48C4F846
:100760007815C4F8683F1221C4F86C3FC4F8703F94
:10077000C4F8743FC4F8783FC4F87C3FC4F8803FA5
:10078000C4F8843FC4F8883F42F6F822C4F86C05E8
:10079000BE4BDFF84493C4F87C95402084F868157C
:1007A000A4F86A25C4F8703502F0BAFA8246002827
:1007B0003FF418AF0DF0D2FA6A7AA97A9AF902C01A
:1007C00000280CBF01230323002A14BF062207229E
:1007D00000290CBF002108210A43AD490193029270
:1007E0004B4600918146AB4A6046402102F026F913
:1007F00095F8233013B1052384F88233B9F1000F43
:100800003FF469AFA44B186065E7122342F6F82164
:10081000A24A84F868354020A14BA4F86A15C4F8B0
:100820006C25C4F8703502F07BFA814600283FF44D
:10083000D9AE0DF093FA697A99F902C0AB7A00311A
:1008400018BF01214AB2002840F09B80002B00F025
:100850000E8142F008024FF0010E4FF4E131029296
:100860000346CDE9001E60468E4A402102F0E6F8BC
:1008700031E70E234FF0000944F620618A4A84F8DC
:1008800068354020894B84F8EC95A4F86A15C4F8C3
:100890006C25C4F8703502F043FA00283FF4A2AE8C
:1008A00001886B7A90F90200B3EB090201F48251DE
:1008B00018BF0122B1F5825F00F0B580AB7A84F8F1
:1008C000F595002B0CBF00230823012113434FF49F
:1008D000E132CDE9011300920023754A402102F074
:1008E000ADF8F8E603010A22102093FBF2F3A3F51A
:1008F000B06341F60B21C4F8BC34C4F8C034C4F86A
:10090000C434C4F8C834C4F8CC34C4F8D034C4F8FF
:10091000D434C4F8D834C4F8DC34C4F8E034C4F8AF
:10092000E434C4F8E834C4F8EC34C4F8F034C4F85F
:10093000F434C4F8F8345F4A84F868055E4BA4F8D0
:100940006A154020C4F86C25C4F8703502F0E8F947
:1009500000283FF447AE6B7A584A90F902000092A3
:10096000003318BF01230322CDE9012340210023D6
:10097000534A02F063F8534A031C18BF0123106066
:100980002BE6002B64D14FF0030E4FF4E1320291BD
:10099000CDE9002E6046434A402102F04FF831E78E
:1009A000BCF1000F11D042F008020321CDE9011281
:1009B0004FF4E13300930023434A402102F03EF814
:1009C000424B1860344B186079E6AB7A83B342F03F
:1009D00008024FF0030E4FF4E13102926346CDE975
:1009E000001EE9E73A4B3B4A1A600DF0F1F802238A
:1009F00089F800300123E3E595F80AC0BCF1000F47
:100A00001ED001234DE60221032284F8A81484F8A5
:100A1000B124072145F2F05284F88CA484F86815BB
:100A2000A4F86A2523E684F8F595032108234DE709
:100A30004FF0030C4FF4E132CDE901C10092BBE766
:100A40004FF0010C4FF4E132CDE901C1009230E6E4
:100A500042F0080203214FF4E133CDE90031029264
:100A6000604600230F4A402101F0E8FFCAE64FF03C
:100A7000010E4FF4E1320291CDE9002E6046094AA1
:100A8000402101F0DBFF26E6759C0008899C0008E8
:100A9000A0860100059E00081C2E0020A1950008DC
:100AA000B595000835960008BDA200082DA30008E2
:100AB000A9A60008159F00084D9F0008A068060021
:100AC000C5AC0008282E0020859B0008A02E002021
:100AD0000C29002051C000088C1F002037B50546A6
:100AE000084614460EF01EFC78B10123022101A82D
:100AF0008DF805308DF804500EF0DBFB20460EF02B
:100B0000C7FBA0F130035842584103B030BD70B567
:100B100040F2014444EA800404F086FD0C4E054690
:100B200096F8F83F06EB8303D3F8D80FE3070AD50E
:100B3000F0F7E5FF640805F1340507D004F074FD13
:100B40008542FBD8ECE7F0F7D5FFF3E770BD00BFB7
:100B5000001000200D49B1F8F93F30B508224AF2E3
:100B6000010580EA030414F0010F4FEA530318BF94
:100B70006B4002F1FF3218BF9BB212F0FF024FEA46
:100B80005000EED1A1F8F93F30BD00BF00100020A9
:100B9000274B1B782DE9F041002B47D0254B1B78C4
:100BA000002B43D0244C237803F0FF07002B3DD1CA
:100BB000224B1A68821A002A38DB214A214D12780A
:100BC000D3F804E0DFF88C80013A062606FB0251D8
:100BD00006FB02524FF00A0C89885288B1FBFCF1E7
:100BE0000EF1010C18F80EE0C3F804C001FB0EF181
:100BF0001044BCF10E0F084488BF5F601860237872
:100C000003F0FF01002BFAD1012323700E4B0F4A92
:100C10001B68128A5A600E4A12685162118841F0AC
:100C2000010111801A6842F001021A60BDE8F081EA
:100C30000F3F002060450020085000205023002076
:100C40000950002010870308584500201850002044
:100C500050450020C87C03080B4A136803605368A2
:100C6000436030B59368094C83601821002301FB71
:100C700003429579AD0602D51379C37230BD0133B5
:100C80000C2BF4D1FAE700BFD77C03087488030863
:100C900070470C4B1B78DB0700D570470A4A136876
:100CA000002BFAD04FF47A7101FB03F39842F4D38E
:100CB000064B1B781BB9064B99681B690B60002318
:100CC00013607047FF280020703E0020643E002023
:100CD000F03D002070B50C4CA3689BB15A68821A95
:100CE000002A0FDB0546002603E05A68AA1A002AEC
:100CF00008DB99681E731A68A16018469047A368BC
:100D0000002BF2D170BD00BF502300202DE9F0432D
:100D100091F800C0077BDFF8A8E0077500236FEAB1
:100D20000C0C5FFA8CFC47758775C775077647769C
:100D30008776C77607774777C383038443848384A2
:100D4000C3849846142405254CFA05F303F00103E7
:100D5000002B14BF19260A26434415F0010F04EB9B
:100D600006015FFA83F889B214BFB9464FF0000953
:100D70002346C21801339BB2994282F81490F8D1ED
:100D8000013D34446B1CA4B2DED118F0010F14BF36
:100D900019250A25611989B22346C21801339BB26D
:100DA0008B421775F9D12C44A4B2631C04449BB246
:100DB00000222275AEF80C300361BDE8F08300BF5D
:100DC000502300202DE9F04FDFF898A0BAF80E303C
:100DD0000B3383B01FFA83F901F1060B4FF00108C2
:100DE0004FF0000E002711F801CB3E464D46012280
:100DF000A5F10B039BB2019108E08189ADF80210C7
:100E000001339BB289B2AB42217508D0C418002AC5
:100E1000F3D1C41801339BB2AB422275F6D103441F
:100E20000136092F019983F814E0F6B20CD0092E8F
:100E300015D008FA07F313EA0C0F14BF01220022A1
:100E40000C35ADB20137D3E709F1780959451FFADE
:100E500089F9C7D1AAF80EE003B0BDE8F08F0022EF
:100E6000EEE700BF502300202DE9F047DFF860E0F7
:100E7000BEF8103004331FFA83FC01F10908012782
:100E800011F8016BE1460025A9F1040307FA05F208
:100E90009BB23240CAB190F80CA0C41801339BB287
:100EA0004B4584F814A0F5D101350433082D1FFA01
:100EB00083F9E9D10CF1200C41451FFA8CFCDFD1FC
:100EC0000023AEF81030BDE8F0879246E5E700BF9A
:100ED00050230020436A8269D154436A0169C26B7E
:100EE00001338B4228BF002343623AB370B4EFF35F
:100EF0001183502282F31288C66B3268D20704D560
:100F0000DBB283F3118870BC7047716869B9D0E9AE
:100F10000942944218D085691544F56018D9A21A7F
:100F200072608462002280F85820326842F0010228
:100F3000DBB2326083F3118870BC7047426D136876
:100F400043F0800313607047012280F85820D7E7F0
:100F50000469A21A72608162E4E7034610B4846BEC
:100F6000D968406954B19A6C8C1A013A005D5DF8F9
:100F7000044B08BF0A46C0B29A6470471A6A805C84
:100F800001328A4228BF2246C0B21A625DF8044B81
:100F90007047C36B13B190F858007047D0E909034C
:100FA000181AB0FA80F040097047D0E909120369B5
:100FB000914238BFC9188A1AC16B013B19B14968FF
:100FC0000A449A4201D2981A704700207047836BF6
:100FD00043B1826C5B689A4291BF981AC0689B1AB1
:100FE000C0187047D0E907239A422FBFD01AC068B3
:100FF0008018C01A7047F8B522220446002102303A
:1010000024F055F80C4F00222346052104251046F4
:10101000D65D9E700132042AD9701D719871597184
:1010200003F10803F4D101232380522384F82230F2
:1010300064232384F8BD00BF8487030808B50FF03C
:101040007DFC084B1B7843B1012B0AD10649074BA5
:101050000748084A0860DA6002E0044B054ADA6093
:10106000FEE708BD0C3F0020FC9F002000ED00E0E3
:10107000EFBEADDE0400FA05024A034B1278197880
:1010800021F0B4BF0D3F00200E3F002030B50446D4
:10109000406D21710368A26823F00103036087B0EB
:1010A0006379009213F0040F4FEA03324FEA0323EF
:1010B00014BF4FF48055002503F4806302F40052FE
:1010C0000195CDE90223002511F0010305952ED1EC
:1010D000049308238D07694648BF04930AF0C0FCB7
:1010E0002079636D617900F00202002A15BF4FF488
:1010F00040324FF480324FF40034002410F0010FDE
:10110000586808BF2246CC074CBF024320EA0202BF
:101110005A609A6809074CBF42F0080222F00802A0
:101120009A601A6842F001021A6007B030BD0423C9
:1011300004930C23CEE72DE9F0415F4C636946F23E
:10114000A712C31A93422DED028B03D8BDEC028B7C
:10115000BDE8F081594B60611B6813F004032CD18A
:101160001846574A94F82410127812F0010217D04A
:10117000F1B90125C4E90A010A46084684F8245059
:101180000BB1504B1860504B1B780E2BDED1BDECD1
:10119000028B4E4B1E2158809A801980BDE8F08149
:1011A00031B1D4E90A5184F82420401B4A42E7E7D0
:1011B000D4E90A12401A5242E2E7DFF83081444E85
:1011C00098F806303788A569013BB5FBF3F59FB366
:1011D000404A9FED410A1368002B1946B8BFD91D3C
:1011E000A3EBE1031D44002D2B46B8BFEB1DDB1024
:1011F00007EE903AF8EEE77A156027EE800AF2F7EC
:1012000055FADFED367A20EE270AF2F795FAF7EE77
:10121000007A77EEC07A9FED320A236A67EE807A11
:101220009D42FDEEE77AC4ED077A3FD0013F0023EF
:1012300037802562184694E707EE905A9FED260AFC
:10124000284DF8EE677AB7EE008A27EE800AF2F7AB
:101250002DFADFED227A20EE270AF2F76DFADFEDA4
:10126000207A38EE400A20EE270A23F0A1FEB8F8D3
:101270000830DFED1D6A07EE103AE369C01AB8EED8
:10128000C77A07EE900AA7EE668AB8EEE70AD5EDB0
:10129000097AF8EEE77A20EE080A67EEA67AA7EE5A
:1012A000870A23F085FE012368625AE7002213466D
:1012B0003280104655E700BF5023002070290020DF
:1012C000FF280020742900207027002074270020A8
:1012D000F03600204C0B002008942537B1DC423E4C
:1012E000D048874A8C1D00206F12833AA42F00201B
:1012F0002DE9F8432E4B1B685B0701D4BDE8F8834A
:101300002C4C2D4D94F83090B9F1010F3CD1EB6984
:10131000284698472B69284698472B6A04F13401E0
:1013200004F138009847254AA6699179D4E90F83DA
:10133000D4E90D2008F10107AA625A1C8F4208BFA8
:101340000027032AE8622AD01D49226494F8442029
:1013500041F823004ABB04EB880804EB8703C8F874
:1013600048009A6CAB89E763B61A30440022A0614A
:1013700084F83020002BC1D0124A642B1268B8BF09
:1013800064231361BDE8F8836B6928469847AB690D
:10139000284698470122EB8984F83020EAE7084A7A
:1013A00084F8449000239060236421F043FCD2E74A
:1013B00070290020502300208C1D0020A42F002025
:1013C000A06A00204C230020A24B1B68002B46D0B3
:1013D0002DE9F04B5B6984B09847E8B19E4C41F22F
:1013E000BC43E358002B1ADC6378022B1CD0032B80
:1013F00012D141F2D853E35C2BBB41F2C443E35C0E
:101400002BBB41F20853E35C2BBB41F24C53E35C32
:1014100013B1924809F088F904B0BDE8F08B07F0E9
:10142000E1FF6378022BE2D1A3784FF00109072B8B
:10143000F2D8DFE813F05C00EB00720053001800F4
:10144000AC00B6001500864809F06EF9D5E785486E
:1014500009F06AF9D5E7844809F066F9D5E77047DD
:1014600003236370D8E72278237DDFF81C827F4E48
:10147000032A14BF4FF480778027002B00F0B2803E
:10148000012BFAD17A4B62681968D8F800004FEA4C
:10149000412C00234FF0FF31B1FBFCF112EB010BAB
:1014A00043F1000C0021614500F1020008BF5845DE
:1014B00038BF83465A466F49022008F041FC032892
:1014C00000F2C58001A353F820F000BF19140108F1
:1014D000BB15010819140108BB15010841F290530E
:1014E000E35C002B98D0644809F01EF994E70023D0
:1014F00003AD29461846092208F016F901288BD1B8
:10150000039B93F8FE21552A00F0C08041F2D4528B
:1015100002210123A15463707EE7584B00930325F9
:101520003023052256495448A5700CF07FFD73E71F
:1015300023690622652BA27033D92278032A14BFAF
:101540006FF0FF026FF07F02A3F1650303EA02036D
:1015500003F1010314BF4FF4807280229A42236189
:101560001FD2D8F80020E66802329F19974202D3B2
:1015700007F0AAFF2369434A6660D16FA76049025A
:1015800003FB01F342E9073305211660A170A2684D
:101590003649012008F0B6FA012840F013810623ED
:1015A000A3700021344808F0EBF9012840F00A81CB
:1015B000A3780133DBB2A37039E7D4E901232569AD
:1015C000991AA94288BFC4E903210328B0D0013386
:1015D000B3FBF7F207FB12320AB13B449B1A00221D
:1015E00063602275D8F8002031460232002008F0EE
:1015F000A7FB03282BD801A353F820F019140108E6
:1016000043160108191401083115010803AD41F210
:101610001C662946A0590023092208F085F80128F4
:101620007FF4FAAE0023039A2370B2F80B30B3F5BF
:10163000007F6DD041F2D45203210123A154637085
:10164000EAE6636884F814900133A3601AE7237D07
:1016500013E700BF602A0020BC6D00200883002033
:101660009483002080820020C4820020C06D00206E
:10167000EC830020C46D00204C830020657A0108B3
:1016800060C8030870830020E483002093F8FF21E2
:10169000AA2A7FF43BAFD3F8C61149B193F8C2210F
:1016A000A2F10B0001282DD902F0F702062A29D059
:1016B000D3F8D61149B193F8D221A2F10B00012839
:1016C00020D902F0F702062A1CD0D3F8E61149B15E
:1016D00093F8E221A2F10B00012813D902F0F702DE
:1016E000062A0FD0D3F8F61100293FF40FAF93F874
:1016F000F231A3F10B02012A04D903F0F703062B00
:101700007FF404AF41F21C620123A150A3707EE775
:10171000137C022B8ED192F8FE31552B8AD192F890
:10172000FF31AA2B86D1D589A7592E492F440F60A6
:10173000567B41F23061731E7F2B66503FF67AAFC5
:10174000734236EA03037FF475AF41F238617302E6
:10175000013B6350D18A01B9516A234841F22463A5
:10176000E150B2F811305B0103F2FF135B1203602A
:10177000B2F8130000B9106A49001D440D44401B23
:1017800041F2286C40F6F475B0FBF6F0A84244F83C
:101790000C0024D94FF6F475A8421CD90320207000
:1017A000D56A124A3B440B4441F22C6041F23C6141
:1017B0001278235065500AB907F0E8FDA378013389
:1017C000A37029E602287FF427AE41F2D452012308
:1017D000A354637020E6022222700025E1E7012372
:1017E000237027E7DC830020FC830020BC830020DB
:1017F00070B5244924480A784B78CD7B2349244E80
:10180000C2EB0214C2EB840203EB4304002D03EB92
:101810008403204D204C01EB430300EB420214BF34
:101820002821202133602A60216011F057F83022EE
:1018300000211A481A4C23F03AFC28680EF0A8FC44
:1018400010F0BEFF174A184B1079184AC4F8082147
:101850006421C82211FB00210022C3E90112C3E95F
:101860000322C3E90522DA6183F8202083F82120CE
:10187000FDF750F894F80E11B4F80C01BDE8704073
:101880000FF0F4BD5C290020A41000203C120020C1
:101890005C2D002058290020100E0020B0380020B8
:1018A000502300205030002084290020FC15002007
:1018B0002DE9F04F2DED028BA0F10A0387B00C4605
:1018C000E72B00F25887DFE813F066045607560747
:1018D0005607560756075607560756075607560720
:1018E0005607560756075607560756075607560710
:1018F0005607560756075607560748045607560711
:10190000560739045607560756072C04560755063E
:1019100056075607560716015607B90656073007E9
:1019200056074501560756075607A6029F02560757
:101930008C025607560725045607560756075607C2
:101940005607800256075607560756076102560784
:101950001B025607FD01E2015607560756075607B8
:10196000560756075607A0015607590156078D0519
:101970005607E3045607B604560756075607560798
:10198000780412032807D506C206560756072E010B
:1019900023015607FF05F800560756075607560756
:1019A000E800560756077A035607560756076B0393
:1019B0005403EC025607560756075607DD02560732
:1019C000CE02AC025607560756075607560756076B
:1019D000560756075607560756075607560756071F
:1019E00056077804560756075607560756075607F0
:1019F00056075607560756075607560756075607FF
:101A000056075607560756075607560756075607EE
:101A100056075607560756075607560756075607DE
:101A2000560756075607560756075607180456070F
:101A300056075607560756075607560756075607BE
:101A400056075607560756075607560756075607AE
:101A5000560756075607560756075607560756079E
:101A6000560756075607560756075607560756078E
:101A7000560756075607560756075607560756077E
:101A8000560756075607560756075607560756076E
:101A90005607F6035607EB039B03A9495223226816
:101AA000501C2060137011F8013F002BF7D101206A
:101AB00007B0BDEC028BBDE8F08FA24800220168A0
:101AC000256802EB42035B0019446E1C097A26600C
:101AD00029700168256819446E1C497A26602970AE
:101AE000016825680B4401329B7A691C052A216034
:101AF0002B70E4D1DBE7202500212046F1F7B5FD6E
:101B0000013DF9D12368904A591C21601D709FE363
:101B10008E4B08461968F1F7A8FD20460021F1F721
:101B2000BBFD0120C4E78A4D08462988F1F7B4FDC2
:101B300069882046F1F7B0FDB5F90430854AD91718
:101B400082FB0323C1EBA301204689B2F1F7A4FD78
:101B50000120ADE7804D814E05F1200795F9021077
:101B60007F4B93F906208A4203F1080300F0308688
:101B70009E42F6D10835AF42F0D198E70B68794D17
:101B8000794A6978794E581C206019702368127858
:101B9000591C21601A7023683279591C21601A700F
:101BA0002368B278591C21601A7031882046F1F7F9
:101BB00073FD318A2046F1F76FFD23680022591C1E
:101BC00021601A702368F278591C21601A7023680A
:101BD0002A79591C21601A702368EA78591C2160FF
:101BE0001A7023682A78591C21601A70698B204664
:101BF000F1F752FD698A2046F1F74EFD23682A7DF0
